:100000000C94890E0C94AA0E0C94AA0E0C94AA0EB1
:100010000C94AA0E0C94AA0E0C94AA0E0C94AA0E80
:100020000C94AA0E0C94AA0E0C94B5620C94D26295
:100030000C94AA0E0C94AA0E0C9493630C94C063B7
:100040000C94ED630C941A640C9447640C947464DF
:100050000C94A1640C94CE640C94FB640C942865FD
:100060000C94AA0E0D94B1140D94E8140C94AA0EDD
:100070000C94AA0E0C94AA0E0C94AA0E0C94AA0E20
:100080000C94AA0E0C94AA0E0C94AA0E0C94AA0E10
:100090000C94AA0E0C94AA0E0C94AA0E0D94E53F93
:1000A0000D9417400D9449400D947B400C9491F3AE
:1000B0000C94AA0E0C94AA0E0C94AA0E0C9417671A
:1000C0000C9444670C9471670C949E670C94CB67F6
:1000D0000C94F8670C9425680C9452680C947F6813
:1000E0000C94AC680C94AA0E0D94D5130D940C14BA
:1000F0000C94AA0E0C94AA0E0C94AA0E0C94AA0EA0
:100100000C94AA0E0C94AA0E0C94ACF60C94AA0EA5
:100110000C94AA0E0C94AA0E0C94AA0E0D941D3FDA
:100120000D944F3F0D94813F0D94B33F0C94AA0E54
:100130000C94AA0E0C9455650C9482650C94AF65D2
:100140000C94DC650C9409660C9436660C9463661A
:100150000C9490660C94BD660C94EA660C94AA0EFE
:100160000D9443140D947A140C94AA0E0C94AA0EB8
:100170000C94AA0E0C94AA0E0C94AA0E0C94AA0E1F
:100180000C94AA0E0C94AA0E0C94AA0E0C94AA0E0F
:100190000C94AA0E0C94AA0E0C94AA0E0C94AA0EFF
:1001A0000C945EF30C94AA0E0C94AA0E0C94AA0E56
:1001B0000C94D9680C9406690C9433690C946069AA
:1001C0000C948D690C94BA690C94AA0E0C94AA0E26
:1001D0000C94AA0E0C94AA0E0C94AA0E0D941F1542
:1001E0000D9456150C94AA0E0C94AA0E0C94AA0EFB
:1001F0000C94AA0E0C9452750C940D76630FE60FB6
:10020000750FE60F870FE60F990FB30F990FCD0FFC
:10021000CD0F9411A811BC11E211081283127012B3
:1002200083124A124A120A180A1842187F18C31871
:100230000018AC19C819051A63196319B921C3212B
:10024000CD21D721E121EB21F521FA21FF2109223E
:1002500009227D267D26842684269726BA267D2699
:10026000BA2684268426F326F326FB26FB261027AF
:100270003727F3263727FB26FB261C282728362876
:10028000512867288928CF28D828F328AF28AF28F5
:10029000F35B6A5C6A5C835B6A5C6A5C6A5C6A5C8E
:1002A0006A5C6A5C6A5C6A5C6A5C6A5C6A5C6A5C1E
:1002B0006A5C6A5C985B6A5C6A5C6A5C6A5C6A5CE1
:1002C0006A5C6A5CED5B4B5C6A5C6A5C585C6A5CAD
:1002D0006A5C6A5C6A5C6A5C6A5C065C6A5C6A5C52
:1002E000645C6A5C675C6A5C6A5C6A5C6A5C615CF0
:1002F0006A5C6A5C6A5C6A5C6A5C6A5C6A5C6A5CCE
:100300006A5C6A5C6A5C6A5C6A5C6A5C6A5C6A5CBD
:100310006A5C6A5C6A5C6A5C6A5C6A5C6A5C6A5CAD
:100320006A5C6A5C6A5C6A5C6A5C6A5C6A5C6A5C9D
:100330006A5C6A5C6A5C6A5C6A5C6A5C6A5C6A5C8D
:100340006A5C6A5CF05B267029702C702F703270CA
:1003500035703870A577B877CB77DE77F17704788A
:100360001778117D117D9C7CD37CD37C547C547C8C
:10037000D37CD37CD37CD37CD37CD37CD37CD37C05
:10038000D37CD37CD37CD37CD37CD37CD37C547C74
:10039000D37CD37CD37CD37CD37C1D825D83588279
:1003A00087825D835D835D835D835D835D835D8324
:1003B0005D835D835D835D835D835D835D835D833D
:1003C0005D835D835D835D835D835D835D835D832D
:1003D0005D835D835D835D835D835D835D835D831D
:1003E0005D835D835D835D835D835D835D835D830D
:1003F0005D835D835D835D835D835D8302835D8358
:10040000C1825D835D831D835D835D835D835D83C9
:100410005D835D835D835D835D835D835D83D0826A
:100420005D83DE82D38C038B3C8B868BEC8B378C8D
:100430004C8C7E8CA08CC18C868E138D1B8D388D40
:10044000778D8A8DD48DF68D0D8E228E818E818E44
:10045000818E818E818E818E818E818E818E818E24
:10046000398E418E4C8E618E678ECEA7D9A7ABA7F1
:10047000B7A7D9A7D9A7D9A7D9A7D9A7D9A7D9A79E
:10048000D9A7D9A7D9A7D9A7D9A7D9A7D9A7C3A782
:10049000D9A7D9A7D9A7D9A7D9A7D9A7D9A7D9A75C
:1004A000D9A7D9A7D9A7D9A7D9A7CEA7D9A7ABA785
:1004B000B7A7D9A7D9A7D9A7D9A7D9A7D9A7D9A75E
:1004C000D9A7D9A7D9A7D9A7D9A7D9A7D9A7C3A742
:1004D00030B233B284B284B284B284B284B284B211
:1004E00084B284B284B284B284B284B284B284B25C
:1004F00084B284B284B284B284B26AB284B284B266
:1005000084B284B284B284B250B284B284B284B26F
:1005100084B284B236B284B284B284B284B284B279
:1005200084B284B284B284B284B284B284B284B21B
:1005300084B284B284B284B284B26AB284B284B225
:1005400084B284B284B284B250B284B284B284B22F
:1005500084B284B236B22DB52AB53FB53FB53FB5AA
:100560003FB53FB53FB53FB53FB53FB53FB53FB5EB
:100570003FB53FB53FB53FB576B449B467B43FB575
:100580003FB5EDB430B43FB53FB53FB53FB53FB52E
:1005900058B430B53FB53FB580B43FB53FB53FB572
:1005A0003FB53FB53FB53FB53FB53FB53FB53FB5AB
:1005B0003FB53FB53FB53FB576B449B467B43FB535
:1005C0003FB5EDB430B43FB53FB53FB53FB53FB5EE
:1005D00058B430B53FB53FB580B415B758B767B715
:1005E00067B767B767B767B767B767B767B767B71B
:1005F00067B767B767B767B74CB667B703B7FDB6F6
:1006000065B60FB767B767B775B64CB667B767B764
:1006100024B759B609B75DB767B76BB61AB7F7B65F
:1006200070B667B71FB748B662B767B767B75FB648
:1006300067B767B767B767B767B767B703B7FDB699
:1006400065B60FB767B767B775B64CB667B767B724
:1006500024B759B609B75DB767B76BB61AB7F7B61F
:1006600070B667B71FB748B662B767B767B75FB608
:1006700028B63EBD2EBD30BD32BD34BD36BD38BD01
:100680003ABD5BBD4BBD4DBD4FBD51BD53BD55BD0D
:1006900057BD88BDB6BD90BDB6BD90BDB6BD90BDC1
:1006A000B6BD90BDB6BD90BDB6BDB6BDB6BDB6BDFE
:1006B000B6BDB6BDB6BD97BD9EBDAABDAABD15CF80
:1006C00044CD50CD9BCDCCCEB0CDF2CD16CE3FCECD
:1006D0009ACECBD5CBD50DD6E8D679D769D86BD9FC
:1006E00022DA6BD936DB36DB82DD82DD9EDDDFDDB3
:1006F000FFDD2EDE63DE83DE63DEB2DEE7DE3DE1BC
:1007000070E1A3E124E298E25FE356E4E0E456E41A
:10071000B4E5C5E60D94FE010D94D9020D94F102E5
:100720000D9455010D9457030D9471024E414E499D
:100730004E495459494E46CDCCCC3D0AD7233C179F
:10074000B7D13877CC2B329595E6241FB14F0A00EC
:100750000020410000C84200401C4620BCBE4CCADC
:100760001B0E5AAEC59D743235304D4F686D003248
:10077000354D4F686D003630487A003530487A0084
:100780004E6F6E2D496E740048692D4C4F004750D6
:10079000530054696D650044697374616E6365004C
:1007A0005075736820427574746F6E00496D706582
:1007B0007269616C004D657472696300494E430053
:1007C000444543004F4E004F4646005B0856084CD8
:1007D00008450839083208260815080708F407E113
:1007E00007327843495053263278444356472641CE
:1007F000435647003278496D702E204349505326A6
:1008000032784443564700506172616C6C656C20CD
:1008100043495053003278496D702E20434950535C
:100820002644435647003278496D702E2043495084
:100830005300347844435647004349505326327896
:100840004443564700327844435647004349505387
:1008500026444356470044435647004349505300FB
:10086000FA103810760FB40EF20D300D6E0CAC0B82
:10087000EA0A280AC7095B119910D70F150F530E02
:10088000910DCF0C0D0C4B0B890AC70953616D708C
:100890006C652F7365633A004552524F52202020F9
:1008A00020202000432D434950532C20522D4349F2
:1008B00050532C2000000000000000000000000049
:1008C0000000000000000000000000000000000028
:1008D0000000000000000000000000000000000018
:1008E0000000000000000000000000000000000008
:1008F00000000000000000000000000000000000F8
:1009000000000000004C6F2D434950532C204869D3
:100910002D434950532C200000000000000000002F
:1009200000000000000000000000000000000000C7
:1009300000000000000000000000000000000000B7
:1009400000000000000000000000000000000000A7
:100950000000000000000000000000000000000097
:10096000000000000000434950532C20000000000C
:100970000000000000000000000000000000000077
:100980000000000000000000000000000000000067
:100990000000000000000000000000000000000057
:1009A0000000000000000000000000000000000047
:1009B0000000000000000000000000000000000037
:1009C00000000000000000414356474C506F6C2C63
:1009D00020414356474C526D732C20414356475299
:1009E000506F6C2C204143564752526D732C20009F
:1009F00000000000000000000000000000000000F7
:100A000000000000000000000000000000000000E6
:100A100000000000000000000000000000000000D6
:100A20000000000000000000522D44435647204FB4
:100A30006E2C204C2D44435647204F6E2C204C6F7B
:100A40002D43495053204F6E2C2048692D43495067
:100A500053204F6E2C20522D44435647204F66663C
:100A60002C204C2D44435647204F66662C204C6F5B
:100A70002D43495053204F66662C2048692D434929
:100A80005053204F66662C2000522D444356472079
:100A90004F66662C204C2D44435647204F66662CEB
:100AA000204C6F2D43495053204F66662C204869D7
:100AB0002D43495053204F66662C20522D444356F7
:100AC00047204F6E2C204C2D44435647204F6E2C10
:100AD000204C6F2D43495053204F6E2C2048692DD8
:100AE00043495053204F6E2C2000432D434950530F
:100AF000204F6E2C20522D43495053204F6E2C20F6
:100B0000432D43495053204F66662C20522D4349B4
:100B10005053204F66662C200000000000000000AB
:100B200000000000000000000000000000000000C5
:100B300000000000000000000000000000000000B5
:100B40000000000000000000000000432D43495059
:100B500053204F66662C20522D43495053204F6638
:100B6000662C20432D43495053204F6E2C20522D8C
:100B700043495053204F6E2C20000000000000001D
:100B80000000000000000000000000000000000065
:100B90000000000000000000000000000000000055
:100BA000000000000000000000000000522D44433F
:100BB0005647204F6E2C204C6F2D43495053204FE9
:100BC0006E2C2048692D43495053204F6E2C2052E3
:100BD0002D44435647204F66662C204C6F2D4349C9
:100BE0005053204F66662C2048692D4349505320AE
:100BF0004F66662C2000000000000000000000008E
:100C000000000000000000000000000000522D4421
:100C1000435647204F66662C204C6F2D4349505356
:100C2000204F66662C2048692D43495053204F665B
:100C3000662C20522D44435647204F6E2C204C6F7B
:100C40002D43495053204F6E2C2048692D43495065
:100C500053204F6E2C200000000000000000000018
:100C600000000000000000000000000000004C6FC9
:100C70002D43495053204F6E2C2048692D43495035
:100C800053204F6E2C204C6F2D43495053204F66FC
:100C9000662C2048692D43495053204F66662C200E
:100CA0000000000000000000000000000000000044
:100CB0000000000000000000000000000000000034
:100CC0000000000000000000000000000000004CD8
:100CD0006F2D43495053204F66662C2048692D43A1
:100CE000495053204F66662C204C6F2D434950537A
:100CF000204F6E2C2048692D43495053204F6E2CB5
:100D000020000000000000000000000000000000C3
:100D100000000000000000000000000000000000D3
:100D200000000000000000000000000000000000C3
:100D3000522D44435647204F6E2C204C2D44435691
:100D400047204F6E2C20462D44435647204F6E2C93
:100D500020422D44435647204F6E2C20522D4443B1
:100D60005647204F66662C204C2D44435647204F53
:100D700066662C20462D44435647204F66662C203D
:100D8000422D44435647204F66662C200000000049
:100D900000522D44435647204F66662C204C2D446C
:100DA000435647204F66662C20462D444356472025
:100DB0004F66662C20422D44435647204F66662CD2
:100DC00020522D44435647204F6E2C204C2D444337
:100DD0005647204F6E2C20462D44435647204F6ED9
:100DE0002C20422D44435647204F6E2C20000000FB
:100DF0000000522D44435647204F6E2C204C2D446A
:100E0000435647204F6E2C2043495053204F6E2CA1
:100E100020522D44435647204F66662C204C2D44CB
:100E2000435647204F66662C2043495053204F6657
:100E3000662C200000000000000000000000000000
:100E400000000000000000000000000000000000A2
:100E5000000000522D44435647204F66662C204C1C
:100E60002D44435647204F66662C2043495053205B
:100E70004F66662C20522D44435647204F6E2C203F
:100E80004C2D44435647204F6E2C2043495053204D
:100E90004F6E2C2000000000000000000000000049
:100EA0000000000000000000000000000000000042
:100EB00000000000522D44435647204F6E2C204C1A
:100EC0002D44435647204F6E2C20522D4443564705
:100ED000204F66662C204C2D44435647204F6666B3
:100EE0002C200000000000000000000000000000B6
:100EF00000000000000000000000000000000000F2
:100F000000000000000000000000000000000000E1
:100F10000000000000522D44435647204F66662CC7
:100F2000204C2D44435647204F66662C20522D44BA
:100F3000435647204F6E2C204C2D44435647204F9C
:100F40006E2C2000000000000000000000000000E7
:100F50000000000000000000000000000000000091
:100F60000000000000000000000000000000000081
:100F7000000000000000522D44435647204F6E2CC5
:100F80002043495053204F6E2C20522D4443564746
:100F9000204F66662C2043495053204F66662C2014
:100FA0000000000000000000000000000000000041
:100FB0000000000000000000000000000000000031
:100FC0000000000000000000000000000000000021
:100FD00000000000000000522D44435647204F6699
:100FE000662C2043495053204F66662C20522D44D6
:100FF000435647204F6E2C2043495053204F6E2CB0
:1010000020000000000000000000000000000000C0
:1010100000000000000000000000000000000000D0
:1010200000000000000000000000000000000000C0
:101030000000000000000000522D44435647204F9E
:101040006E2C20522D44435647204F66662C2000BC
:101050000000000000000000000000000000000090
:101060000000000000000000000000000000000080
:101070000000000000000000000000000000000070
:101080000000000000000000000000000000000060
:10109000000000000000000000522D44435647208D
:1010A0004F66662C20522D44435647204F6E2C200D
:1010B0000000000000000000000000000000000030
:1010C0000000000000000000000000000000000020
:1010D0000000000000000000000000000000000010
:1010E0000000000000000000000000000000000000
:1010F0000000000000000000000043495053204F52
:101100006E2C2043495053204F66662C200000006F
:1011100000000000000000000000000000000000CF
:1011200000000000000000000000000000000000BF
:1011300000000000000000000000000000000000AF
:10114000000000000000000000000000000000009F
:101150000000000000000000000000434950532040
:101160004F66662C2043495053204F6E2C200000C0
:10117000000000000000000000000000000000006F
:10118000000000000000000000000000000000005F
:10119000000000000000000000000000000000004F
:1011A000000000000000000000000000000000003F
:1011B00000000000000000000000000044656C61B9
:1011C000792054696D653B0046696C65204E616D00
:1011D000653A2000436861696E6167652C200000F4
:1011E0004C6F63616C54696D652C204C6F63616C4E
:1011F000444D592C204C61742D4465672C204E536E
:101200002C204C6F6E2D4465672C2045572C2046B2
:101210006978537461742C204E756D5361742C2061
:1012200050444F502C20416C745F4D2C2043686B10
:101230002C20436F6D6D00000000000000000000D6
:10124000000000000000000000000000000000009E
:10125000000000000000000000000000004C6F6370
:10126000616C54696D652C204C6F63616C444D5901
:101270002C204C61742D4465672C204C61742D4DDD
:10128000696E2C204C61742D5365632C204E532CB9
:10129000204C6F6E2D4465672C204C6F6E2D4D6970
:1012A0006E2C204C6F6E2D5365632C2045572C20DF
:1012B000466978537461742C204E756D5361742C9B
:1012C0002050444F502C20416C745F4D2C204368BB
:1012D0006B2C20436F6D6D000000484558434F5202
:1012E0004445522043414C4942482E545854000032
:1012F000007777772E636174682D746563682E6359
:101300006F6D0000000000004C494D4954454420D9
:101310003930352D3835372D313035300000004328
:101320004154484F44494320544543484E4F4C4F45
:1013300047590000007B702C30302C662C007B70ED
:101340002C30302C657D007B702C30302C6F7D0074
:10135000456E746572204143564720282746272052
:10136000666F722046726F6E742C202742272066AB
:101370006F72204261636B290A0D20616E642073D5
:101380007570706C79203332302B363430207369AD
:101390006E65776176652077697468205065616B4A
:1013A000546F5065616B20766F6C74616765206F58
:1013B0006620302E385600456E7465722053434FB8
:1013C000504520766F6C7461676520696E206D569C
:1013D00020284E4E4E4E4E2900456E7465722043B5
:1013E00049505320766F6C7461676520696E206D7B
:1013F000562A313020284E4E4E4E4E2900456E74EE
:101400006572204443564720766F6C74616765208F
:10141000696E206D562A313020284E4E4E4E4E2990
:1014200000571450144C144814441440143114310F
:1014300014432D53474E44205B352D3430565D0008
:10144000432D4200432D4600432D5200432D4C00B6
:10145000522D53474E4400432D53474E44002061C4
:101460006E6420656E74657220766F6C746167655A
:1014700020696E206D562A313020284E4E4E4E4E39
:101480002900506C6561736520636F6E6E656374CF
:1014900020004572726F722C206D697373696E67DC
:1014A00020414443206E756D2028302D3729000AD5
:1014B0000D5363616C696E6743616C6962204F66AE
:1014C000667365743A20004572726F722C20656EE7
:1014D00074657220766F6C7461676520696E206D2B
:1014E000562A313020284E4E4E4E4E29009B157CF8
:1014F0001566155A1536152315FB1443535B302F0B
:10150000312F322F332F345D5B76767676765D2001
:101510002D204443205363616C696E672043616CE6
:101520006962004342202D20426174746572792003
:1015300043616C696200435A5B302F312F322F3385
:101540002F345D202D204443205A65726F4F66660C
:101550007365742043616C69620056202D20566EBD
:10156000756D626572004C5B696E785D5B4F4E2FE6
:101570004F46465D202D204C65647300416E6E2001
:101580002D2052656164204144433120666F7220F2
:101590006E6E207365636F6E64730041202D205260
:1015A0006561642041444331004552524F52004F1F
:1015B0004B00434154482054454348204845584334
:1015C0004F52444552205630302E39380001000227
:1015D0000003000400050006000A000C000F0014C0
:1015E000001E003C007800B400F0002C01680100EF
:1015F0000000000B0002000100B80B0F270100647F
:10160000006801100E010010271027102710271066
:101610002710270100010001000100F8010100016D
:101620000002000100F401000000000100000000C1
:10163000000A00F1D8000001000100C800000064A9
:1016400000640064006400640064000000000000A6
:1016500000000050FE00000000000000000100003B
:101660000000000100000000000A0000000100016D
:1016700000020058020000FA00FA00FA00FA0078AE
:1016800000780000000000000001000000010001DF
:10169000000000000001000100008000190080002F
:1016A00019008000190080001900800019008000D6
:1016B00019008000190080001900000100FF03E6F6
:1016C00000E600F916EB16DD16D616244A42494EFE
:1016D0002C39342C3100244A5341564500244A41C8
:1016E00053432C47504753412C3100244A41534324
:1016F0002C4750524D432C3100244A4153432C4730
:10170000504747412C310024504D544B3636372A30
:1017100033350024504D544B3331342C302C312C84
:10172000302C312C312C302C302C302C302C302CD7
:10173000302C302C302C302C302C302C302C302CC9
:10174000302A323900756E6C6F67206C62616E648E
:10175000747261636B7374617461006C6F67206C89
:1017600062616E64747261636B7374617461206F23
:101770006E74696D6520313000756E6C6F67207016
:101780007372706F7361006C6F6720707372706F2B
:101790007361206F6E74696D65203130006461740F
:1017A000756D20757365720020302E3020302E301C
:1017B00020302E3020302E300075736572646174D5
:1017C000756D2000646174756D207767733834001F
:1017D000756E6C6F67206770616C6D006C6F672051
:1017E0006770616C6D206F6E74696D6520313000BB
:1017F00059184A183B182C1824180B18FE17245097
:1018000047524D432C2C2C39362C00245047524D36
:10181000432C412C2C3130302C2C2C2C2C2C2C2CCF
:101820002C2C2C00245047524D4345002450475245
:101830004D4F2C5047524D542C3000245047524DA0
:101840004F2C5047524D462C3100245047524D4F9B
:101850002C47504753562C3000245047524D4F2CA4
:101860002C3400BA18AB189C188D187E186F1844C9
:101870005A203D20000000000000000000004459F4
:10188000203D20000000000000000000004458201F
:101890003D2000000000000000000000466C617464
:1018A000203D2000000000000000004D616A6F72C2
:1018B00041203D20000000000000535450522044BD
:1018C0004154554D2E54585400061AF919EC19DF9D
:1018D00019D219C519B819AB199E1991198419771C
:1018E000196A195D1950194319361929191C190F4C
:1018F000190219F518414356473220524D53203DE5
:101900002000414356473120524D53203D20004294
:10191000415454202043616C203D2000414320204D
:10192000205343616C203D200041432020205A4336
:10193000616C203D200041444337205653636C20A6
:101940003D200041444337205A43616C203D200034
:1019500041444336205653636C203D2000414443AC
:1019600036205A43616C203D2000414443352056C7
:1019700053636C203D200041444335205A43616C41
:10198000203D200041444334205653636C203D20C9
:101990000041444334205A43616C203D20004144BF
:1019A0004333205653636C203D2000414443332091
:1019B0005A43616C203D200041444332205653631A
:1019C0006C203D200041444332205A43616C203D4D
:1019D000200041444331205653636C203D20004198
:1019E000444331205A43616C203D20004144433040
:1019F000205653636C203D200041444330205A431D
:101A0000616C203D200046696C6520496E646578F4
:101A1000203D2000B41C9E1C881C721C5C1C461CB3
:101A2000301C1A1C041CEE1BD81BC21BAC1B961BC3
:101A3000801B6A1B541B3E1B281B121BFC1AE61A38
:101A4000D01ABA1AA41A8E1A781A621A454E44008D
:101A50000000000000000000000000000000000086
:101A60000000444356472044656665637420566110
:101A70006C203D200000000044435647204465662A
:101A800065637420456E203D2000000000005379FE
:101A90006E632054797065203D2000000000000036
:101AA00000000000434950532052616E6765202BAF
:101AB0002F2D3556203D2000000047505320436F06
:101AC0006F726420696E20444D53203D2000000059
:101AD0004C6F63616C47505354696D654F66667314
:101AE0006574203D20004143204672657175656E26
:101AF0006379203D200000000000000042726F6BFF
:101B0000656E5769726520416C61726D203D2000E1
:101B100000004C6F7720506F7420416C61726D2013
:101B20003D20000000000000496E70757420496D72
:101B3000706564616E6365203D20000000004443D1
:101B400056474D44656C4F4E203D2000000000007C
:101B500000000000444356474D44656C4F46462004
:101B60003D20000000000000000043495053324D6A
:101B700044656C4F4E203D20000000000000000036
:101B800043495053324D44656C4F4646203D20003A
:101B900000000000000043495053314D44656C4F34
:101BA0004E203D200000000000000000434950533B
:101BB000314D44656C4F4646203D2000000000003A
:101BC0000000537461727457697468203D200000EE
:101BD00000000000000000004F666654696D65203B
:101BE0005B6D7365635D203D200000000000546F55
:101BF00074616C4379636C65205B7365635D203D44
:101C00002000000054696D652056616C7565203DAB
:101C100020000000000000000000436861696E6160
:101C2000676520446972656374696F6E203D2000AA
:101C3000537461727420436861696E616765203D09
:101C400020000000000044697374616E63652056D3
:101C5000616C7565203D2000000000004D656173DA
:101C60007572656D656E7420556E697473203D20C4
:101C7000000053746F7261676520416374696F6E11
:101C8000203D2000000000005375727665792054D5
:101C9000797065203D2000000000000000004F70BA
:101CA000657261746F72204E616D65203D20000089
:101CB00000000000537572766579204E616D6520D5
:101CC0003D20000000000000000054532D5453201C
:101CD0004F4E203D200054532D5453204F46462054
:101CE0003D20004E4557205453204F4E203D2000AC
:101CF0004E4557205453204F4646203D2000545314
:101D0000204F4E203D20005453204F4646203D207A
:101D1000000011241FBECFEFCDBFDFE5DEBF00E026
:101D20000CBF1DE2A0E0B0E2EEE2F3E902E00BBF7F
:101D300002C007900D92A83EB107D9F722E5A8EEA0
:101D4000BDE201C01D92A832B207E1F70E94433BF9
:101D50000D9495490C940000CF93DF93CDB7DEB777
:101D60002B97CDBFDEBFBE016F5F7F4F80E092E05B
:101D70000F94FD40AE01485F5F4F68E080E092E065
:101D80000F9459418A819B819F789B8395E09D8325
:101D9000817E8A831C82BE016F5F7F4F80E092E06C
:101DA0000F94AD4081E0888788E18987AE01485F64
:101DB0005F4F68E080E092E00F94204180E092E085
:101DC0000F940E3F2B96CDBFDEBFDF91CF910895CC
:101DD0009FB7F894E0E0F2E08081806280839FBF4B
:101DE0000895009781F02091060223FF0EC02091F4
:101DF0003C0230913D02FC012083318388E08093D6
:101E0000060281E0089580E0089580E00895CF9271
:101E1000DF92EF92FF92CF93DF930097D1F061159D
:101E20007105C9F0EB01FC01A081B18128EE33E01E
:101E30000F94AD446B017C0183E10E9452B89B0179
:101E4000AC01C701B6010F9458442883398381E05F
:101E500003C080E001C080E0DF91CF91FF90EF9060
:101E6000DF90CF900895EAEDF6E31082118214829C
:101E7000158212821382168217828BE00E9476B836
:101E8000672B682B692B19F41092E23603C081E0AE
:101E90008093E236EAEDF6E3118612860895CF9339
:101EA000DF93EC01892B09F491C0862F90E0FC01AF
:101EB0003197EB30F10508F089C08827E250FF4FD9
:101EC0008F4F0D9496448091E236811107C088812E
:101ED00099818093DE369093DF3678C08A819B812A
:101EE0008093DE369093DF3671C08091E2368111A7
:101EF00007C08A819B818093DE369093DF3666C06F
:101F00008E819F818093DE369093DF365FC0809113
:101F1000E236811107C08C819D818093DE369093DB
:101F2000DF3654C08A859B858093DE369093DF36FA
:101F30004DC08091E23681110BC088819981EAED14
:101F4000F6E3848395838A819B81868397833EC051
:101F50008C819D81EAEDF6E3848395838E819F8158
:101F60008683978333C08091E23681110BC08A81CA
:101F70009B81EAEDF6E3848395838C819D81868342
:101F8000978324C0EAEDF6E3888599858483958359
:101F90008A859B858683978319C08091E23681115B
:101FA0000BC08C819D81EAEDF6E3848395838E815D
:101FB0009F81868397830AC0EAEDF6E38C859D8531
:101FC000848395838E859F8586839783DF91CF91C8
:101FD0000895EAEDF6E3848195818083918386817B
:101FE0009781828393830895EAEDF6E381E0818708
:101FF00012860895EAEDF6E311861286089580911F
:10200000E436089583E10E9476B8672B682B692B2C
:1020100019F08091E336089580E00895CF92DF9221
:10202000EF92FF926B01072E000CEE08FF08C2161C
:10203000D306E406F5067CF486179707E4F0092E2C
:10204000000CAA0BBB0BE1E0281739074A075B0716
:10205000ACF4E0E013C06C01092E000CEE08FF08A0
:10206000C216D306E406F50644F0E1E068177907E6
:102070002CF4E0E003C0E0E001C0E0E08E2FFF9030
:10208000EF90DF90CF900895FF920F931F93CF931F
:10209000DF93CAEDD6E30EED16E3F12CE991F99149
:1020A000309719F1AF010F2E000C660B770BDB0197
:1020B000CA0177231CF40196A11DB11DB595A79502
:1020C000979587959A01AB01280F391F4A1F5B1F0F
:1020D000BF01FF2314F46F5F7F4F759567958A8169
:1020E0009B819CDF813009F0F394C017D107B1F6D2
:1020F000FF2011F079DF01C07DDF6BDFDF91CF9131
:102100001F910F91FF900895EAEDF6E381E090E0D2
:10211000A0E0B0E08787908BA18BB28B838B948BF0
:10212000A58BB68B178A1386148615861686108E95
:102130000895EAEDF6E381E0878B108E0895EAEDCD
:10214000F6E3178A108E08958091F236089584E19F
:102150000E9476B8672B682B692B19F08091F136B5
:10216000089580E00895EAEDF6E387859089A189D6
:10217000B289838B948BA58BB68B83859485A5853B
:10218000B6858787908BA18BB28B08956093E536D7
:102190007093E6368093E7369093E83608958F92F1
:1021A0009F92AF92BF92CF92DF92EF92FF92EAEDB1
:1021B000F6E3C388D488E588F68887859089A18965
:1021C000B289C816D906EA06FB0691F48090E53676
:1021D0009090E636A090E736B090E836C4DFC81499
:1021E000D904EA04FB0411F4A4DF04C0A8DF02C090
:1021F000BADFFCCFFF90EF90DF90CF90BF90AF9011
:102200009F908F9008958BE10E9476B86093F3368B
:102210007093F4368093F5369093F636A7EFB6E3D5
:10222000EAEDF6E382EE96E31D9211A212A2329637
:102230008E179F07C9F7EAEDF6E311A612A60895D7
:1022400081E090910337911101C080E008958AE107
:102250000E9476B8672B682B692B39F081E090914A
:102260000337911103C080E0089580E008950F9333
:102270001F938B019C018091F3369091F436A091CD
:10228000F536B091F6360097A105B10529F1880F12
:10229000991FAA1FBB1FAC01BD01440F551F661F2C
:1022A000771F440F551F661F771F840F951FA61FAA
:1022B000B71FB901A80133233CF444275527BA01BD
:1022C000401B510B620B730B21E084179507A60787
:1022D000B7071CF020E001C020E0822F1F910F9172
:1022E00008950F931F93CF93DF93009709F40BC1C9
:1022F000AAEDB6E35D961C925D975E961C925E9782
:102300005F961C925F9790961C92462F50E0FA01C0
:102310003297EA30F10508F0F6C0EC018827E75F54
:10232000FE4F8F4F0D9496448091E236811108C084
:102330006C817D818E819F819ADF8093F736E3C027
:10234000688179818A819B8192DF8093F736DBC037
:102350008091E236811108C0688579858A859B85E0
:1023600086DF8093F736CFC0688179818A819B812F
:102370007EDF8093F736C7C08091E236811111C0AD
:10238000688579858A859B8572DF0AED16E3F801F9
:10239000858F6C857D858E859F8569DFF801868FA9
:1023A000B2C0688179818A819B8161DF0AED16E381
:1023B000F801858F6C817D818E819F8158DFF801C6
:1023C000868FA1C08091E236811111C06C857D8518
:1023D0008E859F854CDF0AED16E3F801858F6889AD
:1023E00079898A899B8943DFF801868F8CC068814F
:1023F00079818A819B813BDF0AED16E3F801858FA5
:102400006C817D818E819F8132DFF801868F7BC058
:102410008091E23681111FC0688979898A899B89F8
:1024200026DF0AED16E3F801858F6C897D898E8998
:102430009F891DDFF801868F688D798D8A8D9B8D30
:1024400016DFF801878F6C8D7D8D8E8D9F8D0FDF50
:10245000F80180A358C0688179818A819B8107DF58
:102460000AED16E3F801858F6C817D818E819F8155
:10247000FEDEF801868F688579858A859B85F7DE83
:10248000F801878F6C857D858E859F85F0DEF8014C
:1024900080A339C08091E236811111C068897989A1
:1024A0008A899B89E4DE0AED16E3F801858F6C8941
:1024B0007D898E899F89DBDEF801868F24C0688143
:1024C00079818A819B81D3DE0AED16E3F801858F3D
:1024D0006C817D818E819F81CADEF801868F13C059
:1024E0008091E236811108C06C857D858E859F853F
:1024F000BEDE8093F73607C0688179818A819B812F
:10250000B6DE8093F736DF91CF911F910F9108953A
:10251000843040F5EAEDF6E341A552A5242F30E0E2
:10252000082E02C0359527950A94E2F720FF0AC0CD
:10253000252F30E0082E02C0359527950A94E2F742
:1025400020FD10C021E030E0B90102C0660F771F06
:102550008A95E2F7CB01EAEDF6E3462B41A7809599
:10256000852382A70895843090F421E030E0A9010A
:1025700002C0440F551F8A95E2F7CA018095EAED23
:10258000F6E391A5982391A792A5892382A70895A0
:10259000BF92CF92DF92EF92FF920F931F93CF9350
:1025A000DF9307EF16E3CAEDD6E36E017801B12C95
:1025B000F70181917F01F60121A190E0820F911D29
:1025C00022A1820F911D039719F48B2DA1DF02C068
:1025D0008B2DC9DFB394F2E0CF0ED11C84E0B8128A
:1025E000E7CF22EE36E389A18AA3F80181918F011A
:1025F00089A32296C217D307B1F7DF91CF911F911C
:102600000F91FF90EF90DF90CF90BF9008958430AE
:1026100060F42091033730E0A90102C05595479539
:102620008A95E2F7CA018170089580E008958430A8
:1026300060F42091043730E0A90102C05595479518
:102640008A95E2F7CA018170089581E00895843087
:1026500000F5662379F0EAEDF6E321E030E0A90128
:1026600002C0440F551F8A95E2F7CA0192A5892B33
:1026700082A70895EAEDF6E321E030E0A90102C067
:10268000440F551F8A95E2F7CA01809592A58923C8
:1026900082A70895CF93833009F128F4813031F077
:1026A000823061F02CC0883008F129C08091F13669
:1026B000882329F181E08093F23621C0C1DD88238F
:1026C000F1F061E080E0C3DF61E081E0C0DF61E064
:1026D00082E0BDDF61E083E0BADF11C08091E336C4
:1026E000882369F081E08093E43609C0CCEFC80FFD
:1026F0008C2F8DDF882319F061E08C2FA8DFCF911C
:102700000895009781F0FC01DC01AE5BBD4F808134
:102710008C936083643021F481E00C9469F7089510
:1027200080E00C9469F70895009719F0FC0180810E
:10273000089580E008950F931F93CF93DF931F9226
:10274000CDB7DEB7009709F4BBC08C0181E0D8019A
:102750008C9311961C92119712961C9212971396B5
:102760001C92139714961C92149715961C92159709
:10277000169682E1E7EFF3E201900D928A95E1F778
:10278000C80148960E9474BEF801808D8783818DB0
:102790008087828D8187838D8287CE0101960E94FA
:1027A00095BE89818B3429F481E0D8015C968C93A5
:1027B00002C0F801148E80E00E9452B8673EF3E038
:1027C0007F078105910514F59F938F937F936F93F6
:1027D00083EE90E29F938F93C801C5969F938F934A
:1027E0000F94C346D801D5968C91D59750968C936B
:1027F0005097D6968C91D69751968C935197D796A1
:102800008C91D79752968C93CDBFDEBFD8015D9641
:102810001C925D975E961C925E97D1961C92D19702
:10282000D2961C92F801EB5CFD4F1082319610821B
:1028300031961082319681E0808331961082118228
:1028400012821382349681E090E0A0E0B0E08083B1
:102850009183A283B383349610823196D8018C91F0
:102860008083E751F24086E0DF011D928A95E9F707
:10287000E85EFD4F108211823296108211823296EC
:102880001082118232961082118232961082319615
:1028900010823296108231961082319610823196D3
:1028A00010823196108231961082319610821182F8
:1028B00012821382349610823196108231961082E1
:1028C0000F90DF91CF911F910F910895009741F0E4
:1028D000613021F421E0FC0121AB0895FC0111AA33
:1028E0000895009719F0FC0181A9089580E00895EA
:1028F000009741F0613021F421E0FC0122AB089502
:10290000FC0112AA0895009719F0FC0182A908950C
:1029100080E008958F929F92AF92BF92DF92EF92E4
:10292000FF920F931F93CF93DF934115510509F445
:102930006BC08A017B01C82F0E9423BDD82F8C2F2A
:102940000E9440BDD82EDD2309F460C0882309F41D
:102950005FC08D2F0E9452B84B015C018D2D0E94EB
:1029600052B8672B682B692B39F4F8011082118259
:102970001282138280E04DC09701280D391D032E6D
:10298000000C440B550BC63050F4A0E1B7E20F9495
:10299000B344F801608371838283938309C0A8EEF6
:1029A000B3E00F94B344F80160837183828393830F
:1029B0008D2D0E9452B89B01AC01F801608171819C
:1029C000828193810F947A4488279927DC01821BA6
:1029D000930BA40BB50BF80180839183A283B3837F
:1029E0008C2F0E94F6BFF80180809180A280B38076
:1029F000DC01CB01880D991DAA1DBB1D808391832D
:102A0000A283B38381E005C080E003C080E001C001
:102A100080E0DF91CF911F910F91FF90EF90DF90B9
:102A2000BF90AF909F908F900895CF93DF930097C2
:102A300009F460C0EC010F948309813091F58C8317
:102A40000E9450F48823F9F08091053D811119C04E
:102A500089E0E9EEF0E2A7E4B2E401900D928A95F4
:102A6000E1F7E7E4F2E401900020E9F73197AF01E4
:102A70004754524421E067E472E487E697E30F94F9
:102A8000D9110E9489F40E9453F4882399F185E3B7
:102A900096E40E9483C50E944DF48A830E949AF4B2
:102AA00029C01C820F94AF098823F9F08091053D5D
:102AB000811119C089E0E2EFF0E2A7E4B2E40190ED
:102AC0000D928A95E1F7E7E4F2E401900020E9F73E
:102AD0003197AF014754524421E067E472E487E63E
:102AE00097E30F94D9110F94B2090F949B098111A8
:102AF0000F949E09DF91CF9108950F931F93CF9369
:102B0000DF93009709F463C0EC010F94FA0B88235C
:102B100081F18B8181115BC08091053D811126C0BF
:102B20000F94C309182F0E944DF41F921F931F92F8
:102B30008F9384E091E29F938F9307E412E41F93B5
:102B40000F930F94C346F80101900020E9F73197E5
:102B5000AF014754524420E0B80187E697E30F9451
:102B6000D9118DB79EB708968DBF9EBF81E08B832C
:102B70002EC08B81813059F51B828091053D8111DA
:102B800026C00F94C309C82F0E944DF41F92CF9303
:102B90001F928F938BEF90E29F938F93C7E4D2E4C1
:102BA000DF93CF930F94C34609900020E9F7219754
:102BB000AE014754524420E067E472E487E697E3AD
:102BC0000F94D9118DB79EB708968DBF9EBFDF9128
:102BD000CF911F910F910895CF92DF92EF92FF92C4
:102BE0000F931F93CF93DF93009709F4AAC0611549
:102BF000710509F4A6C08B01EC010E9421C5882350
:102C000009F49FC00F94420A6B017C010F94E70BFB
:102C100086E10E9476B8AB01BC018FED9AE30E9479
:102C2000B7C5D701C6010197A109B109883E9340F4
:102C3000A105B10508F03FC00E94A8B1823088F11B
:102C40008091053D81112DC00E944DF41F928F93FC
:102C500080919D511F928F93FF92EF92DF92CF92BE
:102C600087E191E29F938F930F2EF7E4EF2EF2E42A
:102C7000FF2EF02DFF92EF920F94C346F7010190C3
:102C80000020E9F73197AF014754524421E0B701E2
:102C900087E697E30F94D9118DB79EB70C968DBF39
:102CA0009EBF2CE433E446E655E460EA74E4C801D0
:102CB0000E942AD143C0D701C601895E9340A10971
:102CC000B10984369105A105B105C0F586E693E406
:102CD0000E9419C5811132C08091053D811125C026
:102CE000FF92EF92DF92CF9283E291E29F938F93D4
:102CF0000F2EF7E4EF2EF2E4FF2EF02DFF92EF926D
:102D00000F94C346F70101900020E9F73197AF0116
:102D10004754524421E0B70187E697E30F94D91155
:102D20008DB79EB708968DBF9EBF2CE433E446E670
:102D300055E460EA74E4C8010E942AD1CE010E94E1
:102D40003AC5DF91CF911F910F91FF90EF90DF90E7
:102D5000CF900895FC01892B39F0118689E0DF01BD
:102D60001D928A95E9F712860895FC01892B41F09E
:102D7000118689E0DF011D928A95E9F71286138694
:102D800008950F931F93CF93DF93C8E0D7E300E636
:102D900017E3CE01DFDF2B96C017D107D1F78CE9FF
:102DA0009AE3E3DF88EA9AE3E0DFDF91CF911F91B6
:102DB0000F910895FC01892B31F081E092859130CB
:102DC00019F080E0089580E008951F93CF93DF937A
:102DD000CDB7DEB76097CDBFDEBF9C01FE01319657
:102DE000AE014F5E5F4F21933193255F3F4FE41754
:102DF000F507C9F7892B31F110E010C0E12FF0E0A1
:102E0000EE0FFF1F81E090E08C0F9D1FE80FF91F70
:102E100080819181CFDF8823D1F01F5F0F94E70C71
:102E2000181760F382E00E9476B86B3069F48091E5
:102E3000A73A882359F081E09091B33A911107C0E5
:102E400080E005C080E003C081E001C080E06096C2
:102E5000CDBFDEBFDF91CF911F910895CF92DF925A
:102E6000EF92FF920F931F93CF93DF93CDB7DEB70F
:102E70002597CDBFDEBF19821A821B821C824115A5
:102E8000510559F16A017B01182FCA0163DFAE01B8
:102E90004F5F5F4FB701812F3DDD8823C9F0098166
:102EA0001A812B813C814BE0BE016B5F7F4FC601D5
:102EB0000F94F918F60101900020E9F73197EC1909
:102EC000FD09D6011996EC93199781E01A968C9317
:102ED00069817A818B819C8103C060E070E0CB01C5
:102EE0002596CDBFDEBFDF91CF911F910F91FF904F
:102EF000EF90DF90CF9008958F929F92AF92BF9204
:102F0000EF92FF920F931F93CF93DF930097A1F05F
:102F10006115710589F0142F7B01EC010E949CF76B
:102F20004B015C01113009F431D9950184014BE06A
:102F3000B701CE010F944B17DF91CF911F910F91E5
:102F4000FF90EF90BF90AF909F908F900895AF92B9
:102F5000BF92CF92DF92EF92FF920F931F93CF9386
:102F6000DF93CDB7DEB76097CDBFDEBF8C01CE015A
:102F700001967C014096F70161937193655F7F4FE5
:102F8000E817F907C9F70115110509F46BC282E0CA
:102F90000E9476B8D62E96E0D91206C0C8010F94CA
:102FA0004208811165C239C38FEF8D0D823030F434
:102FB000C8010F944208811107C02FC3C8010F94A4
:102FC0004208882309F429C380E2E6E1FEE3DF0139
:102FD0001D928A95E9F780E1E5E7F9E3DF011D92AB
:102FE0008A95E9F78D2D90E0FC013197EB30F105E2
:102FF00008F03AC28827ED5EFE4F8F4F0D9496443D
:1030000058010F2EF6E1CF2EFEE3DF2EF02D01E06A
:1030100010E00EC10F943F08C82E49815A81F80173
:10302000608171811BDF0F2EF6E1EF2EFEE3FF2E94
:10303000F02DD7016D937D938D939C9313974B81C6
:103040005C81F801628173818C2D08DFD7011496B1
:103050006D937D938D939C931797B2E0DB1206C21C
:103060008091163E9091173EA091183EB091193E66
:103070008093753990937639A0937739B0937839E6
:1030800081E0CBC258010F2EF6E1CF2EFEE3DF2EFA
:10309000F02D01E010E00BC01F5F0F5FE2E0EE0ECD
:1030A000F11CF2E0AF0EB11C84E0C80ED11C11235C
:1030B00009F4FBC1123009F4EAC1D7014D915C91CA
:1030C000F5016081718180E0C9DED6016D937D9349
:1030D0008D939C9313970430F8F28091163E909153
:1030E000173EA091183EB091193E80937539909388
:1030F0007639A0937739B093783981E08EC2580140
:103100000F2EF6E1CF2EFEE3DF2EF02D01E010E0D2
:103110000BC01F5F0F5FB2E0EB0EF11CE2E0AE0EE2
:10312000B11CF4E0CF0ED11C112309F4DBC1123025
:1031300009F4CAC1D7014D915C91F501608171819B
:1031400082E08CDED6016D937D938D939C931397D3
:103150000430F8F2E5E7F9E3A6E1BEE34D915D91B5
:103160006D917C911397408351836283738314968E
:103170008D919D910D90BC91A02D84839583A68304
:10318000B78381E04AC258010F2EF6E1CF2EFEE34D
:10319000DF2EF02D01E010E00BC01F5F0F5FB2E0EB
:1031A000EB0EF11CE2E0AE0EB11CF4E0CF0ED11C30
:1031B000112309F4B8C1133009F4A3C1113009F483
:1031C000A2C1143009F4A1C1D7014D915C91F50160
:1031D0006081718180E042DED6016D937D938D9395
:1031E0009C9313970630C8F2E5E7F9E3A6E1BEE346
:1031F0004D915D916D917C911397408351836283D2
:10320000738314968D919D910D90BC91A02D848314
:103210009583A683B78381E000C21F5F0F5FB2E092
:10322000EB0EF11CE2E0AE0EB11CF4E0CF0ED11CAF
:10323000112309F499C1143009F484C1812F8B7FC3
:10324000813009F481C1823009F480C1D7014D91E8
:103250005C91F5016081718185E000DED6016D939E
:103260007D938D939C9313970830B8F2E5E7F9E3CB
:10327000A6E1BEE34D915D916D917C9113974083E2
:1032800051836283738314964D915D916D917C910E
:103290001797448355836683778318964D915D9184
:1032A0006D917C911B9740875187628773871C962D
:1032B0008D919D910D90BC91A02D84879587A687B7
:1032C000B78781E0AAC158010F2EF6E1CF2EFEE3A9
:1032D000DF2EF02D01E010E00BC01F5F0F5FB2E0AA
:1032E000EB0EF11CE2E0AE0EB11CF4E0CF0ED11CEF
:1032F000112309F458C1143009F445C1812F8B7F83
:10330000813009F442C1D7014D915C91F501608192
:10331000718180E0A3DDD6016D937D938D939C93A5
:1033200013970830D0F2E5E7F9E3A6E1BEE34D914B
:103330005D916D917C911397408351836283738378
:1033400014968D919D910D90BC91A02D84839583B1
:10335000A683B78381E061C1680106E11EE35E01D7
:10336000B9E0AB0EB11CF701419151917F01D6013B
:103370006D917D916D0180E071DDF8016193719334
:10338000819391938F01EA14FB0469F781E045C1B1
:1033900058010F2EF6E1CF2EFEE3DF2EF02D01E0D7
:1033A00010E00BC01F5F0F5FF2E0EF0EF11C82E038
:1033B000A80EB11C94E0C90ED11C112309F402C15E
:1033C000133009F40DC1D7014D915C91F501608175
:1033D000718180E043DDD6016D937D938D939C9345
:1033E00013970630F8F28091163E9091173EA09107
:1033F000183EB091193E8093753990937639A09319
:103400007739B093783981E008C158010F2EF6E181
:10341000CF2EFEE3DF2EF02D01E010E00BC01F5F8A
:103420000F5FB2E0EB0EF11CE2E0AE0EB11CF4E077
:10343000CF0ED11C112309F4E2C0D7014D915C914C
:10344000F5016081718181E0123009F480E006DDD0
:10345000D6016D937D938D939C9313970430F8F26E
:1034600081E0DBC080E0D9C080E0D7C081E0D5C07A
:1034700080E2E6E1FEE3DF011D928A95E9F780E153
:10348000E5E7F9E3DF011D928A95E9F7B9CDF70188
:1034900040815181D5016D917C9183E0DFDCF601A3
:1034A0006083718382839383F7CDD7014D915C91C3
:1034B000F5016081718183E0D1DCD6016D937D934C
:1034C0008D939C931397E8CDF70140815181D501ED
:1034D0006D917C9183E0C2DCF6016083718382830D
:1034E000938317CED7014D915C91F5016081718175
:1034F00083E0B4DCD6016D937D938D939C931397F9
:1035000008CE83E003C082E001C082E0F701408181
:103510005181D5016D917C91A1DCF60160837183AD
:10352000828393833ACED7014D915C91F5016081FE
:10353000718183E093DCD6016D937D938D939C9391
:1035400013972BCE83E003C082E001C084E0F70133
:1035500040815181D5016D917C9180DCF6016083C1
:1035600071838283938359CED7014D915C91F5018C
:103570006081718183E072DCD6016D937D938D93C0
:103580009C9313974ACE83E001C082E0F70140810B
:103590005181D5016D917C9161DCF601608371836D
:1035A000828393839ACED7014D915C91F50160811E
:1035B000718183E053DCD6016D937D938D939C9351
:1035C00013978BCEF70140815181D5016D917C918C
:1035D00083E044DCF6016083718382839383E2CECF
:1035E000D7014D915C91F5016081718183E036DCFA
:1035F000D6016D937D938D939C931397D3CEF70152
:1036000040815181D5016D917C9180E027DCF601EC
:10361000608371838283938302CF6096CDBFDEBFC8
:10362000DF91CF911F910F91FF90EF90DF90CF909E
:10363000BF90AF9008950F941006882329F00F943F
:10364000210684E0809327060895CF93DF930097A7
:1036500099F1EC0188818130A8F0833018F0863030
:1036600019F010C0E8DF25C08091280682FD03C054
:1036700084E0809325060F94AA058823D1F00F9447
:10368000BB0517C00F94AA05882399F00F94BB05BA
:1036900084E0809327060DC08D8181110DC00F94A9
:1036A000EE05882349F00F94FF0584E080932706F8
:1036B00003C08881863081F7DF91CF9108950E9401
:1036C0005BC90F94C70A20E137E240E050E00F9455
:1036D0005844672B682B692BE1F40E945BC9813049
:1036E00019F40C946FC808950E945BC9823021F4CC
:1036F00081E00C945EC908950E945BC9833019F47F
:103700000C9464CB08950E945BC9843011F40C942E
:10371000B8CB08950F931F93CF93DF931F921F92FF
:10372000CDB7DEB719821A820097B9F08C010E94DA
:10373000725190E006969E012F5F3F4F43E060E09C
:10374000800F911F0F94AA15882339F049815A815F
:1037500060E070E080E00E9461B80F900F90DF9110
:10376000CF911F910F9108959F92AF92BF92CF92E8
:10377000DF92EF92FF920F931F93CF93DF931F92ED
:10378000CDB7DEB7009709F44BC05C0182E00E9420
:1037900076B8962E8501095D1F4FBE016F5F7F4F82
:1037A000C8010E943ED5882391F0F501C7A0D0A49E
:1037B000E1A4F2A489E00E9476B8AB01BC0101EE5D
:1037C00016E421ED36E489810F94E20A17C0BE01A8
:1037D0006F5F7F4FC8010E9418DDF501C7A0D0A41C
:1037E000E1A4F2A489E00E9484B8AB01BC0101EE1F
:1037F00016E421ED36E489810F94E20AFBE09F1282
:103800000BC0F50147A150A561A572A589EC96E40E
:103810000F94C70D81E005C00F94310E81E001C007
:1038200080E00F90DF91CF911F910F91FF90EF906B
:10383000DF90CF90BF90AF909F900895CF92DF928E
:10384000EF92FF920F931F93CF93DF931F92CDB709
:10385000DEB7009779F18C01BE016F5F7F4F8796CD
:103860000E9483DF882399F0F801C7A0D0A4E1A4C7
:10387000F2A489E00E9476B8AB01BC0101EE16E427
:1038800021ED36E489810F94E20A81E014C0F80149
:10389000C7A0D0A4E1A4F2A489E00E9484B8AB013F
:1038A000BC0101EE16E421ED36E489810F94E20AB1
:1038B00081E001C080E00F90DF91CF911F910F91C7
:1038C000FF90EF90DF90CF90089589E10E9476B845
:1038D000623059F482E00E9476B8673041F0693076
:1038E00031F0613021F081E0089580E0089580E0BA
:1038F000089589E10E948CF8623059F482E00E94B8
:103900008CF8673041F0693031F0613021F081E0AE
:10391000089580E0089580E008952F923F924F929D
:103920005F926F927F928F929F92AF92BF92CF924F
:10393000DF92EF92FF920F931F93CF93DF93CDB758
:10394000DEB76497CDBFDEBFB82E8B017A0189E167
:103950000E9476B8A62E0115110509F46CC280915B
:10396000053D882339F00F2EF7E6CF2EF7E3DF2E43
:10397000F02D06C00F2EFEE6CF2EF8E3DF2EF02D41
:1039800082E08A1508F4A12C8BE7F801808383E795
:1039900081838CE28283F2E3BF1207C082E38A0D47
:1039A000F80183838CE284830BC0F801B3828CE23C
:1039B0008483F0E3BF1609F4E8C182E3B8120FC2B2
:1039C00088E097E3FE0132969E012E5E3F4F819381
:1039D00091930B962E173F07D1F788E08983E11466
:1039E000F10469F086E0F701D801159601900D9277
:1039F0008A95E1F70F2EFBE0FF2EF02D04C00F2E6D
:103A0000F5E0FF2EF02DF801EF0DF11D8CE2808323
:103A100082E00E9476B8762E872D072C000C990B39
:103A20009F937F9280E291E29F938F93F394C801DA
:103A30008F0D911D9F938F930F94C346F8010190B2
:103A40000020E9F73197E01BF10B7F01FF24F8011B
:103A5000EE0DFF1D118221E0A701B801C6010F94F0
:103A6000D9110F900F900F900F900F900F908091A1
:103A7000053D811112C01A8A21E040E050E0BE01EC
:103A80006E5E7F4F87E697E30F94D91120E0A70180
:103A9000B80187E697E30F94D91191E09A1508F4DD
:103AA000F9C01982912C0F2EFCE28F2EF02DF80117
:103AB0003196EB8BFC8B0F2EF5E04F2EFDE35F2E46
:103AC000F02D5BC00F94E70C6980861509F45CC08B
:103AD000F8018082E62CF12CF701EE0FFF1F81E048
:103AE00090E08C0F9D1FE80FF91FA180B280F501B7
:103AF000418550E0B5018B899C890F949546F5016D
:103B000081856894332431F8380E8F5FF801E80F0F
:103B1000F11D8082F7013196EE0FFF1F81E090E0EA
:103B20008C0F9D1FE80FF91FA180B280F501418520
:103B300050E0B501C801830D911D0F949546F50124
:103B4000E1843E0C639463946982E32CF12CF801C8
:103B5000EE0DFF1D118221E0A701B801C6010F94EF
:103B6000D911F2018081811107C020E0A701B801BD
:103B700087E697E30F94D91193940F94E70C8695F9
:103B8000981608F49FCF53C1FBE07F12CFC0198273
:103B900080E00F2EFCE25F2EF02D48019FEF891A86
:103BA000990A0F2EF0E32F2EFCE23F2EF02D0F2E60
:103BB000F5E06F2EFDE37F2EF02DF8015082E82E08
:103BC000F12CF701EE0FFF1FEE0DFF1DEE0FFF1F93
:103BD000EE0FFF1FE456F54C82858C3419F08235C8
:103BE00031F00CC0F4012082318212820FC081E3D7
:103BF0009CE2F40180839183128208C085E0E5E3B2
:103C0000F1E2D40101900D928A95E1F7F80101905B
:103C10000020E9F74E2E401A5701AA0CBB1CB50133
:103C20006E0D7F1D660F771F660F771F6456754CEC
:103C3000FB01418550E0C801840D911D0F9495460C
:103C4000F501EE0DFF1DEE0FFF1FEE0FFF1FE456F7
:103C5000F54CE1844E0CE42CF12CF801EE0DFF1D27
:103C6000118221E0A701B801C6010F94D911F30117
:103C70008081811107C020E0A701B80187E697E3A2
:103C80000F94D911E98081E08E0D8983823008F488
:103C900094CF4CC01982612C0F2EFCE25F2EF02DC8
:103CA0004801FFEF8F1A9F0A0F2EF5E0AF2EFDE3BC
:103CB000BF2EF02D36C00F94E70C79808715B1F137
:103CC000F8015082E72DF0E0EE0FFF1F81E090E059
:103CD0008C0F9D1FE80FF91FE180F280F7014185ED
:103CE00050E0B701C4010F949546F701E184E394D5
:103CF00073947982F12CF801EE0DFF1D118221E001
:103D0000A701B801C6010F94D911F5018081811175
:103D100007C020E0A701B80187E697E30F94D91107
:103D200063940F94E70C8695681628F20F2EFCE238
:103D3000FF2EF02DF801F08284E00E9476B8605DDD
:103D4000F8016183F28240E0BE016F5F7F4FC801DE
:103D50000396D2D8898193E0980FF801E90FF11DFD
:103D60009DE790838C5FE82EF12CF801EE0DFF1D8E
:103D7000118221E0A701B801C6010F94D9118091E9
:103D8000053D882309F445C056C00F2EFFE9EF2EEC
:103D9000F4E4FF2EF02DF701408150E068E674E472
:103DA000C80105960F949546F701808195E0980F1C
:103DB000F801E90FF11D9DE790838A5FE82EF12C51
:103DC000F801EE0DFF1D118221E0A701B801C60127
:103DD0000F94D9118091053D81112DC011C021E0B2
:103DE00045E050E0B801C6010F94D9118091053D1E
:103DF000811121C0F0E3BF120FC045E050E002C0C6
:103E00004E2D5F2D20E0B80187E697E30F94D9117E
:103E100012C04E2D5F2D02C045E050E021E0B801F8
:103E200087E697E30F94D91106C01982B1CE8BE0D3
:103E300078127CCFFACF6496CDBFDEBFDF91CF91F1
:103E40001F910F91FF90EF90DF90CF90BF90AF90B8
:103E50009F908F907F906F905F904F903F902F90AA
:103E60000895CF93892B81F00E948050CAE00E9470
:103E700043510E947D50882321F00E94935081116C
:103E800005C0C150A1F703C0C0E001C0C1E08C2F44
:103E9000CF91089589E10E9476B8611104C00E9413
:103EA00064F4882371F081E04091A2515091A351B4
:103EB0006091A4517091A551452B462B472B09F0D9
:103EC00080E008958F929F92AF92BF92CF92DF923F
:103ED000EF92FF920F931F93CF93DF930097A9F177
:103EE000EC0186E00E9476B84B015C0184E00E9400
:103EF00076B8162F87E00E9476B8062F812F0E9491
:103F000080F70E949CF76B017C0186169706A80635
:103F1000B906D9F0AB01BC0186E00E94CEB9882376
:103F2000A1F00E9429F7B701A60186E00E946CB8B3
:103F3000B701A60186E00E949FF8602F812F0E94A2
:103F400080F768E0CE010E948113DF91CF911F912D
:103F50000F91FF90EF90DF90CF90BF90AF909F9028
:103F60008F90089582E10E9476B828E0E4EDF1E5B3
:103F7000DF01322F1D923A95E9F7ECEDF1E5DF0113
:103F80001D922A95E9F721E030E0672B682B692B19
:103F900011F420E030E0F901E153FF4D80818560AC
:103FA000EAE9F1E582AF83AF81E00895009761F01F
:103FB000613031F4FC01EB5CFD4F21E0208308957A
:103FC000FC01EB5CFD4F108208950097B1F0FC01FD
:103FD00080818430A1F40F941A0A823039F089E18B
:103FE0000E9476B8672B682B692B59F00F94F7095C
:103FF00091E0811107C090E005C090E003C090E01F
:1040000001C090E0892F08950F931F93CF93DF9302
:104010008C01EB01209709F442C01882892B19F119
:1040200089E10E9476B8F80180818130C0F0833048
:1040300018F08530D0F013C0611106C02097B9F098
:1040400087E4888380E02EC06150623090F0209732
:1040500091F087E4888380E025C0209771F082E4A6
:10406000888380E01FC080E01DC081E01BC080E02D
:1040700019C081E017C080E015C080E013C081E066
:1040800011C080E00FC089E10E9476B8F8018081FC
:10409000813018F3833080F2853088F3DECF892BAE
:1040A00091F7EFCFDF91CF911F910F910895009776
:1040B00039F0FC0180818150843020F481E0089542
:1040C00080E0089580E00895009751F0FC01808120
:1040D000813040F0843010F0853021F481E0089583
:1040E00080E0089580E00895CF92DF92EF92FF92F2
:1040F000CF93DF93009709F45FC0EC0183E00E9447
:1041000076B86B017C01AB01BC0155276627772788
:1041100083E00E94CEB9882309F44BC08C2DFE01A8
:10412000EA5CFD4FC082813021F1823009F044C049
:1041300088E00E9476B8FE01E85CFD4F6083AB0129
:10414000BC0155276627772788E00E94CEB98111E8
:1041500005C081E0FE01E85CFD4F8083FE01E95C63
:10416000FD4F1082C75CDD4F188219821A821B82B4
:1041700023C087E00E9476B8F62E84E00E9476B8CD
:10418000862F6F2D0E9480F785E00E9476B80E94EE
:1041900031F8FE01E35CFD4F60837183828393837A
:1041A0000E9449F7C75CDD4F188219821A821B8270
:1041B00003C0CA5CDD4F1882DF91CF91FF90EF9072
:1041C000DF90CF900895009761F1FC01E95CFD4F0D
:1041D000208131963081321710F021111BC0FC0173
:1041E000E95CFD4F315030833296408151816281CC
:1041F0007381403821E5520721E06207710598F488
:104200004F5F5F4F6F4F7F4F408351836283738354
:1042100081E00895FC01E95CFD4F2150208380E09E
:10422000089580E0089580E008950F931F93CF9341
:10423000DF93009741F1EC010E9460F7FE01E35C1F
:10424000FD4F008111812281338160177107820740
:104250009307D8F00E9449F7FE01E75CFD4F80818B
:104260009181A281B381803821E5920721E0A207E4
:10427000B10568F40196A11DB11D80839183A283CD
:10428000B38381E005C080E003C080E001C080E02E
:10429000DF91CF911F910F910895CF93DF930097F6
:1042A00009F43DC0FC01EB5CFD4F20812223B9F1F4
:1042B000EC018BDE813021F4CB5CDD4F18822FC006
:1042C00089E10E9476B861111AC00F941A0A8130F0
:1042D00031F1823089F4DEDD882309F10F94D409AD
:1042E000CB5CDD4F188286E693E40E9413C585E31C
:1042F00096E40E943AC513C00F94080A10C0CADDA4
:10430000882369F00F94D409CB5CDD4F188286E6D0
:1043100093E40E9413C585E396E40E943AC5DF91B9
:10432000CF910895FF920F931F93CF93DF93611561
:10433000710509F47CC04115510509F478C08A0162
:10434000EB01F82E82E10E948CF821E0672B682BAC
:10435000692B09F420E08F2D90E0FC013197EB30C0
:10436000F10508F05BC08827E25EFE4F8F4F0D9489
:1043700096441882E22FF0E0E153FF4D8081856082
:10438000F801808354C083E08883E22FF0E0E1539A
:10439000FF4D8081F80180834AC01882E22FF0E04F
:1043A000E153FF4D80818160F801808340C083E04C
:1043B0008883E22FF0E0E153FF4D8081F801808394
:1043C00036C01882E22FF0E0E153FF4D808181601A
:1043D000F80180832CC083E08883E22FF0E0E15372
:1043E000FF4D8081F801808322C0188285E0F801AA
:1043F00080831DC0188281E0F801808318C0188274
:10440000E22FF0E0E153FF4D80818160F80180836D
:104410000EC0188281E0F801808309C01882E22F63
:10442000F0E0E153FF4D80818560F8018083DF91EA
:10443000CF911F910F91FF9008958F929F92AF920D
:10444000BF92CF92DF92EF92FF920F931F93CF9381
:10445000DF93892B09F486C089E00E9476B89B011E
:10446000AC01A8EEB3E00F94B3446B017C010F9450
:104470002B0AC616D706E806F90609F475C0C70167
:10448000B60128EE33E040E050E00F945844F22E9D
:10449000D22F2E3108F06AC0213009F469C00F9480
:1044A0002B0A28EE33E040E050E00F945844822F6E
:1044B000F21638F46F2D0F942544C92F992309F46F
:1044C0005CC00F94C309E82E6D2F0F942544D92F9B
:1044D000892F90E08E0D911DCA970CF04BC08D2E48
:1044E000912CA12CB12C0F94420A162F072FD82EF5
:1044F000C92EA8EEB3E0A50194010F94B3444F2D4B
:104500000F94700AC091053DC11136C00F94420A44
:104510009F938F937F936F93CF92DF920F931F930D
:104520001F92DF931F92EF928AE391E29F938F9302
:1045300007E412E41F930F930F94C346F801019010
:104540000020E9F73197AF014754524421E0B80108
:1045500087E697E30F94D9118DB79EB740968DBF2C
:104560009EBF0BC0C0E009C0C0E007C0C1E005C0ED
:10457000C0E003C0C1E001C0C0E08C2FDF91CF914B
:104580001F910F91FF90EF90DF90CF90BF90AF9071
:104590009F908F900895EF92FF920F931F93CF9368
:1045A000DF932091053D222339F00F2EF7E6EF2E01
:1045B000F7E3FF2EF02D06C00F2EFEE6EF2EF8E3F8
:1045C000FF2EF02D0097D1F1EC018BE7888388E670
:1045D00089838CE28A8392E69B838C837F936F939B
:1045E00085E791E29F938F93CE0105969F938F93DA
:1045F0000F94C346FE0101900020E9F73197EC1BB0
:10460000FD0B8F01112721E0A801BE01C7010F9406
:10461000D9110E94A8B10F900F900F900F900F909A
:104620000F90873059F48091053D811107C021E03A
:10463000A801BE0187E697E30F94D911DF91CF91CE
:104640001F910F91FF90EF9008958F929F92AF92DC
:10465000BF92CF92DF92EF92FF920F931F93CF936F
:10466000DF93009709F470C02091053D222339F0B3
:104670000F2EF7E6EF2EF7E3FF2EF02D06C00F2EDC
:10468000FEE6EF2EF8E3FF2EF02DEC018BE788839A
:1046900088E689838CE28A8393E79B838C8304EB8F
:1046A0001AE3F801848C0E94AE9C982EA090043DE1
:1046B000B090013DF801C280D0800E9464F41F9246
:1046C0008F921F929F921F92AF921F92BF921F9242
:1046D000CF921F92DF921F928F93F80185811F92D4
:1046E0008F9384811F928F9383811F928F938AE58A
:1046F00091E29F938F93CE0105969F938F930F9492
:10470000C346FE0101900020E9F73197EC1BFD0B39
:104710008F01112721E0A801BE01C7010F94D91113
:104720008DB79EB748968DBF9EBF8091053D811184
:104730000BC0A80142505109BE016F5F7F4F21E0BD
:1047400087E697E30F94D911DF91CF911F910F91D5
:10475000FF90EF90DF90CF90BF90AF909F908F90A1
:104760000895FF920F931F93CF93DF9300D01F9272
:10477000CDB7DEB70F943206882349F00F94430675
:104780000E94E80E8CEE90E460DF80E057C0CE011E
:1047900001960E94F10E882309F450C01091A806DA
:1047A00000916806F0902806BE016D5F7F4FCE0134
:1047B00001960E94070F882309F43FC00E94B4B1FC
:1047C0008823A1F18091053D811130C0F0FAFF24CA
:1047D000F0F81F92FF92029501701F920F9316FB43
:1047E000112710F91F921F938A818F9389818F93CC
:1047F0008C818F938B818F9389E791E29F938F9325
:1048000007E412E41F930F930F94C346F80101903D
:104810000020E9F73197AF014754524421E0B80135
:1048200087E697E30F94D911CDBFDEBF6B817C8102
:104830008CEE90E4B0DE81E001C081E02496CDBF33
:10484000DEBFDF91CF911F910F91FF9008958823D4
:1048500021F081E08093043D08951092043D089575
:104860000F931F93CF93DF936115710571F000973C
:1048700061F0EB018C010F945406882331F00F9402
:104880006506BE01C8010E94B98ADF91CF911F91D0
:104890000F910895CF93DF93009751F0EC010F949F
:1048A000A006882329F0CE010E94FB8C0F94B1064C
:1048B000DF91CF910895009791F0FC01ED5BFD4FE2
:1048C0002FEF3FE720833183329620E030E82083CA
:1048D00031833296108211823296108211820895AD
:1048E0000F93CF93DF930097A1F0662371F0EA0155
:1048F000FC01E55BFD4F81E08083C9010F94390C19
:10490000602FCE010E94B19C04C0FC01E55BFD4F0D
:104910001082DF91CF910F910895EF92FF920F9344
:104920001F93CF93DF931F921F92CDB7DEB70097EF
:1049300009F458C06115710509F454C0FC0121A99E
:10494000211104C022A9222309F44CC08B017C014F
:10495000FC0111AA12AA0E9444100E94CF100E94CA
:10496000C812F70143A954A9B7016B5C7F4F9E01A0
:104970002F5F3F4FC8010F94BA3AC8010F94683CAB
:10498000F701E85AFD4FD701AE5ABD4F8C91808395
:10499000319611968C918083F70123A934A98981DE
:1049A0009A812817390719F00E945E9D02C00E9463
:1049B000EE9CE8E2F1E4808190E0DC01A85DBE4B72
:1049C00025853685880F991FFC01E85DFE4B4181E6
:1049D00052811F960C9161E0C70182DF0E944D8FCA
:1049E0000F949F0C0F900F90DF91CF911F910F911B
:1049F000FF90EF9008950F931F93CF93DF9300974D
:104A000009F448C06115710509F444C08B01EC013B
:104A1000FC01E55BFD4F80818823C1F1DB018C91B6
:104A2000882341F10F94550C8823A1F1F80160818E
:104A300061506083611108C00E94239D0E94109DF7
:104A4000C55BDD4F188226C070E0F801E60FF71F46
:104A5000D8011D962D913C911E97660F771FA60FCA
:104A6000B71F11964D915C911297078561E0CE01B9
:104A700037DF10C00F94550C882361F00E94239DEE
:104A80000E94109DC55BDD4F188204C00E94239DCB
:104A90000E94109DDF91CF911F910F9108958F92E9
:104AA0009F92BF92CF92DF92FF920F931F93CF936B
:104AB000DF93009709F4DAC06115710509F4D6C0D7
:104AC0002091053D222309F4C0C0C7E6D7E3BFC04B
:104AD0008B014C010E94A710B82E0E942711D82EDE
:104AE0000E940210C82E8D2D90E08B0D911D8C0D13
:104AF000911D892B71F4F401E45BFD4F80818130BD
:104B000009F4B4C081E0808380E090E00F946C0CE5
:104B1000ADC0F401E45BFD4F8081823009F43EC0FA
:104B2000BB2051F00E94A410811108C061E0CE01A9
:104B30000E94258F01E003C000E001C000E0CC200E
:104B400009F48AC00E94FF0F811186C063E0CE0184
:104B50000E94258F01E080C0DD2081F0812F0E941E
:104B60000713882359F0812F0E941713811106C063
:104B700064E0610FCE010E94258F01E01F5F1430B9
:104B800059F7002309F472C0E401C45BDD4F82E0F1
:104B9000888384EF91E00F946C0C68C00F94880CAC
:104BA000882309F463C0BB2009F45DC00E94A410EF
:104BB000811159C00E94759DCC2009F44FC0FF247B
:104BC000F39401C0F12C0E94FF0F811149C00E9493
:104BD000759D16C0D0E0C0E0DD2069F08D2F0E94E9
:104BE0000713882341F08D2F0E941713811103C0F2
:104BF0000E94739DC1E0DF5FD43071F7CC23E1F0F8
:104C000084EF91E00F946C0CD8018C9190E0F80146
:104C1000E80FF91F1D962D913C911E97880F991F43
:104C2000A80FB91F11964D915C911297078561E00D
:104C300084EB9AE355DE1AC0F401E45BFD4F8081FA
:104C40008230A1F481E0808311C0CEE6D8E3FC017C
:104C50002081243059F43CCF10E07ECFFF24F39420
:104C6000F110CECFB7CFC110ADCFB4CFDF91CF9180
:104C70001F910F91FF90DF90CF90BF909F908F90EA
:104C80000895009721F0FC01E45BFD4F60830895D7
:104C9000CF93DF930097C1F0EC01198218820E9434
:104CA000791C813031F482E0888389E1898391E045
:104CB00006C0CE010E94B6E091E0811190E081E053
:104CC000992319F080E001C080E0DF91CF91089531
:104CD000CF93892B09F44CC082E00E9476B8862FCE
:104CE00090E0FC013297EA30F10508F043C08827D4
:104CF000E75DFE4F8F4F0D94964440E050E0BA01BF
:104D000080E00E94C8BF37C040E050E0BA0180E0B8
:104D10000E94C8BFC82F40E050E0BA0181E00E9465
:104D2000C8BFC80F81E0C23031F180E024C040E04C
:104D300050E0BA0180E00E94C8BFC82F40E050E0B8
:104D4000BA0181E00E94C8BFC80F40E050E0BA013C
:104D500082E00E94C8BFC80F40E050E0BA0183E083
:104D60000E94C8BFC80F81E0C43029F080E003C0B2
:104D700080E001C080E0CF910895CF92DF92EF9262
:104D8000FF92843098F4E82FF0E0EE0FFF1FEE0F53
:104D9000FF1FEB58F64CC080D180E280F3800E9468
:104DA00098BF6C197D098E099F0903C060E070E00F
:104DB000CB01FF90EF90DF90CF900895CF93892B98
:104DC00009F453C082E00E9476B8862F90E0FC017F
:104DD0003297EA30F10508F04AC08827ED5CFE4FB3
:104DE0008F4F0D94964480E0C8DFAB01BC0180E09A
:104DF0000E94C8BF3DC080E0C0DFAB01BC0180E0C5
:104E00000E94C8BFC82F81E0B8DFAB01BC0181E0C0
:104E10000E94C8BFC80F81E0C23051F180E028C0B5
:104E200080E0ABDFAB01BC0180E00E94C8BFC82FAF
:104E300081E0A3DFAB01BC0181E00E94C8BFC80FC5
:104E400082E09BDFAB01BC0182E00E94C8BFC80FBB
:104E500083E093DFAB01BC0183E00E94C8BFC80FB1
:104E600081E0C43029F080E003C080E001C080E030
:104E7000CF910895883009F485C028F4833041F03B
:104E8000853079F1A6C08A50823008F453C0A1C0A1
:104E9000EAE9F1E5868D978DA0A1B1A1428D538DF0
:104EA000648D758D841B950BA60BB70B8639910508
:104EB000A105B10508F48FC046A157A160A571A551
:104EC00082A193A1A4A1B5A1481B590B6A0B7B0B2E
:104ED00081E0463951056105710508F483C080E021
:104EE0000895EAE9F1E582A193A1A4A1B5A1468DB7
:104EF000578D60A171A1841B950BA60BB70B86394A
:104F00009105A105B10508F468C046A557A560A99B
:104F100071A982A593A5A4A5B5A5481B590B6A0B39
:104F20007B0B81E0463951056105710508F45AC0D3
:104F300080E00895EAE9F1E582A193A1A4A1B5A1D9
:104F4000468D578D60A171A1841B950BA60BB70BE5
:104F500086399105A105B10508F441C042A953A9BC
:104F600064A975A986A597A5A0A9B1A9481B590B45
:104F70006A0B7B0B81E0463951056105710590F1A3
:104F800080E00895EAE9F1E5868D978DA0A1B1A1B1
:104F9000428D538D648D758D841B950BA60BB70BBD
:104FA00086399105A105B105E0F042A553A564A598
:104FB00075A586A197A1A0A5B1A5481B590B6A0BA1
:104FC0007B0B81E0463951056105710558F080E0A1
:104FD000089580E0089581E0089581E0089581E0DA
:104FE000089581E00895CF9382E10E9476B8C1E0F0
:104FF000672B682B692B09F4C0E082E00E9476B829
:1050000088E0E4EDF1E5DF01982F1D929A95E9F72C
:10501000ECEDF1E5DF011D928A95E9F7862F90E02E
:10502000FC013197EB30F10508F0EFC08827E35C15
:10503000FE4F8F4F0D949644EC2FF0E0E153FF4D5F
:1050400080818560EAE9F1E582AF83AFE8C0EC2FAB
:10505000F0E0E153FF4D8081EAE9F1E582AF83AFF3
:1050600083E08093DC518093DD51D9C083E002DF7F
:10507000EC2FF0E0E153FF4D908121E0811101C060
:1050800020E0822F892BEAE9F1E582AF84AF83E04B
:105090008093DC518093DE51892F816083AF85AF8F
:1050A000BEC0EC2FF0E0E153FF4D8081EAE9F1E56D
:1050B00082AF84AF93E09093DC519093DE5183AF45
:1050C00085AF82E08093DD518093DF51A8C085E0F9
:1050D000D1DEEC2FF0E0E153FF4D208191E0811112
:1050E00001C090E0892F822BEAE9F1E582AF85AF1C
:1050F00093E09093DC519093DF5183AF86AF82E0D1
:105100008093DD518093E051822F816084AF87AF1F
:1051100086C0EC2FF0E0E153FF4D8081EAE9F1E534
:1051200082AF86AF93E09093DC519093E05183AFD0
:1051300087AF92E09093DD519093E15184AF8093DB
:10514000DA5194E09093DE519093E25185AF8093D1
:10515000DB5185E08093DF518093E35160C0862F5F
:1051600089DE91E0811101C090E0892F8F70EAE91A
:10517000F1E582AF86AF93E09093DC519093E051DC
:1051800083AF87AF82E08093DD518093E15181E06E
:1051900084AF8093DA5195AF9093DB5140C0EAE938
:1051A000F1E585E082AF84AF87E083AF85AF37C09C
:1051B00088E060DE91E0811101C090E0EC2FF0E02A
:1051C000E153FF4D8081892BEAE9F1E582AF85AF9C
:1051D00083E08093DC518093DF5191E093AF96AFF1
:1051E00084AF87AF1CC0EC2FF0E0E153FF4D80810E
:1051F0008160EAE9F1E582AF84AF83AF85AF81E0FA
:105200008093DD518093DF510AC0EC2FF0E0E15331
:10521000FF4D80818560EAE9F1E582AF83AF81E0EF
:10522000CF9108951F93CF93DF930097D9F1EC01AD
:1052300019AA1AAA0E94C11687E00E9476B8162FF2
:1052400084E00E9476B8862F612F0E9480F789E162
:105250000E9476B8613071058105910521F481E0E5
:105260000F94590A03C080E00F94590A0E94651CEC
:10527000813031F4CE010E941E1C0E94B21F04C076
:10528000CE010E94B41BAFDE0F94EA0CCE010E9447
:1052900074200F94750B0E94330F0E9484100E949B
:1052A00003111982DF91CF911F910895CF93DF935E
:1052B000009791F0FC012081243071F4EC010E94F0
:1052C000621FCE01AFDF0F94E6091092003D63E04C
:1052D000CE010E9481131982DF91CF910895882316
:1052E00021F081E08093053D08951092053D0895D9
:1052F0008091053D0895AF92BF92CF92DF92EF92D9
:10530000FF920F931F93CF93DF93DC01009709F473
:105310005AC04115510509F458C02115310509F449
:1053200056C0FA01C081D0E0F901008110E061159A
:10533000710561F0FC017C01E60EF71E9191C90F29
:10534000D11D0C0F1D1FEE16FF06C1F7F9017B01E1
:105350006D01DA01CC930083F601E60FF71F8CE2B2
:1053600080838BE181835B01A2E0AA0EB11CAC0CAF
:10537000BD1C8C2F82958F700F948D15F501808345
:105380005701F3E0AF0EB11CAC0CBD1C8C2F8F701D
:105390000F948D15D5018C93E7012496CC0DDD1D5E
:1053A000802F82958F700F948D158883D701159665
:1053B000E601CA0FDB1F802F8F700F948D15888335
:1053C000C701069605C0CB0103C0CB0101C0CB01CC
:1053D000DF91CF911F910F91FF90EF90DF90CF90D1
:1053E000BF90AF9008952F923F924F925F926F922D
:1053F0007F928F929F92AF92BF92CF92DF92EF9265
:10540000FF920F931F93CF93DF93CDB7DEB76197D2
:10541000CDBFDEBF7C016B013A01490189E10E94E9
:1054200076B8562E82E00E9476B8162FE114F10469
:1054300009F41DC1C114D10409F41BC16B3009F07A
:1054400020C16114710409F416C18114910409F496
:1054500014C1FE013296CE014296C192D1922BE048
:10546000C20ED11C8E179F07C1F78DE0D701D596CC
:105470008C93D59782E090E0D3968D939C93D497AC
:105480008AE0D6968C935701B7E3AB0EB11C41E08E
:10549000BE016F5F7F4FC5010E947C172981F70114
:1054A00083A994A9820F911D9C012F5F3F4F23ABCD
:1054B00034ABE80FF91F2CE225ABF1E0F51590F5C0
:1054C000512C0F2EFCE24F2EF02D61C0E52DF0E0A7
:1054D000EE0FFF1F81E090E08C0F9D1FE80FF91F7A
:1054E000C180D280D701D3968D919C91D497C596D7
:1054F000F601418550E0B6018E0D9F1D0F94954633
:10550000D60119962C91F70183A994A9820F911DB8
:105510009C012F5F3F4F23AB34ABE80FF91F45AA27
:10552000539405C0512C0F2EFCE24F2EF02D0F94FA
:10553000E70C581658F2AAC0E52DF0E0EE0FFF1F59
:1055400081E090E08C0F9D1FE80FF91FC180D28091
:10555000D701D3968D919C91D497C596F60141853C
:1055600050E0B6018E0D9F1D0F949546D6011996F9
:105570002C91F70183A994A9820F911D9C012F5FA3
:105580003F4F23AB34ABE80FF91F45AA53940F9458
:10559000E70C8695581680F279C0D6011A968C9140
:1055A0001F928F933F922F92F70183A994A9C596DA
:1055B0008E0D9F1D9F938F930F94C346F30101900F
:1055C0000020E9F73197E619F709D701D396ED9353
:1055D000FC93D497CF01C596F601418550E0B60102
:1055E0008E0D9F1D0F949546D60119962C91F701AB
:1055F00083A994A9820F911D9C012F5F3F4F23AB7C
:1056000034ABE80FF91F15ABFCE0CF0ED11C0F90A7
:105610000F900F900F900F900F904C145D0409F0B5
:10562000BCCF0130D9F4D701D3968D919C91D497FA
:10563000C596840101501F4FF801408150E0B4012C
:105640008E0D9F1D0F949546D8012C91F70183A9CB
:1056500094A9820F911D83AB94AB2BC0D701D39635
:10566000ED91FC91D497EE0DFF1D15AA22C080E0AC
:105670003FC080E03DC080E03BC080E039C080E0BA
:1056800037C08114910409F0E4CEF9CF1B3049F6FC
:1056900063012301B8E14B0E511C0F2EF8E92F2EA8
:1056A000F1E23F2EF02D3701E5E36E0E711C1CE296
:1056B00074CFA7014E5A5D4FF701E85AFD4F808124
:1056C000DA018C9397012D5A3D4F31968081F90173
:1056D0008083D701D3966D917C91D49762507109E4
:1056E000C50109DE0296F70183AB94AB81E081AB83
:1056F0006196CDBFDEBFDF91CF911F910F91FF90DB
:10570000EF90DF90CF90BF90AF909F908F907F9061
:105710006F905F904F903F902F9008952F923F92FF
:105720004F925F926F927F928F929F92AF92BF92B1
:10573000CF92DF92EF92FF920F93CF93DF93CDB78B
:10574000DEB76097CDBFDEBF009709F46EC061156C
:10575000710509F46AC09B01FE013196DE01519684
:1057600021933193255F3F4FEA17FB07C9F76A0181
:105770007B011C01B12C12C0EB2DF0E0EE0FFF1FDE
:1057800081E090E08C0F9D1FE80FF91F80819181CF
:105790000E94DA16882309F448C0B3940F94E70CEA
:1057A000B81650F30F94420A4B015C010F942B0A78
:1057B0002B013C0186E693E40E9419C5082F811154
:1057C0000BC09EE1890E911CA11CB11C8414950490
:1057D000A604B70450F115C040E050E06CEE70E450
:1057E00080E30E948D1C26E633E4A601B701C101C7
:1057F000FADD48E654E46CEE70E482E30E948D1C0E
:105800000EC000E026E633E4A601B701C101EBDDDE
:1058100040E050E06CEE70E482E30E948D1C86E66E
:1058200093E40E9413C50E94C1166096CDBFDEBFEF
:10583000DF91CF910F91FF90EF90DF90CF90BF90CD
:10584000AF909F908F907F906F905F904F903F9020
:105850002F900895009789F06115710571F0411539
:10586000510559F02115310541F0FC011082FB0171
:105870001082FA011082F901108208952F923F924E
:105880004F925F926F927F928F929F92AF92BF9250
:10589000CF92DF92EF92FF920F931F93CF93DF93FC
:1058A000CDB7DEB72597CDBFDEBF009709F461C045
:1058B0004115510509F45FC02115310509F45DC09A
:1058C000613BE4E07E0708F45AC02B01E0EB4E1A7E
:1058D000E4E05E0A612C712CE2E04E165104610492
:1058E00071040CF454C02C833D831A018C01C12C2B
:1058F000D12C7601C3944B01A12CB12CB501A4018C
:105900004C195D096E097F09C8010F94BA3C9E01CC
:105910002F5F3F4F41E050E0BE016D5F7F4FC801F8
:105920000F946E3981112DC08B818B3191F18FEFE6
:10593000C81AD80AE80AF80AC414D504E604F70419
:10594000ECF225C089819A810497E8F0B10187E4DF
:1059500092E40F947F19982F882341F16C817D8107
:1059600089E492E40F947F1991E081111FC090E0C7
:105970001DC090E01BC090E019C090E017C090E0FF
:1059800015C090E013C090E011C090E00FC090E00F
:105990000DC09E012F5F3F4F44E050E067E472E48A
:1059A000C8010F946E39882369F2EFCF892F2596AD
:1059B000CDBFDEBFDF91CF911F910F91FF90EF9090
:1059C000DF90CF90BF90AF909F908F907F906F901F
:1059D0005F904F903F902F9008950097A9F0611528
:1059E0007105B1F0FC019C01260F371F60E070E0EB
:1059F000CB0141914D3021F46F5F7F4F8F4F9F4F0F
:105A00002E173F07B1F7089560E070E0CB010895CD
:105A100060E070E0CB0108952F923F924F925F9229
:105A20006F927F928F929F92AF92BF92CF92DF92AE
:105A3000EF92FF920F931F93CF93DF9300D01F92AB
:105A4000CDB7DEB7009709F455C00115110509F46B
:105A500053C0613B7440C0F4F8011082118212827D
:105A6000138280E04CC009811A81B801C101B5DF01
:105A7000460E571E681E791E0815190500F1C00E46
:105A8000D11EE11CF11C0BC00B831C8349011A01C0
:105A90005C01C12CD12C7601412C512C3201B70173
:105AA000A601C5010F94BA3C9E012F5F3F4FA40190
:105AB000B101C5010F946E398823A9F21FC0F6E227
:105AC0004F1651046104710440F4EB81FC81108293
:105AD00011821282138281E012C0F5E24F1A51083E
:105AE00061087108EB81FC8140825182628273827D
:105AF00081E005C080E003C080E001C080E0249622
:105B0000CDBFDEBFDF91CF911F910F91FF90EF903E
:105B1000DF90CF90BF90AF909F908F907F906F90CD
:105B20005F904F903F902F900895009741F0FC01B7
:105B3000EC5AFD4F6081718182819381089560E00C
:105B400070E0CB010895009739F0FC01EC5AFD4F4D
:105B500010821182128213820895CF93DF930097EF
:105B600081F12091053D21112CC0EC010F942E07ED
:105B7000882339F1CE010E9489930F9413070E9464
:105B80004DF41F928F938CE991E29F938F93C7E41A
:105B9000D2E4DF93CF930F94C34609900020E9F736
:105BA0002197AE014754524420E067E472E487E64F
:105BB00097E30F94D9110F900F900F900F900F90C3
:105BC0000F90DF91CF9108952115310551F0505874
:105BD00061097109F901408351836283738381E014
:105BE000089580E00895009719F0FC01848D0895D0
:105BF00080E008952F923F924F925F926F927F9232
:105C00008F929F92AF92BF92CF92DF92EF92FF92CC
:105C10000F931F93CF93DF93CDB7DEB72597CDBFFB
:105C2000DEBFE114F10409F49EC0170148015901D7
:105C30006A017B01182FC1010E94B51624013501AC
:105C40004C185D086E087F08143031F484E10E941E
:105C500052B89B01AC0105C085E10E9452B89B017E
:105C6000AC01440C551C661C771CD301C201880F83
:105C7000991FAA1FBB1F880F991FAA1FBB1F480E81
:105C8000591E6A1E7B1E211531054105510549F03B
:105C9000C301B2010F947A442A833B834C835D8312
:105CA00008C08FEF8A8390EE9B83A5EFAC83B5E0AD
:105CB000BD836A817B818C819D812AE030E040E058
:105CC00050E00F947A445F934F933F932F93FF924A
:105CD000EF92DF92CF92BF92AF929F928F92C301C9
:105CE000B2012AE030E040E050E00F947A445F9344
:105CF0004F933F932F9387EB91E29F938F9307E40A
:105D000012E41F930F930F94C346F80101900020F3
:105D1000E9F73197AF014754524420E0B80187E6D4
:105D200097E30F94D9110A811B812C813D814BE0AF
:105D3000BE016F5F7F4FC1010F94F918F10101900F
:105D40000020E9F73197E219F309D1011996EC9394
:105D5000199781E01B968C93CDBFDEBF6A817B8152
:105D60008C819D8104C060E070E080E090E0259629
:105D7000CDBFDEBFDF91CF911F910F91FF90EF90CC
:105D8000DF90CF90BF90AF909F908F907F906F905B
:105D90005F904F903F902F9008952F923F924F9297
:105DA0005F926F927F928F929F92AF92BF92CF92AB
:105DB000DF92EF92FF920F931F93CF93DF93CDB7B4
:105DC000DEB72897CDBFDEBFCA01E982FA82CD8255
:105DD000DE82AB82BC826115710509F4B7C0009701
:105DE00009F4B6C0EF2809F4B5C0802E912EA22E7A
:105DF000B32E25EB82169104A104B10438F00F2EC6
:105E0000F4EB8F2E912CA12CB12CF02DDB01CD9039
:105E1000DD90ED90FC90B0E8DB1AE108F108FB01A1
:105E2000C082D182E282F38221E02093BF30F2E08F
:105E30008F169104A104B10408F46AC0FB012FEB92
:105E400030E32F83388794012150304C220F331FC9
:105E5000220F331F1B01220E331E4601570100E0A3
:105E600010E098014481558166817781505861091D
:105E70007109448355836683778341905190619083
:105E80007190441955096609770914161506160606
:105E9000170634F441E0AF81B88511964C9304C0E5
:105EA000AF81B88511961C92AF81B88511965C912F
:105EB0001197BD016F5F7F4F6F8378874C915417A7
:105EC00081F0D801AA0FBB1FAA0FBB1FA80FB91FD3
:105ED0004D925D926D927C9213970F5F1F4F2F4FE3
:105EE0003F4F4081518162817381C416D506E60619
:105EF000F70614F46A017B01481559056A057B050C
:105F000014F44A015B01E215F30509F0ABCF05C0BB
:105F10004601570100E010E09801A981BA810D9374
:105F20001D932D933C931397ED81FE81309721F0C3
:105F300080829182A282B382EB81FC81309761F0F2
:105F4000C082D182E282F38281E007C080E005C096
:105F500080E003C080E001C081E02896CDBFDEBFB5
:105F6000DF91CF911F910F91FF90EF90DF90CF9035
:105F7000BF90AF909F908F907F906F905F904F9069
:105F80003F902F9008958F929F92AF92BF92CF92A1
:105F9000DF92EF92FF920F931F93FC01892BA1F1E7
:105FA0006115710599F1008111812281338184810C
:105FB0009581A681B781081719072A073B0744F581
:105FC000C084D184E284F384C816D906EA06FB06AD
:105FD0000CF584849584A684B784C814D904EA0493
:105FE000FB04D4F488159905AA05BB05BCF40C156F
:105FF0001D052E053F0524F481E0FB0180830FC0C1
:10600000FB01108281E00BC080E009C080E007C086
:1060100080E005C080E003C080E001C080E01F9107
:106020000F91FF90EF90DF90CF90BF90AF909F9037
:106030008F9008953F924F925F926F927F928F92CE
:106040009F92AF92BF92CF92DF92EF92FF920F9307
:106050001F93CF93DF93009709F448C021153105B2
:1060600009F446C0443051056105710508F442C089
:106070006A017B01E4E0CE1AD108E108F108E1F100
:1060800059018C01912C312C812C412C512C320145
:10609000E501C90DD11DBE01C201880F991F880FEE
:1060A000991F800F911F6FDF882379F088818823E3
:1060B00011F0839401C0339483E0480E511C611C9D
:1060C000711C9394E2E0E91550F08FEF481A580ADA
:1060D000680A780A4C145D046E047F04C8F28820B4
:1060E00069F081E0332059F080E009C080E007C00A
:1060F00080E005C080E003C081E001C081E0DF9165
:10610000CF911F910F91FF90EF90DF90CF90BF90B4
:10611000AF909F908F907F906F905F904F903F9047
:1061200008952F923F924F925F926F927F928F923B
:106130009F92AF92BF92CF92DF92EF92FF920F9316
:106140001F93CF93DF93CDB7DEB76A97CDBFDEBF86
:10615000582ED92E862E972E19821A821B821C82C7
:106160001D821E821F82188619861A861B861C862F
:106170001D861E861F86188A82E00E9476B86B30C4
:1061800009F0CAC00F94200E882309F4C6C00F94EA
:106190000F0E252C3D2CCE0101968B8B9C8BDE01A6
:1061A0001996AD8BBE8BA98BBA8B652C7D2C689410
:1061B000552452F8298E3A8E482C392C4C016F8A7E
:1061C000788EA988BA8864010F2EF8EEEF2EFDE2D2
:1061D000FF2EF02D04EB10E020E030E04FEE5DE20A
:1061E000B301852DDADD882331F14091E82D5091FE
:1061F000E92D6091EA2D7091EB2D2CEE3DE28FEEB2
:106200009DE218DF882361F08091EC2D90E0A0E002
:10621000B0E0EF89F88D80839183A283B38314C0AB
:106220008EEF90E0A0E0B0E0EF89F88D808391835D
:10623000A283B38309C08FEF90E0A0E0B0E0F30148
:1062400080839183A283B3835394F0E36F1AFDEFAD
:106250007F0A84E0880E911CA989BA891496A98BBB
:10626000BA8BB6E05B12ABCF932C298C3A8C642CA2
:10627000792C6894552452F80F2EF5E44F2EF02D0A
:106280000F2EF2E5DF2EF02D0F2EFCE4CF2EF02D99
:10629000AB88BC888D889E88698A7A8AF4010191CE
:1062A0001191219131914F01D5014D915D916D91E8
:1062B0007D915D017301852D9DDC65317105810541
:1062C00091051CF4F30142861AC0F101808191818D
:1062D000A281B3810097A105B10529F4A989BA89E2
:1062E0001A96CC920CC00197A105B10521F4E98959
:1062F000FA89D28604C0A989BA891A964C92539415
:10630000BCE06B0E711CE0E32E1AEDEF3E0AF6E0E6
:106310005F12C2CF81E001C080E06A96CDBFDEBFD0
:10632000DF91CF911F910F91FF90EF90DF90CF9071
:10633000BF90AF909F908F907F906F905F904F90A5
:106340003F902F9008951F93CF93DF93009709F408
:10635000DAC0EC018881843069F128F4813049F099
:106360008230C9F0D0C0883011F1893009F4A7C05B
:10637000CAC08B81813009F0C6C08C81813009F0A0
:10638000C2C00F94080ACE010E94122962E0CE0119
:106390000E948113B8C08091C146813029F463E026
:1063A000CE010E948113AFC00E945F1BACC00E944F
:1063B000D54BA9C0CE010E944D2182E00E9476B843
:1063C0006B3041F068E077E38CE89AE30E94A7170E
:1063D000182F10C00F94200E8823E1F068E077E3B7
:1063E0008CE89AE30E94A717182F6CE97AE38AEFEA
:1063F0009BE497DE113071F482E00E9476B8162F8C
:106400008CE89AE30E944F0F612F86E19EE30E9481
:10641000711107C088E097E30E94E516882309F40C
:1064200065C04CE95AE368E077E3CE0177D95EC0F6
:106430000E9471F8882309F463C00F94860B66E507
:106440007EE3CE010E948D240E9460F859C08981AC
:10645000811159C0CE010E941521882341F00F946B
:10646000860B66E57EE3CE010E948D244CC019AAFE
:1064700081E08AAB48C089A9882309F444C0898196
:10648000811141C0CE010E94E320882341F00F9486
:10649000860B66E57EE3CE010E948D2434C019AAE6
:1064A00032C00E9471F8882371F10F94860B66E563
:1064B0007EE3CE010E948D240E9460F824C0CE01AC
:1064C0000E944D2168E077E38CE89AE30E9497FCF4
:1064D000813031F088E097E30E94ECFC882399F04A
:1064E00068E077E3CE010F9415000DC0FE01EA5C71
:1064F000FD4F8081813009F49BCF823091F6BBCF74
:1065000089A98111A4CFDF91CF911F910895CF93D5
:106510000E9437C0C82F88E10E9476B8C61741F0A4
:1065200061E080E00E944DF661E081E00E944DF65E
:10653000CF910895CF930E9437C0C82F88E10E9461
:1065400076B8C61749F061E080E00E944DF661E040
:1065500081E00E944DF608C060E080E00E944DF6A8
:1065600060E081E00E944DF6CF910895EF92FF9296
:106570000F931F93CF93DF93CDB7DEB72797CDBF90
:10658000DEBF7C01FB0184818D8385818E838681C2
:106590008F8380819181A281B38189839A83AB8328
:1065A000BC83870180EAE81688E0F80629F460E1F8
:1065B00083E00F94E02314C080EBE81688E0F8062F
:1065C00029F460E283E00F94E02313C080EAE81628
:1065D00089E0F80629F460E184E00F94E02312C01A
:1065E000003B89E0180729F460E284E00F94E0237F
:1065F00012C0003A8AE0180729F460E185E00F94A0
:10660000E02310C0003B8AE0180729F460E285E02F
:106610000F94E02307C0003A1B4021F460E186E0BC
:106620000F94E023BE016F5F7F4FC7010E94086C8B
:106630002796CDBFDEBFDF91CF911F910F91FF90C5
:10664000EF900895DC01892BE1F0E62FE695E695C1
:10665000E69580E2E89FF0011124FA5F808567707B
:1066600021E030E002C0220F331F6A95E2F72823B1
:1066700081E009F480E08C9311968C931197129627
:106680001C920895CF93DF93009709F4A5C06D3253
:1066900009F0A4C03091A80621E0432F407235FFD5
:1066A00020E0FC0120833181231709F499C0EC011B
:1066B000442309F46BC0311169C00F94C2060097DE
:1066C000F9F40E947829811119C086E0EFEDF1E21A
:1066D000A7E4B2E401900D928A95E1F7E7E4F2E4D1
:1066E00001900020E9F73197AF014754524421E06F
:1066F00067E472E487E697E30F94D9111A8268C0C1
:10670000803D974008F50E947829811119C086E0E4
:10671000E5EEF1E2A7E4B2E401900D928A95E1F78B
:10672000E7E4F2E401900020E9F73197AF01475424
:10673000524421E067E472E487E697E30F94D911AD
:106740000F94D6061A8244C081E08A830F94D6063D
:106750000E94782981113CC086E0EBEEF1E2A7E4CB
:10676000B2E401900D928A95E1F7E7E4F2E401903A
:106770000020E9F73197AF014754524421E067E424
:1067800072E487E697E30F94D91122C01A8281E060
:1067900090E00F94E9060E947829811119C086E0E3
:1067A000E1EFF1E2A7E4B2E401900D928A95E1F7FE
:1067B000E7E4F2E401900020E9F73197AF01475494
:1067C000524421E067E472E487E697E30F94D9111D
:1067D000888189838A8105C080E003C080E001C090
:1067E00080E0DF91CF91089585E396E40C94E6CCA8
:1067F00008950E947829811117C069EC72E487E638
:1068000097E30F94851180914B43813029F549EC32
:1068100052E46BEC72E487E697E30E94FCB589ECE6
:1068200092E40D947611089569EC72E487E697E39B
:106830000E94219A80914B43813071F424EB3AE31A
:1068400049EC52E46BEC72E487E697E30E94129AFB
:1068500089EC92E40D94761108950E948E8E88231F
:1068600029F087EC9FE30C944A2408950E9478292C
:1068700081112EC065EE7FE38EE698E30E94219A97
:1068800080916740813021F50E947829811112C0E2
:1068900062E480916737909168370E94ED6A409179
:1068A000E53F5091E63F21E067EE7FE387E697E31F
:1068B0000F94D91124EB3AE345EE5FE367EE7FE3F3
:1068C0008EE698E30E94129A85EE9FE30D9476116E
:1068D0000895CF92DF92EF92FF920F931F93CF9381
:1068E000DF930E947829882319F007E617E302C096
:1068F0000EE618E386ED9FE30E942C9C882331F07E
:1069000066ED7FE3C8010E94302488C28091E43F95
:106910008150823008F054C10E94AE9C882309F453
:106920007DC261E97EE38FE09DE30E94B39B80918D
:10693000C23F813009F072C2E090913EF090923EE9
:1069400082E0E816F10408F469C28091E43F8130E6
:1069500039F48091963E8F7D8C3409F0CBC00AC00B
:106960008091963E843209F0C5C08091973E833570
:1069700009F0C0C00E947829811156C087E0E7EF76
:10698000F1E2A7E4B2E401900D928A95E1F7E7E421
:10699000F2E401900020E9F73197AF0147545244E7
:1069A00020E067E472E487E697E30F94D911109230
:1069B000933E1092943EE114F104A1F080E090E047
:1069C000C1E9DEE3FC01EF56F14C658187E697E310
:1069D0000F9465128A819B8101968A839B838E1511
:1069E0009F0580F30F94980B1F928F938EEF91E287
:1069F0009F938F93C7E4D2E4DF93CF930F94C34662
:106A000009900020E9F72197AE014754524421E054
:106A100067E472E487E697E30F94D9110F900F9023
:106A20000F900F900F900F900F94980B882371F197
:106A300081E00E94FC89813069F481E99EE30E9433
:106A4000F99B81E99EE30E940B9C0F94750B0E94B9
:106A5000FD9C02C00E945E9DE8E2F1E4808190E02E
:106A6000DC01A85DBE4B25853685880F991FFC018A
:106A7000E85DFE4B418152811F960C9161E084EBF1
:106A80009AE30E9470240F949F0C93C0E092C53F3C
:106A9000F092C63F0F94980B682FC8010E94DA8CC1
:106AA0000E947829811185C00F94980B1F928F93B3
:106AB0008091E43F1F928F9384E092E29F938F93A3
:106AC000C7E4D2E4DF93CF930F94C346099000202C
:106AD000E9F72197AE014754524421E067E472E49C
:106AE00087E697E30F94D911EDB7FEB73896EDBF5F
:106AF000FEBF5FC00E947829811157C08091E43F9A
:106B0000823049F48091963E843229F48091973EF8
:106B1000873409F44AC08AE0E2E2F2E2A7E4B2E490
:106B200001900D928A95E1F7E7E4F2E401900020EC
:106B3000E9F73197AF014754524420E067E472E42B
:106B400087E697E30F94D911E1E9FEE312821382FD
:106B500080819181892BA9F080E090E0EF01FC0118
:106B6000EF56F14C658187E697E30F9465128A81B1
:106B70009B8101968A839B832881398182179307A1
:106B800070F3E7E4F2E480E290E080839183019087
:106B90000020E9F73197AF014754524421E067E400
:106BA00072E487E697E30F94D91181E99EE30E948E
:106BB0000B9C81E99EE30E94F99B0F94750B2EC1FB
:106BC0000F9438076B017C0161E97EE38FE09DE360
:106BD0000E94489B8091C23F813039F0F5E6CF1684
:106BE000D104E104F10408F419C10F944F07809116
:106BF000C23F813079F481E99EE30E947C9C882326
:106C000021F0E090C43FF12C40C0E090913EF09024
:106C1000923E3BC00F2EF1E9EF2EFEE3FF2EF02D4A
:106C2000F70181818F9380818F938CE292E29F9311
:106C30008F93C7E4D2E4DF93CF930F94C3460990B8
:106C40000020E9F72197AE014754524421E067E460
:106C500072E487E697E30F94D9111092C43F0F9026
:106C60000F900F900F900F900F90F70180819181FE
:106C70008739910530F086E990E08093913E9093BA
:106C8000923EE090913EF090923E0E9478298111D0
:106C90005DC0FF92EF928BE492E29F938F93C7E4E3
:106CA000D2E4DF93CF930F94C34609900020E9F715
:106CB0002197AE014754524420E067E472E487E62E
:106CC00097E30F94D9111092933E1092943E0F9037
:106CD0000F900F900F900F900F90E114F104A1F01E
:106CE00080E090E0C1E9DEE3FC01EF56F14C658104
:106CF00087E697E30F9465128A819B8101968A83C8
:106D00009B838E159F0580F30F94980B1F928F9392
:106D10008EEF91E29F938F93C7E4D2E4DF93CF93FA
:106D20000F94C34609900020E9F72197AE0147541C
:106D3000524421E067E472E487E697E30F94D911A7
:106D40000F900F900F900F900F900F900F94980B43
:106D5000882371F181E00E94FC89813069F481E926
:106D60009EE30E94F99B81E99EE30E940B9C0F9495
:106D7000750B0E94FD9C02C00E945E9DE8E2F1E45A
:106D8000808190E0DC01A85DBE4B25853685880FAB
:106D9000991FFC01E85DFE4B418152811F960C91C9
:106DA00061E084EB9AE30E9470240F949F0C30C042
:106DB000E092C53FF092C63F0F94980B682FC80130
:106DC0000E94DA8C0E947829811122C00F94980BBE
:106DD0001F928F9388E592E29F938F93C7E4D2E44A
:106DE000DF93CF930F94C34609900020E9F72197D2
:106DF000AE014754524421E067E472E487E697E32A
:106E00000F94D9110F900F900F900F900F900F903B
:106E100081E99EE30E94F99B0F94750BDF91CF915E
:106E20001F910F91FF90EF90DF90CF9008958F9278
:106E30009F92AF92BF92CF92DF92EF920F931F93E8
:106E4000CF93DF93EC0180E00E9452B84B015C01CC
:106E5000209709F45CC11E8EFE01E15BFD4F10829C
:106E6000CE010E94311F882309F451C16E0185E3D0
:106E7000C80ED11CBE01625E7F4FC6010E9490ED1C
:106E80008D8F81111FC00E947829811119C08BE15B
:106E9000ECE6F2E2A7E4B2E401900D928A95E1F704
:106EA000E7E4F2E401900020E9F73197AF0147549D
:106EB000524421E067E472E487E697E30F94D91126
:106EC00081E08E8F63EF74E4C6010E9459F2FE01E7
:106ED000E25BFD4F808383EF94E40E9404BF88232C
:106EE000A1F181E0FE01E15BFD4F808383EF94E43B
:106EF0000E94A1BE0E947829811127C0FE01E15B9A
:106F0000FD4F80811F928F93319780811F928F93C5
:106F100087E892E29F938F9307E412E41F930F9305
:106F20000F94C346F80101900020E9F73197AF01B3
:106F30004754524421E0B80187E697E30F94D911F2
:106F4000ADB7BEB71896ADBFBEBF8E8D813039F0DC
:106F5000FE01E15BFD4F8081813009F05CC00E9441
:106F60007829811119C08CE1EAE9F2E2A7E4B2E4E0
:106F700001900D928A95E1F7E7E4F2E40190002098
:106F8000E9F73197AF014754524421E067E472E4D6
:106F900087E697E30F94D9116894EE24E2F806EBA4
:106FA00012E2A5019401BE01685E7F4FCE010696F4
:106FB0000E945C548D8340E050E0BA01CE010E94F3
:106FC000A32D8D81882309F4A2C082E00E9476B8A7
:106FD000062F8BE00E9476B821E0611120E0BE010F
:106FE0006D5C7F4F46E55EE3C6010E94604DCE01B9
:106FF0000E948A1B9E01275A3D4FAE01485A5D4FA1
:10700000BE016D5A7D4FCE018E5A9D4F0E942A2C93
:107010000E9465F97CC08E010A5F1F4FB80186E5AA
:107020009EE30E9434538D83811139C0A5019401E0
:10703000BE01685E7F4FC8010E9496508D8340E07C
:1070400050E0BA01CE010E94A32D8D81882309F45E
:107050005EC082E00E9476B8062F8BE00E9476B870
:1070600021E0611120E0BE016D5C7F4F46E55EE3EB
:10707000C6010E94604DCE010E948A1B9E01275AC4
:107080003D4FAE01485A5D4FBE016D5A7D4FCE0156
:107090008E5A9D4F0E942A2C0E9465F938C08E019D
:1070A0000C5A1D4F0F2EF6E5AF2EFEE3BF2EF02D2E
:1070B000F5016285738520E032E0A601C5010E94DA
:1070C0000C2D015011096E01FEEACF1AFDEFDF0A07
:1070D000D5011A966D917C911B979801A601C50167
:1070E0000E943E2CFE01E85AFD4FD6018C91808310
:1070F000C75ADD4FF80180818883D5011A964D91DA
:107100005D916D917C911D97C5010F94BA3CDF9103
:10711000CF911F910F91EF90DF90CF90BF90AF90E4
:107120009F908F9008956DE285E097E3ABDA882316
:1071300009F467C080917331882309F446C00E9426
:107140007F5E84E0809326060F94FF0583EF94E42E
:107150000E9497CB84EB9AE36ADE8091033D8823FB
:10716000F1F00E945BC9813019F0823069F017C0DC
:107170008091023D882329F083EF94E40E94F9C8AE
:107180000EC00E94CCC80BC08091023D882329F01C
:1071900083EF94E40E947BCA02C00E9446CA109208
:1071A00073310F949F0C84EB9AE30E941D2281118E
:1071B0000F94080A84EB9AE30E9412296091F63C2E
:1071C00084EB9AE30E9481131CC00F949F0C0F94D0
:1071D000E60966E084EB9AE30E94811361E08AEBA2
:1071E0009AE30E9402530E9481500F94A21A0E94B7
:1071F000555E81E08093733184E0809325060F947F
:10720000FF0580917331882331F00E94D35C811196
:10721000FCCF8091733108954F925F926F927F926D
:107220008F929F92AF92BF92CF92DF92EF92FF9296
:107230001F93CF93DF93CDB7DEB72797CDBFDEBFC8
:107240007C011092C24610E00F2E812CFBE49F2E91
:10725000A12CB12CF02D0F2EF7E4CF2EF2E4DF2E6F
:10726000F02D0F2EF0E84F2EF5E25F2E612C712CE1
:10727000F02D111120C080E096E9A0E0B0E0F70108
:1072800080839183A283B3838AE0EBEBF2E2D601A1
:1072900001900D928A95E1F7F60101900020E9F73F
:1072A0003197AF014754524421E0B60187E697E396
:1072B0000F94D9115CC0113001F580EC92E1A0E08F
:1072C000B0E0F70180839183A283B38389E0E5EC8A
:1072D000F2E2D60101900D928A95E1F7F601019054
:1072E0000020E9F73197AF014754524421E0B6013D
:1072F00087E697E30F94D9113AC01230E9F4D70129
:107300004D925D926D927C92139789E0EEECF2E2E1
:10731000D60101900D928A95E1F7F60101900020C7
:10732000E9F73197AF014754524421E0B60187E6AF
:1073300097E30F94D9111BC0F70180829182A2823A
:10734000B38289E0E7EDF2E2D60101900D928A95D1
:10735000E1F7F60101900020E9F73197AF014754BA
:10736000524421E0B60187E697E30F94D911D70183
:1073700014968C9114978D8315968C9115978E8306
:1073800016968C9116978F838D919D910D90BC913F
:10739000A02D89839A83AB83BC8360E185E00F9441
:1073A000E023BE016F5F7F4F80EA9AE00E94086C85
:1073B0000F94120C08C085E396E40E94E6CC81305D
:1073C00041F00E941B1B0F94250C803A9F4098F3BC
:1073D0007AC011111DC08CE0E0EEF2E2A7E4B2E445
:1073E00001900D928A95E1F7E7E4F2E40190002024
:1073F000E9F73197AF014754524421E067E472E462
:1074000087E697E30F94D91182E08093C24678C053
:107410001130E9F48BE0ECEEF2E2A7E4B2E4019083
:107420000D928A95E1F7E7E4F2E401900020E9F794
:107430003197AF014754524421E067E472E487E694
:1074400097E30F94D91181E08093C24659C012305E
:10745000E9F48BE0E7EFF2E2A7E4B2E401900D92E9
:107460008A95E1F7E7E4F2E401900020E9F731972B
:10747000AF014754524421E067E472E487E697E3A2
:107480000F94D91183E08093C2463AC08BE0E2E0CA
:10749000F3E2A7E4B2E401900D928A95E1F7E7E404
:1074A000F2E401900020E9F73197AF0147545244CC
:1074B00021E067E472E487E697E30F94D91184E052
:1074C0008093C2461DC01F5F143009F0D2CE89E000
:1074D000EDE0F3E2A7E4B2E401900D928A95E1F7C2
:1074E000E7E4F2E401900020E9F73197AF01475457
:1074F000524421E067E472E487E697E30F94D911E0
:107500002796CDBFDEBFDF91CF911F91FF90EF9007
:10751000DF90CF90BF90AF909F908F907F906F90B3
:107520005F904F900895CF92DF92EF92FF920F936A
:107530001F93CF930E9419C0882309F49CC084EB49
:107540009AE30E949413883009F495C084EB9AE37F
:107550000E949413863009F48EC00F94D60C8823B1
:1075600019F10F94E00C81111FC00F94E30C0E94DD
:107570007829811119C088E1E6E1F3E2A7E4B2E4D9
:1075800001900D928A95E1F7E7E4F2E40190002082
:10759000E9F73197AF014754524421E067E472E4C0
:1075A00087E697E30F94D9110F94CC0C882309F444
:1075B00062C00F94E6090E9481500E9478298111CF
:1075C00019C08EE0EEE2F3E2A7E4B2E401900D927E
:1075D0008A95E1F7E7E4F2E401900020E9F73197BA
:1075E000AF014754524421E067E472E487E697E331
:1075F0000F94D9110F94DD0501E010E0C0E00F2ECB
:10760000F2E1CF2EF1E2DF2EF02D0F2EF7E4EF2E78
:10761000F2E4FF2EF02D0F94CC05882341F10F9456
:10762000DD05CF5F0E94782981111CC01F930F9345
:10763000DF92CF92FF92EF920F94C346F701019031
:107640000020E9F73197AF014754524421E0B701D8
:1076500087E697E30F94D9110F900F900F900F903A
:107660000F900F900F5F1F4FC33019F0D4CFC3306E
:1076700090F20E948DF3CF911F910F91FF90EF90A8
:10768000DF90CF900895F8940E9487610F948B2328
:107690000F94A21A0E94DB9A0E9429F60E94A0D39E
:1076A00041E060EA78E08EE698E30F943B1265E1F2
:1076B00070E280EA98E00E94B632E0EAF8E0838166
:1076C0008F7C8061838385EE9FE30F94761161E068
:1076D00087EC9FE30E941C9C41E060EA7BE08FE026
:1076E0009DE30F943B126EE070E280EA9BE00E9403
:1076F000B632E0EAFBE083818F7C8061838381E99D
:107700009EE30E94F99B81E99EE30E940B9C61E04D
:1077100086ED9FE30E941C9C1092E43F1092EB4088
:1077200088E690E40F94761141E060EA7AE085E81B
:1077300099E30F943B1267E070E280EA9AE00E94BE
:10774000B632E0EAFAE083818F7C8061838341E096
:1077500060EA79E087E697E30F943B1260E070E21D
:1077600080EA99E00E94B632E0EAF9E083818F7CFA
:107770008061838389EC92E40F9476110F946B05FA
:107780000F9481070F9412090F94AE0B0F94A50765
:107790000F947E0D0E943CF40E94F0F70E94AC0E04
:1077A000C0E060E08C2F0E944DF6CF5FC830C9F773
:1077B00087E08093A2007894E0E2F6E082E086839E
:1077C00084E086830E940EB8811110C00E9414B913
:1077D0000E943EB90E9465BE0E94F5BE0E94EABFAB
:1077E0000E9431C081E08093013D27C00E94D8BD36
:1077F000882309F181E08093013D0E94782981115D
:107800001CC08DE1ECE3F3E2A7E4B2E401900D9239
:107810008A95E1F7E7E4F2E401900020E9F7319777
:10782000AF014754524421E067E472E487E697E3EE
:107830000F94D91102C01092013D0E945DBD0E94BB
:1078400065F90E94B8BD81E00F94C4086DE285E03F
:1078500097E30E9422330E94109D66E673E485E35D
:1078600096E40E945AC585E396E40E943CC084EBEE
:107870009AE30E949B1380E00E9469F783EF94E4EF
:107880000E9497CB84EB9AE3D2DA81E00E94ABB1FD
:1078900080E00E94A5B180E00E94AEB180E00E942D
:1078A000B1B10E94C1160E9487320E94DF9A85E31F
:1078B00096E40E943CC087E090E2AEDC0E945BC987
:1078C000813029F48091023D0E9429CF25C00E9479
:1078D0005BC9823091F481E00E945EC98091023DD3
:1078E000882329F083EF94E40E947BCA02C00E949F
:1078F00046CA81E00E9410CA0FC00E945BC9833053
:1079000029F487E492E40E9440CB06C00E945BC940
:10791000843011F40E9467CF84E0809326060E9491
:10792000ACD384EB9AE30E94122987E697E30E9486
:1079300011A50E94E80E09E513E2C7E4D2E40E9413
:10794000F43366E673E485E396E40E94EC1584EB79
:107950009AE30E947D1584EB9AE30E94151584EB4F
:107960009AE30E94AD2D84EB9AE30E94A3310E941A
:10797000F933D9DB0E942D340E94693484EB9AE3F9
:107980000E94251B0E94D9D30E94A8B1833031F5F3
:107990000E944A1F882311F10E94782981111EC07C
:1079A0000F94C3091F928F931F930F93DF93CF936D
:1079B0000F94C346FE0101900020E9F73197AF0113
:1079C0004754524421E0BE0187E697E30F94D91152
:1079D0000F900F900F900F900F900F900E94B12377
:1079E00068E271E484EB9AE30E94FB2468E271E4AC
:1079F00084EB9AE30E944F250E9474F894DD0FB641
:107A000007FC9DCF80E00E9404770E941877FFCF8B
:107A1000EF92FF920F931F93CF93DF93009749F15B
:107A20006115710541F14115510539F18A017B015B
:107A3000EC010F944A46F80180839183892B89F0E9
:107A4000D70120E030E0FE01E20FF31FE491ED9357
:107A50002F5F3F4FF801808191812817390798F3F4
:107A600002C020E030E0F701E20FF31F108281E056
:107A700005C080E003C080E001C080E0DF91CF91CD
:107A80001F910F91FF90EF9008950F931F93CF9345
:107A9000DF930097C9F061157105C1F041155105DB
:107AA000B9F0EA018B01FC0165917491C8010F9452
:107AB0004346F80101900020E9F73197E01BF10BF4
:107AC000E883F98381E005C080E003C080E001C065
:107AD00080E0DF91CF911F910F9108957F928F9257
:107AE0009F92AF92BF92CF92DF92EF92FF920F934D
:107AF0001F93CF93DF931F921F92CDB7DEB70097EE
:107B000009F49BC06115710509F497C0D42E7B015F
:107B10008C01AE014F5F5F4FBC018FE193E178DFD5
:107B2000882309F48AC089819A815C012FEFA21A07
:107B3000B20AF801E80FF91F20E22083B8016A0DAC
:107B40007B1DAE014F5F5F4F88E093E161DF8823CB
:107B500009F473C089819A81A80EB91EF801EA0D53
:107B6000FB1D8DE0808382E0A80EB11C8AE081833A
:107B7000B8016A0D7B1DAE014F5F5F4F81EF92E14F
:107B800047DF882309F459C0A981BA81AA0EBB1E18
:107B900048018A0C9B1C0F2EFDE07F2EF02DF40176
:107BA00070820F2EFAE0CF2EF02DC182C501029611
:107BB000800F911F0E9434B8F401748ED5015E9637
:107BC000C58EDD2059F1A00FB11F8AE0E1E6F3E296
:107BD00001900D928A95E1F7F7E2AF0EB11C0E9479
:107BE00038BEBC01C8018A0D9B1D0F94A5460E949A
:107BF00038BEFC0101900020E9F73197E81BF90B32
:107C0000E131F10518F4E983FA8304C080E190E0E2
:107C100089839A83A981BA81AA0DBB1DF801EA0F55
:107C2000FB1F8DE0808312968AE08183F801EA0FC2
:107C3000FB1F1082F701A083B1830F900F90DF919B
:107C4000CF911F910F91FF90EF90DF90CF90BF9059
:107C5000AF909F908F907F900895CF92DF92EF9298
:107C6000FF920F931F93CF93DF931F921F92CDB775
:107C7000DEB76115710591F14115510579F1009754
:107C800069F17A016B018C0119821A82AE014F5F92
:107C90005F4F88EC91E1BCDE882301F1C8010696B4
:107CA0009F938F938BE693E29F938F9389819A8121
:107CB0008C0D9D1D9F938F930F94C346F6010190E9
:107CC0000020E9F73197EC19FD09D701ED93FC93FA
:107CD0000F900F900F900F900F900F900F900F90AC
:107CE000DF91CF911F910F91FF90EF90DF90CF9098
:107CF0000895BF92CF92DF92EF92FF920F931F935E
:107D0000CF93DF931F921F92CDB7DEB7009709F490
:107D100082C06115710509F47EC06B018C01198266
:107D20001A82DB011D921C92AE014F5F5F4FBC01B6
:107D30008CEB91E16DDE882309F46DC0EAE9F1E591
:107D400087858F9386858F9385858F9384858F9381
:107D500085EF99E29F938F9389819A81800F911F7C
:107D60009F938F930F94C346F80101900020E9F789
:107D70003197E01BF10BE983FA83CDBFDEBFB12C55
:107D80000F2EF0E7EF2EF3E2FF2EF02D2DC0EB2D9E
:107D9000F0E0EE0FFF1FEE0FFF1FE656FE4ADF0179
:107DA0005A9613968C9113978F9312968C911297E3
:107DB0008F9311968C918F93828D8F93FF92EF9278
:107DC00089819A81800F911F9F938F930F94C3464F
:107DD000F80101900020E9F73197E01BF10BE983EE
:107DE000FA83B394CDBFDEBF0F94E70CB81678F2D8
:107DF000E981FA81E00FF11F8DE09AE080839183A1
:107E00001282F80101900020E9F73197E01BF10B95
:107E1000D601ED93FC930F900F90DF91CF911F91BE
:107E20000F91FF90EF90DF90CF90BF900895AF92A9
:107E3000BF92CF92DF92EF921F93CF93DF9300D048
:107E40001F92CDB7DEB719821A821B821C8200975F
:107E500009F47FC06115710509F47BC0E42E5B0154
:107E60006C011FEF120F1B3008F068C0AE014F5FAE
:107E70005F4FBC0184ED91E1CBDD882309F469C03B
:107E80001A3079F5EE2069F069817A816C0D7D1DDB
:107E9000AE014D5F5F4F88E898E0F7DD81110EC0BD
:107EA00058C069817A816C0D7D1DAE014D5F5F4FB9
:107EB00082E798E0EADD882309F44BC069817A8182
:107EC0008B819C81680F791F69837A836C0D7D1D7E
:107ED000AE014D5F5F4F84E798E0D7DD811124C08C
:107EE00038C0EE2089F069817A816C0D7D1D812F6B
:107EF00090E0880F991FAE014D5F5F4F8A58974FF2
:107F0000C4DD811111C025C069817A816C0D7D1D90
:107F1000812F90E0880F991FAE014D5F5F4F805A0F
:107F2000974FB3DD8823A9F029813A818B819C8109
:107F3000820F931FF501808391830BC0AE014F5FC9
:107F40005F4FBC0184ED91E163DD882311F010E007
:107F5000C8CF2496CDBFDEBFDF91CF911F91EF90A8
:107F6000DF90CF90BF90AF90089589E10E9476B8DE
:107F700081E0623009F080E00895CF92DF92EF92C5
:107F8000FF921F93CF93DF9300D01F92CDB7DEB740
:107F900019821A821B821C82009709F453C0611552
:107FA000710509F44FC0142F6B017C01AE014F5FC6
:107FB0005F4FBC0184ED91E12BDD882309F442C0C1
:107FC000173089F01930E1F0113039F569817A8183
:107FD0006E0D7F1DAE014D5F5F4F86E699E018DDA7
:107FE000811127C02FC069817A816E0D7F1DAE017E
:107FF0004D5F5F4F85E099E00BDD81111AC022C013
:1080000069817A816E0D7F1DAE014D5F5F4F84EAFD
:1080100098E0FEDC81110DC015C069817A816E0D7A
:108020007F1DAE014D5F5F4F86E699E0F1DC88234E
:1080300049F029813A818B819C81820F931FF6013F
:10804000808391832496CDBFDEBFDF91CF911F91B6
:10805000FF90EF90DF90CF900895EF92FF920F93F3
:108060001F93CF93DF931F921F92CDB7DEB7198274
:108070001A82009751F16115710539F17B018C016C
:1080800087E10E9476B8662351F0AE014F5F5F4FE3
:10809000B8018DE592E1BCDC81110AC016C0AE01C9
:1080A0004F5F5F4FB80180EE91E1B2DC882369F049
:1080B00089819A81F801E80FF91F2DE020832AE0D9
:1080C00021830296F701808391830F900F90DF91B7
:1080D000CF911F910F91FF90EF900895EF92FF9233
:1080E0000F931F93CF93DF931F921F92CDB7DEB7ED
:1080F000009709F47EC04115510509F47CC0F22EA9
:108100008A01E62EAE014F5F5F4FB801BEDC8111E0
:1081100002C019821A8283E0E81629F18E1538F020
:1081200091E0E91659F082E0E81699F03AC094E03F
:10813000E91619F185E0E81651F133C0E3EFF4E4F4
:1081400001900020E9F73197E35FF44463EF74E4B2
:108150002BC0EAE0F5E401900020E9F7EB50F5448C
:108160006AE075E421C0E1E2F5E401900020E9F75E
:10817000E252F54461E275E417C0E8E3F5E40190EA
:108180000020E9F7E953F54468E375E40DC0EFE436
:10819000F5E401900020E9F7E055F5446FE475E45B
:1081A00003C063EF74E4E0E0EF3008F0EEE0CB01F1
:1081B0008E0F911DFC01108289819A81800F911F81
:1081C0000F94A546F80101900020E9F73197E01BD4
:1081D000F10BFF2091F0C8018E0F911DFC018CE284
:1081E0009DE0808391838AE090E08283938381E0A5
:1081F00005C080E003C080E001C081E00F900F90D7
:10820000DF91CF911F910F91FF90EF9008958F9282
:108210009F92AF92BF92CF92DF92EF92FF920F9315
:108220001F93CF93DF931F921F92CDB7DEB730918C
:10823000023D311104C0FB011082118236C000974B
:10824000A1F1672B91F14115510579F1022F4A01F6
:108250006C010F2EF5E6EF2EF8E1FF2EF02D11E068
:10826000202FA601612FC70139DF8823A9F0F6016D
:1082700001900020E9F731975F01AC18BD089E011D
:108280002F5F3F4FA501B601C4010F94BA3A89810F
:108290009A81A816B90631F41F5FF2E0EF0EF11CC7
:1082A0001630F1F6C4010F94683C0F900F90DF91E7
:1082B000CF911F910F91FF90EF90DF90CF90BF90E3
:1082C000AF909F908F9008958F929F92AF92BF92A0
:1082D000DF92EF92FF920F931F93CF93DF93CDB76F
:1082E000DEB72597CDBFDEBF009709F494C44115D2
:1082F000510509F492C4D22E7A01162FAE014F5FB8
:108300005F4FB701C2DB811102C019821A82163198
:1083100009F06DC00E9448E94B015C01672B682B96
:10832000692BE1F486E10E9476B820E13EE040E06E
:1083300050E00F947A445F934F933F932F938BE7D2
:1083400093E29F938F9389819A818E0D9F1D9F93B6
:108350008F930F94C346CDBFDEBF46C486E10E9413
:1083600076B8992324F586E10E9476B820E13EE0B4
:1083700040E050E00F947A44CA01B9010F94F2161C
:10838000BF92AF929F928F929F938F937F936F93A1
:1083900086E793E29F938F9389819A818E0D9F1D2B
:1083A0009F938F930F94C346CDBFDEBF1DC486E15C
:1083B0000E9476B8BF92AF929F928F9220E13EE0EA
:1083C00040E050E00F947A445F934F933F932F9394
:1083D00087E793E29F938F9389819A818E0D9F1DEA
:1083E0009F938F930F94C346CDBFDEBFFDC3123062
:1083F00060F4812F0E94DBB829813A81BC01C7015A
:10840000820F931F0F94A546EFC3163081F486E0C8
:108410000E9476B88B019C0189819A814BE0BE0154
:108420006B5F7F4F8E0D9F1D0F944B17DDC3153073
:1084300081F485E00E9476B88B019C0189819A8144
:108440004BE0BE016B5F7F4F8E0D9F1D0F94971801
:10845000CBC3123009F06EC082E00E9476B86C3057
:1084600071058105910524F061E070E080E090E005
:10847000013009F049C029813A812E0D3F1DDC01F0
:10848000CB010197A109B109880F991FAE014D5F7A
:108490005F4FB9018553984FF8DA8130F9F4F7014D
:1084A00001900020E9F73197EE19FF09E983FA837B
:1084B00082E00E9476B89F938F937F936F9380E8BA
:1084C00093E29F938F9389819A818E0D9F1D9F9335
:1084D0008F930F94C346CDBFDEBF86C382E00E9458
:1084E00076B89F938F937F936F9381E893E29F93E6
:1084F0008F9389819A818E0D9F1D9F938F930F94E7
:10850000C346CDBFDEBF70C382E00E9476B89F93A2
:108510008F937F936F9386EF99E29F938F938981D7
:108520009A818E0D9F1D9F938F930F94C346CDBF4D
:10853000DEBF5AC31B3059F08DEE810F823038F008
:1085400089EE810F823018F01A3109F05CC0812F5A
:108550000E9476B84B015C01011113C0BF92AF922B
:108560009F926F9386EF99E29F938F9389819A816F
:108570008E0D9F1D9F938F930F94C346CDBFDEBF7B
:1085800033C3672B682B692BF9F469817A816E0DEF
:108590007F1DAE014D5F5F4F87EC97E039DA8111A7
:1085A00023C31F921F921F921F9286EF99E29F93FF
:1085B0008F9389819A818E0D9F1D9F938F930F9426
:1085C000C346CDBFDEBF10C369817A816E0D7F1DAA
:1085D000AE014D5F5F4F84EC97E01ADA811104C35E
:1085E000BF92AF929F928F9286EF99E29F938F9363
:1085F00089819A818E0D9F1D9F938F930F94C346FF
:10860000CDBFDEBFF1C2173009F05CC087E00E9429
:1086100076B84B015C01011113C0BF92AF929F92DB
:108620006F9386EF99E29F938F9389819A818E0D44
:108630009F1D9F938F930F94C346CDBFDEBFD4C2BF
:10864000672B682B692BF9F469817A816E0D7F1D88
:10865000AE014D5F5F4F80EC97E0DAD98111C4C263
:108660001F921F921F921F9286EF99E29F938F9302
:1086700089819A818E0D9F1D9F938F930F94C3467E
:10868000CDBFDEBFB1C269817A816E0D7F1DAE01A3
:108690004D5F5F4F8CEB97E0BBD98111A5C2BF92B4
:1086A000AF929F928F9286EF99E29F938F938981E9
:1086B0009A818E0D9F1D9F938F930F94C346CDBFBC
:1086C000DEBF92C2143009F05CC084E00E9476B82C
:1086D0004B015C01011113C0BF92AF929F926F9347
:1086E00086EF99E29F938F9389819A818E0D9F1DCA
:1086F0009F938F930F94C346CDBFDEBF75C2672B88
:10870000682B692BF9F469817A816E0D7F1DAE01AA
:108710004D5F5F4F85EB97E07BD9811165C21F925A
:108720001F921F921F9286EF99E29F938F938981E8
:108730009A818E0D9F1D9F938F930F94C346CDBF3B
:10874000DEBF52C269817A816E0D7F1DAE014D5F21
:108750005F4F8CEA97E05CD9811146C2BF92AF921D
:108760009F928F9286EF99E29F938F9389819A814E
:108770008E0D9F1D9F938F930F94C346CDBFDEBF79
:1087800033C2133009F0ABC083E00E9476B84B01CE
:108790005C01011113C0BF92AF929F926F9386EF5D
:1087A00099E29F938F9389819A818E0D9F1D9F934C
:1087B0008F930F94C346CDBFDEBF16C291E08916DA
:1087C0009104A104B10461F182E088169104A1042E
:1087D000B10409F445C081149104A104B10409F065
:1087E0005FC069817A816E0D7F1DAE014D5F5F4F65
:1087F00080EA97E00DD98111F7C11F921F921F9255
:108800001F9286EF99E29F938F9389819A818E0DB3
:108810009F1D9F938F930F94C346CDBFDEBFE4C1CE
:1088200069817A816E0D7F1DAE014D5F5F4F87E9D3
:1088300097E0EED88111D8C11F921F921F9281E05C
:108840008F9386EF99E29F938F9389819A818E0D02
:108850009F1D9F938F930F94C346CDBFDEBFC4C1AE
:1088600069817A816E0D7F1DAE014D5F5F4F82E998
:1088700097E0CED88111B8C11F921F921F9282E05B
:108880008F9386EF99E29F938F9389819A818E0DC2
:108890009F1D9F938F930F94C346CDBFDEBFA4C18E
:1088A00069817A816E0D7F1DAE014D5F5F4F80EA59
:1088B00097E0AED8811198C1BF92AF929F928F92EC
:1088C00086EF99E29F938F9389819A818E0D9F1DE8
:1088D0009F938F930F94C346CDBFDEBF85C11931DF
:1088E00009F0ABC089E10E9476B84B015C0101112F
:1088F00013C0BF92AF929F926F9386EF99E29F93BE
:108900008F9389819A818E0D9F1D9F938F930F94D2
:10891000C346CDBFDEBF68C191E089169104A104B2
:10892000B10461F182E088169104A104B10409F454
:1089300045C081149104A104B10409F05FC06981AC
:108940007A816E0D7F1DAE014D5F5F4F8EE897E01F
:108950005FD8811149C11F921F921F921F9286EF0B
:1089600099E29F938F9389819A818E0D9F1D9F938A
:108970008F930F94C346CDBFDEBF36C169817A8124
:108980006E0D7F1DAE014D5F5F4F88E897E040D8C8
:1089900081112AC11F921F921F9281E08F9386EF4F
:1089A00099E29F938F9389819A818E0D9F1D9F934A
:1089B0008F930F94C346CDBFDEBF16C169817A8104
:1089C0006E0D7F1DAE014D5F5F4F80E897E020D8B0
:1089D00081110AC11F921F921F9282E08F9386EF2E
:1089E00099E29F938F9389819A818E0D9F1D9F930A
:1089F0008F930F94C346CDBFDEBFF6C069817A81E5
:108A00006E0D7F1DAE014D5F5F4F8EE897E000D881
:108A10008111EAC0BF92AF929F928F9286EF99E246
:108A20009F938F9389819A818E0D9F1D9F938F9322
:108A30000F94C346CDBFDEBFD7C0123109F05EC070
:108A400082E10E9476B84B015C01011113C0BF9214
:108A5000AF929F926F9386EF99E29F938F93898154
:108A60009A818E0D9F1D9F938F930F94C346CDBF08
:108A7000DEBFBAC0672B682B692B01F569817A814B
:108A80006E0D7F1DAE014D5F5F4F8FE697E00E9438
:108A9000083D8111A9C01F921F921F921F9286EF5D
:108AA00099E29F938F9389819A818E0D9F1D9F9349
:108AB0008F930F94C346CDBFDEBF96C069817A8184
:108AC0006E0D7F1DAE014D5F5F4F87E697E00E9400
:108AD000083D811189C0BF92AF929F928F9286EF1D
:108AE00099E29F938F9389819A818E0D9F1D9F9309
:108AF0008F930F94C346CDBFDEBF76C0153109F00A
:108B00005EC085E10E9476B84B015C01011113C083
:108B1000BF92AF929F926F9386EF99E29F938F934C
:108B200089819A818E0D9F1D9F938F930F94C346C9
:108B3000CDBFDEBF59C0672B682B692B01F569815A
:108B40007A816E0D7F1DAE014D5F5F4F8BE797E021
:108B50000E94083D811148C01F921F921F921F92D0
:108B600086EF99E29F938F9389819A818E0D9F1D45
:108B70009F938F930F94C346CDBFDEBF35C06981ED
:108B80007A816E0D7F1DAE014D5F5F4F86E797E0E6
:108B90000E94083D811128C0BF92AF929F928F9290
:108BA00086EF99E29F938F9389819A818E0D9F1D05
:108BB0009F938F930F94C346CDBFDEBF15C0812F07
:108BC0000E9476B89F938F937F936F9386EF99E27D
:108BD0009F938F9389819A818E0D9F1D9F938F9371
:108BE0000F94C346CDBFDEBFF70101900020E9F727
:108BF0003197EE19FF09DD2091F0C7018E0F911D0D
:108C0000FC018CE29DE0808391838AE090E0828386
:108C1000938381E005C080E003C080E001C081E073
:108C20002596CDBFDEBFDF91CF911F910F91FF90B1
:108C3000EF90DF90BF90AF909F908F9008956F92CC
:108C40007F928F929F92AF92BF92CF92DF92EF92DC
:108C5000FF920F931F93CF93DF931F921F92CDB775
:108C6000DEB70097B1F1672BA1F14115510589F1EC
:108C7000802E922E3A016C010F2EF4E1EF2EFAE1D4
:108C8000FF2EF02D10E0082D292DA601612FC70120
:108C90001BDB8823A9F0F60101900020E9F731974A
:108CA0005F01AC18BD089E012F5F3F4FA501B601C3
:108CB000C3010F94BA3A89819A81A816B90631F492
:108CC0001F5F82E0E80EF11C1C31E9F6C3010F942E
:108CD000683C0F900F90DF91CF911F910F91FF9003
:108CE000EF90DF90CF90BF90AF909F908F907F904C
:108CF0006F9008958F929F92AF92BF92DF92EF9202
:108D0000FF920F931F93CF93DF931F921F92CDB7C4
:108D1000DEB7009709F45EC06115710509F45AC009
:108D20004B017C010E9438BE9F938F9387E893E2AA
:108D30009F938F93FF92EF920F94C346F701019098
:108D40000020E9F73197AF014E195F094231510513
:108D500010F041E150E09E012F5F3F4FB701C40189
:108D60000F94BA3A0F900F900F900F900F900F90B2
:108D7000D12C0F2EF5EBAF2EF9E2BF2EF02D8D2D5D
:108D80000E9452B89F938F937F936F93BF92AF923D
:108D9000FF92EF920F94C346F70101900020E9F78C
:108DA00031978F010E191F099E012F5F3F4FA801B8
:108DB000B701C4010F94BA3ACDBFDEBF89819A8151
:108DC0000817190721F4D39496E1D912D8CFC4011A
:108DD0000F94683C0F900F90DF91CF911F910F91EE
:108DE000FF90EF90DF90BF90AF909F908F9008958D
:108DF0002F923F924F925F926F927F928F929F92AB
:108E0000AF92BF92CF92DF92EF92FF920F931F9398
:108E1000CF93DF93CDB7DEB7E197CDBFDEBF91E053
:108E20009BA76115710509F4B7C34115510509F4F4
:108E3000B5C38A017B0189AB0F949F0C29A921300E
:108E400089F4A80164E771E3CE010B960E94A75153
:108E5000182F86E08BA70E9413FA6DA77EA78FA715
:108E600098AB1AC0A80164E771E3CE010B960E948B
:108E70001C52182F0E9413FA6DA77EA78FA798ABDC
:108E800082E00E948CF8862FAE01445D5F4FBE01E8
:108E9000655D7F4F0E949221112309F481C341E057
:108EA000BE01675F7F4FC7010E946E3D49855A85AD
:108EB000CA01A0E0B0E089839A83AB83BC839E01A2
:108EC000275F3F4FB701CE010B960F94BA3ACE0100
:108ED0000B960F94683CBE01655F7F4FC7010ADFA8
:108EE0000DE0D7010C931AE011961C939E01275FA9
:108EF0003F4F42E050E0B701CE010B960F94BA3AD3
:108F0000CE010B960F94683CE4E7F1E3018B128BE2
:108F10009E01275F3F4F43E150E0BF01CE010B961A
:108F20000F94BA3ACE010B960F94683CB9A9B111CF
:108F30003DC30E9468FA0E9451FA38C301E021E063
:108F4000A701612FC601C0D9882381F0F7010190E4
:108F50000020E9F73197AF014E195F099E01275FA5
:108F60003F4FB701CE010B960F94BA3AE2E0CE0E16
:108F7000D11C1F5F133011F70F2EF6E2CF2EFAE14E
:108F8000DF2EF02D19E001E021E0A701612FC601DD
:108F90009BD9882381F0F70101900020E9F73197F0
:108FA000AF014E195F099E01275F3F4FB701CE0108
:108FB0000B960F94BA3AF2E0CF0ED11C1F5F1B3014
:108FC00011F70F2EF2E18F2E912CA12CB12CF02D48
:108FD00028E182169104A104B10451F401E021E0DA
:108FE000A70169E186E49AE16FD981110EC030C012
:108FF00001E021E0A701682DC401880F991F8C5E54
:10900000954E62D98823C1F007C00F2EF9E18F2E4B
:10901000912CA12CB12CF02DF70101900020E9F743
:109020003197AF014E195F099E01275F3F4FB7018E
:10903000CE010B960F94BA3A33E0830E911CA11C1B
:10904000B11C4AE184169104A104B10408F4C0CF14
:10905000CE010B960F94683C89E00E9476B86F3180
:10906000710581059105C0F4DC01CB01072E7CE080
:10907000880F991FAA1FBB1F7A95D1F7702D89837E
:109080009A83AB83BC8380E090E1A0E0B0E08D8365
:109090009E83AF83B88717C0DC01CB01072E79E030
:1090A000880F991FAA1FBB1F7A95D1F7702D89834E
:1090B0009A83AB83BC8380E092E0A0E0B0E08D8334
:1090C0009E83AF83B88789819A81AB81BC812DA5AE
:1090D0003EA54FA558A9281739074A075B07A1F1F4
:1090E000AE01475F5F4FB70188E998E00E94083DF5
:1090F000813081F4F70101900020E9F73197AF0149
:109100004E195F099E01275F3F4FB701CE010B96B5
:109110000F94BA3ACE010B960F94683CCE010B9691
:109120000F94AF3C39A931113DC20E94DFFA84EBA4
:109130009AE30E941D2281110F94080A84EB9AE39E
:109140000E94122980E03AC2AE01475F5F4FB7012B
:109150008CE898E00E94083D813081F4F70101908D
:109160000020E9F73197AF014E195F099E01275F93
:109170003F4FB701CE010B960F94BA3A48A94F93CF
:109180005FA55F938EA58F939DA59F9388858F93F1
:109190008F818F938E818F938D818F938BE893E254
:1091A0009F938F93FF92EF920F94C346F701019024
:1091B0000020E9F73197AF014E195F099E01275F43
:1091C0003F4FB701CE010B960F94BA3A88E290E078
:1091D00089879A8768E2C7010E944BA4482F50E014
:1091E00060E070E049835A836B837C83682F70E072
:1091F000C7010F94DB18CDBFDEBF8823C9F04981BA
:109200005A819E01275F3F4FB701CE010B960F9405
:10921000BA3A8DE0F70180838AE081839E01275F5F
:109220003F4F42E050E0B701CE010B960F94BA3A9F
:10923000BE016F5F7F4FC7010E942D4049815A8157
:109240009E01275F3F4FB701CE010B960F94BA3AAC
:109250006BE370E0C7010E949EA3A0E0B0E08983A9
:109260009A83AB83BC830E94782981110EC0F701D9
:1092700001900020E9F73197AF014E195F0920E016
:10928000B70187E697E30F94D91149815A816B8121
:109290007C814115510561057105C1F09E01275F73
:1092A0003F4FB701CE010B960F94BA3A8DE0D7012C
:1092B0008C938AE011968C939E01275F3F4F42E08A
:1092C00050E0B701CE010B960F94BA3ACE010B963F
:1092D0000F94683C0E943B5619821A821B821C82A2
:1092E0002DA53EA54FA558A9232B242B252B09F4EA
:1092F00033C180E090E0DC010F2EF4EC2F2EF3E27E
:109300003F2EF02D0F2EF6E98F2EF3E29F2EF02D3B
:10931000880F991FAA1FBB1FBC01CD017E5F8F4F15
:109320009F4F0E9443560E94CE588111FCCF80E08F
:1093300091E0EDE3F1E4DF019C011D92215030400A
:10934000E1F76F010F2EFDE3AF2EF2E4BF2EF02DFB
:109350008F010E945FA3D8018D939D938D01AA1662
:10936000BB06B9F70E940E570F94A21ACE010B96B6
:109370000F94683C412C512C3201F601619171919E
:109380006F01AE014B5F5F4F8BA50E948A1488234B
:1093900009F496C088858F938F818F938E818F93E8
:1093A0008D818F9389819A81AB81BC81840D951DBC
:1093B000A61DB71DBF93AF939F938F939F928F92DC
:1093C000FF92EF920F94C346F70101900020E9F756
:1093D0003197AF014E195F099E01275F3F4FB701DB
:1093E000CE010B960F94BA3A182FCDBFDEBF88235B
:1093F00009F48CC00E947829811126C089819A8144
:10940000AB81BC81840D951DA61DB71DBF93AF9385
:109410009F938F931F921F9340EA53E25F934F9362
:10942000FF92EF920F94C346F70101900020E9F7F5
:109430003197AF014E195F0920E0B70187E697E346
:109440000F94D911CDBFDEBFF70101900020E9F7DD
:109450003197AF014E195F099E01275F3F4FB7015A
:10946000CE010B960F94BA3A182F0E9478298111D9
:109470004DC089819A81AB81BC81840D951DA61D4B
:10948000B71DBF93AF939F938F931F921F93E1EBF1
:10949000F3E2FF93EF93FF92EF920F94C346F7012D
:1094A00001900020E9F73197AF014E195F0920E0E4
:1094B000B70187E697E30F94D911CDBFDEBF26C071
:1094C0000E947829811122C089819A81AB81BC8157
:1094D000840D951DA61DB71DBF93AF939F938F93CA
:1094E0003F922F92FF92EF920F94C346F7010190A3
:1094F0000020E9F73197AF014E195F0920E0B7016D
:1095000087E697E30F94D911CDBFDEBF9FEF491ACD
:10951000590A690A790AA0E84A16510461047104DB
:1095200009F02BCFCE010B960F94683C89819A816C
:10953000AB81BC8180589F4FAF4FBF4F89839A83C7
:10954000AB83BC832DA53EA54FA558A982179307D1
:10955000A407B50708F4DCCECE010B960F94683C47
:10956000CE010B960F94AF3C1092853184E791E3C6
:109570000E94FB5239A9311117C00E94DFFA84EB17
:109580009AE30E941D2281110F94080A84EB9AE34A
:109590000E94122981E012C080E010C080E00EC05D
:1095A00080E00CC080E00AC081E008C00F2EF4E12A
:1095B000CF2EFAE1DF2EF02D10E0C0CCE196CDBF2A
:1095C000DEBFDF91CF911F910F91FF90EF90DF9061
:1095D000CF90BF90AF909F908F907F906F905F9053
:1095E0004F903F902F900895CF92DF92EF92FF928D
:1095F0000F931F93CF93DF931F921F92CDB7DEB7C8
:10960000009709F457C06115710509F453C07B0137
:109610008C01AE014F5F5F4FBC018FE193E10E946F
:10962000083D882309F446C089819A816C012FEF97
:10963000C21AD20AF801E80FF91F20E22083B8010C
:109640006C0D7D1DAE014F5F5F4F88E093E10E947E
:10965000083D882379F189819A81C80ED91EF801C5
:10966000EC0DFD1D8DE0808382E0C80ED11C8AE0E8
:109670008183B8016C0D7D1DAE014F5F5F4F8AED98
:1096800092E10E94083D8823A9F089819A81C80E41
:10969000D91EF801EC0DFD1D8DE0808322E0C20E85
:1096A000D11C8AE08183F801EC0DFD1D1082F701C9
:1096B000C082D1820F900F90DF91CF911F910F91B7
:1096C000FF90EF90DF90CF900895EF92FF920F936D
:1096D0001F93CF93DF93CDB7DEB7A297CDBFDEBF89
:1096E000009709F451C06115710509F44FC07B0161
:1096F0008C0160E0CE01039614D7882309F44BC097
:10970000B701C80171DFF701408151819E012F5FD0
:109710003F4FB801CE0103960F94BA3ACE0103969B
:109720000F94683CF7012081318189819A81281743
:10973000390771F5BE016D5F7F4FC801DBDAA70104
:10974000B8018CE49AE10E94083D813099F4F70158
:10975000408151819E012F5F3F4FB801CE0103969A
:109760000F94BA3AF7012081318189819A812817B3
:10977000390781F4CE0103960F94AF3C81E011D7F5
:109780000F949F0C81E007C080E005C080E003C01B
:1097900080E001C080E0A296CDBFDEBFDF91CF9117
:1097A0001F910F91FF90EF9008950F931F93CF9308
:1097B000DF931F921F92CDB7DEB70F949F0C80915D
:1097C000F53C823009F462C028F4882359F08130D6
:1097D00081F1D6C0843009F485C008F464C08A30B1
:1097E000E1F0CEC060E086E39EE37ED5811107C044
:1097F0006091F63C84EB9AE30E948113C9C00E94F9
:1098000064F4811104C081E08093F53CC1C08AE01A
:109810008093F53C0F94B00ABBC00F94C70A6C3D0F
:1098200075408105910508F4B3C081E08093F53C53
:10983000AFC040E067EE7AE389EE9AE30E946E3DA6
:1098400004EB1AE3F80143A954A99E012F5F3F4F8F
:1098500069EE7AE386E39EE30F94BA3A86E39EE3E9
:109860000F94683CF80123A934A989819A812817AB
:10987000390741F01092F53C6091F63CC8010E9416
:10988000811386C082E08093F53C82C000E021E035
:1098900046E35EE367EE7AE389EE9AE3D0D983E0AC
:1098A0008093F53C75C047EE5AE369EE7AE38CE4A9
:1098B0009AE10E94083D813069F44091E73A509165
:1098C000E83A9E012F5F3F4F69EE7AE386E39EE31D
:1098D0000F94BA3A86E39EE30F94AF3C84E0809302
:1098E000F53C56C00E945BC9882381F10F94FA0BA6
:1098F0008823C9F00E944A1F882309F449C084EBD9
:109900009AE30E941D2281110F94080A84EB9AE3C6
:109910000E9412291092F53C6091F63C84EB9AE388
:109920000E94811335C084EB9AE30E941D228111AD
:109930000F94080A84EB9AE30E9412291092F53CD6
:1099400061E084EB9AE30E94811322C00F94420AE3
:10995000672B682B692BE1F484EB9AE30E941D22AC
:1099600081110F94080A84EB9AE30E941229109245
:10997000F53C6091F63C84EB9AE30E94811308C0A9
:109980001092F53C6091F63C84EB9AE30E948113BF
:109990000F900F90DF91CF911F910F9108959F929B
:1099A000AF92BF92CF92DF92EF92FF920F931F93ED
:1099B000CF93DF9300D0CDB7DEB7009709F471C025
:1099C0006115710509F46DC0A42E6B017C018EE058
:1099D000EFECF3E2D70101900D928A95E1F7F701E0
:1099E00001900020E9F73197EE19FF09E983AF01F3
:1099F00055279E012E5F3F4FB701C6010F94BA3A1B
:109A0000B12C0F2EFCE29F2EF02D8B2D0E9498BFC3
:109A10008B019C0148E0BE016F5F7F4FC7010F942F
:109A2000F91882E08B1550F08981F701E80FF11DDC
:109A300090828F5FF701E80FF11D1082F70101900E
:109A40000020E9F73197EE19FF09E983AF015527A7
:109A50009E012E5F3F4FB701C6010F94BA3A89812C
:109A600090E02A813B818217930721F4B394E4E0CC
:109A7000BE12CBCFAA2081F08DE0F70180838AE06F
:109A8000818382E089839E012E5F3F4F42E050E058
:109A9000B701C6010F94BA3AC6010F94683C0F94FF
:109AA0009F0C2396CDBFDEBFDF91CF911F910F9109
:109AB000FF90EF90DF90CF90BF90AF909F90089570
:109AC0009F92AF92BF92CF92DF92EF92FF920F934D
:109AD0001F93CF93DF931F921F92CDB7DEB70097EE
:109AE00009F4E0C06115710509F4DEC041155105A6
:109AF00009F4DCC0902E122F5A016B017C010F94E7
:109B00009F0C41E0B601C7010E946E3DF601408105
:109B100051819E012F5F3F4FB701C5010F94BA3AA3
:109B2000C5010F94683CF6012081318189819A81B9
:109B30002817390709F0BCC08DE0EDEDF3E2D7013D
:109B400001900D928A95E1F7F70101900020E9F765
:109B50003197AF014E195F0955279E012F5F3F4F87
:109B6000B701C5010F94BA3AC5010F94683CB5011D
:109B7000C701C0D88DE0F70180838AE081839E0110
:109B80002F5F3F4F42E050E0B701C5010F94BA3A52
:109B9000C5010F94683C41E0B501C70100DFA60193
:109BA000B70184EB9AE30E942D3EF601408151817A
:109BB0009E012F5F3F4FB701C5010F94BA3AC5010F
:109BC0000F94683CF6012081318189819A812817A0
:109BD000390709F06FC0B601C7010E94793EF6014E
:109BE000408151819E012F5F3F4FB701C5010F9406
:109BF000BA3AC5010F94683CF60120813181898110
:109C00009A812817390709F057C001E021E0A50122
:109C1000B601C70114D821E0A501B601C7010E9411
:109C200007410E94B53F882331F0492DB601C70195
:109C30000E94BD3F06C0292D412FB601C7010E94D9
:109C4000173FF601408151819E012F5F3F4FB701C1
:109C5000C5010F94BA3AC5010F94683CF601208102
:109C6000318189819A812817390741F5B601C701E9
:109C70000E942D40F601408151819E012F5F3F4F90
:109C8000B701C5010F94BA3AC5010F94683C81E051
:109C9000F6014081518129813A814217530779F0B9
:109CA00080E00DC080E00BC080E009C080E007C00C
:109CB00080E005C080E003C080E001C080E00F903C
:109CC0000F90DF91CF911F910F91FF90EF90DF9058
:109CD000CF90BF90AF909F9008952F923F924F9258
:109CE0005F926F927F928F929F92AF92BF92CF922C
:109CF000DF92EF92FF920F931F93CF93DF93CDB735
:109D0000DEB7A897CDBFDEBF4115510509F4D7C115
:109D10002115310509F4D5C16115710509F4D3C1C7
:109D2000280169011A017B0188A70F949F0CA601E5
:109D300064E771E3CE010796A7D6882309F4C5C16D
:109D400041E0BE016B5F7F4FC1010E946E3D4D81BE
:109D50005E819E012B5F3F4FB101CE0107960F94AC
:109D6000BA3ACE0107960F94683CBE01695F7F4FF7
:109D7000C1010E947A461DE0F10110830AE00183CF
:109D80009E012B5F3F4F42E050E0B101CE010796AC
:109D90000F94BA3ACE0107960F94683CE4E7F1E3DA
:109DA000118B028B9E012B5F3F4F43E150E0BF01BF
:109DB000CE0107960F94BA3ACE0107960F94683CED
:109DC0000F2EF4E1CF2EFAE1DF2EF02D10E001E0AE
:109DD00021E0A101612FC6010E946441882381F026
:109DE000F10101900020E9F73197AF0142195309C1
:109DF0009E012B5F3F4FB101CE0107960F94BA3AF7
:109E0000F2E0CF0ED11C1F5F133009F70F2EF6E2E0
:109E1000CF2EFAE1DF2EF02D19E001E021E0A101C3
:109E2000612FC6010E946441882381F0F1010190F5
:109E30000020E9F73197AF01421953099E012B5FCA
:109E40003F4FB101CE0107960F94BA3A22E0C20EFD
:109E5000D11C1F5F1B3009F70F2EF2E18F2E912CC2
:109E6000A12CB12CF02D88E188169104A104B10435
:109E700091F401E021E0A10169E186E49AE10E9408
:109E80006441811116C00F2EFCE18F2E912CA12C64
:109E9000B12CF02D31C001E021E0A101682DC401F9
:109EA000880F991F8C5E954E0E9464418823C1F0F3
:109EB00007C00F2EF9E18F2E912CA12CB12CF02D83
:109EC000F10101900020E9F73197AF0142195309E0
:109ED0009E012B5F3F4FB101CE0107960F94BA3A16
:109EE00093E0890E911CA11CB11CEAE18E1691042D
:109EF000A104B10408F4B7CF1F92F8A5FF938AEE2E
:109F000093E29F938F933F922F920F94C346F10158
:109F100001900020E9F73197AF01421953099E01E2
:109F20002B5F3F4FB101CE0107960F94BA3ACE0195
:109F300007960F94683C612C712C0F900F900F9036
:109F40000F900F900F90411451046104710409F4B3
:109F5000A7C0870175016401812C912C5401F8017F
:109F600041915191619171918F019E012F5F3F4FFE
:109F700088A50E94E42D882309F482C08C818F93E8
:109F80008B818F938A818F9389818F93BF92AF92B8
:109F90009F928F9286E993E29F938F933F922F92A5
:109FA0000F94C346F10101900020E9F73197AF010A
:109FB000421953099E012B5F3F4FB101CE01079615
:109FC0000F94BA3A8FA3CDBFDEBF9FA1992309F4A6
:109FD00057C00E94782981111FC0FF92EF92DF9233
:109FE000CF921F92EFA1EF9380EA93E29F938F931A
:109FF0003F922F920F94C346F10101900020E9F7A0
:10A000003197AF014219530920E0B10187E697E388
:10A010000F94D911CDBFDEBFF10101900020E9F707
:10A020003197AF01421953099E012B5F3F4FB10198
:10A03000CE0107960F94BA3A8FA30E947829811116
:10A040001FC0FF92EF92DF92CF921F929FA19F932A
:10A05000E1EBF3E2FF93EF933F922F920F94C3460D
:10A06000F10101900020E9F73197AF01421953093E
:10A0700020E0B10187E697E30F94D911CDBFDEBF91
:10A080009FEF891A990AA90AB90AEFEFCE1ADE0AD8
:10A09000EE0AFE0A84149504A604B70408F45FCF00
:10A0A000CE0107960F94683CCE0107960F94AF3C03
:10A0B0001092853184E791E39ED281E007C080E071
:10A0C00005C080E003C080E001C080E0A896CDBF5D
:10A0D000DEBFDF91CF911F910F91FF90EF90DF9046
:10A0E000CF90BF90AF909F908F907F906F905F9038
:10A0F0004F903F902F900895089580918931089551
:10A1000008951092893180918831882331F010921E
:10A11000883186E59EE30D94AF3C089586E59EE385
:10A120000D94AF3C0895809188310895CF92DF92CD
:10A13000EF92FF921F93CF93DF93CDB7DEB768976F
:10A14000CDBFDEBF6C017B0184E1E5EFF3E2DE0110
:10A15000159601900D928A95E1F7DA01C9010196F1
:10A16000A11DB11D883E23E09207A105B1050CF4A5
:10A1700060C01F921F921F9281E08F9383EE90E246
:10A180009F938F93CE0101969F938F930F94C34615
:10A190008981898B8A818A8B8B818B8B80E38D83EC
:10A1A0008AE38E83CDBFDEBFE114F10459F0D701FD
:10A1B000FE0138969E01245F3F4F8D918193E217F7
:10A1C000F307D9F710E346E0BE016B5F7F4F86E5EA
:10A1D0009EE30F941C3899EF980F9230C8F48B8946
:10A1E000893399F48A89893361F48989893321F41F
:10A1F0001092883180E03CC08F5F898B1A8B1B8B5B
:10A20000E2CF1B8B8F5F8A8BDECF8F5F8B8BDBCF99
:10A21000882321F01092883180E02AC081E0809369
:10A220008831BE01695F7F4FC6010F94A54681E06A
:10A230001FC0BF93AF939F938F9383EE90E29F9342
:10A240008F93CE0101969F938F930F94C34689817C
:10A25000898B8A818A8B8B818B8B80E38D838AE3C8
:10A260008E83CDBFDEBFE114F10409F0A0CFAACFE9
:10A270006896CDBFDEBFDF91CF911F91FF90EF9029
:10A28000DF90CF90089580E00E94ABF4882361F0C6
:10A290008250823030F580918931882311F11092FB
:10A2A000893110928831089580918931811119C0C6
:10A2B00081E0809389318EE292E0EAE8F1E3DF0108
:10A2C0009C011D9221503040E1F7BF0180E00F94C6
:10A2D000FE378B3019F410928831089581E0809315
:10A2E000883108958AE00895CF93DF93CDB7DEB724
:10A2F0006097CDBFDEBF009719F120E329832AE3E1
:10A300002A832BE0E9E0F4E2DE01139601900D923E
:10A310002A95E1F7613041F441E0BE016F5F7F4F64
:10A320000F941C38982F07C04AE0BE016F5F7F4F23
:10A330000F941C38982F81E0992319F080E001C018
:10A3400080E06096CDBFDEBFDF91CF910895DF92B0
:10A35000EF92FF920F931F93CF93DF93CDB7DEB7AA
:10A360006497CDBFDEBF8C0184E1E4E1F4E2DE015D
:10A37000119601900D928A95E1F70115110509F4E6
:10A3800049C06115710509F447C080E389838AE3F8
:10A390008A834115510559F0DA01FE0134969E0178
:10A3A000285F3F4F9D919193E217F307D9F77B0107
:10A3B0000F2EF0E3DF2EF02D46E0BE016F5F7F4FE2
:10A3C000C8010F941C3899EF980F9230A8F49F851C
:10A3D000993379F48E85893341F48D858933F1F091
:10A3E0008F5F8D87DE86DF86E7CFDF868F5F8E8784
:10A3F000E3CF9F5F9F87E0CF811112C081E1FE0113
:10A400003396D70101900D928A95E1F7F701118AF1
:10A4100081E007C080E005C080E003C080E001C0AB
:10A4200080E06496CDBFDEBFDF91CF911F910F9189
:10A43000FF90EF90DF900895DF92EF92FF920F93DD
:10A440001F93CF93DF93CDB7DEB76497CDBFDEBF49
:10A450008C0184E1E8E2F4E2DE01119601900D92B4
:10A460008A95E1F70115110509F449C061157105D7
:10A4700009F447C080E389838AE38A834115510543
:10A4800059F0DA01FE0134969E01285F3F4F9D91FD
:10A490009193E217F307D9F77B010F2EF0E3DF2E3C
:10A4A000F02D46E0BE016F5F7F4FC8010F941C384E
:10A4B00099EF980F9230A8F49F85993379F48E859F
:10A4C000893341F48D858933F1F08F5F8D87DE8686
:10A4D000DF86E7CFDF868F5F8E87E3CF9F5F9F8723
:10A4E000E0CF811112C081E1FE013396D7010190C6
:10A4F0000D928A95E1F7F701118A81E007C080E0AB
:10A5000005C080E003C080E001C080E06496CDBF5C
:10A51000DEBFDF91CF911F910F91FF90EF90DF9001
:10A5200008950F931F93CF93DF93CDB7DEB7609756
:10A53000CDBFDEBF009761F18C0180E389838AE3A0
:10A540008A838BE0ECE3F4E2DE01139601900D9236
:10A550008A95E1F7613049F441E0BE016F5F7F4FBA
:10A56000C8010F941C38982F0EC041E060E0CE0166
:10A5700003960F948C3E4AE0BE016F5F7F4FC80187
:10A580000F941C38982F81E0992319F080E001C0C6
:10A5900080E06096CDBFDEBFDF91CF911F910F911C
:10A5A0000895CF93DF93CDB7DEB76097CDBFDEBF01
:10A5B0009BE0ECE3F4E2DE01119601900D929A9596
:10A5C000E1F7813041F441E061E0CE0101960F9462
:10A5D0008C3E982F07C041E060E0CE0101960F94B9
:10A5E0008C3E982F81E0911180E06096CDBFDEBF58
:10A5F000DF91CF910895009721F041E061E00D9443
:10A600008C3E08951F93CF93DF93CDB7DEB7649749
:10A61000CDBFDEBF009701F1162FBC0180E3898317
:10A620008AE38A83CE0103960F94A546113041F444
:10A6300041E061E0CE0101960F948C3E982F07C057
:10A6400041E060E0CE0101960F948C3E982F81E0AE
:10A65000992319F080E001C080E06496CDBFDEBF91
:10A66000DF91CF911F910895EF92FF920F931F9367
:10A67000CF93DF93CDB7DEB76497CDBFDEBF611553
:10A68000710589F1009789F18B017C0180E3898351
:10A690008AE38A83CE0103960F94A54643E0BE0168
:10A6A0006F5F7F4FC7010F941C38873069F460E0FB
:10A6B000C801A8DF982F8823D9F043E0BE016F5F5F
:10A6C0007F4FC7010F941C38811111C0F7014285DB
:10A6D000538564857585C7010F94BA3C91E0882342
:10A6E00039F090E005C090E003C090E001C090E038
:10A6F000892F6496CDBFDEBFDF91CF911F910F915F
:10A70000FF90EF900895CF93DF93CDB7DEB76097BA
:10A71000CDBFDEBF0097C1F020E329832AE32A835F
:10A720002AE0E7E4F4E2DE01139601900D922A9507
:10A73000E1F741E0BE016F5F7F4F0F941C3891E05D
:10A74000882319F090E001C090E0892F6096CDBF7A
:10A75000DEBFDF91CF9108953F924F925F926F924B
:10A760007F928F929F92AF92BF92CF92DF92EF92A1
:10A77000FF920F931F93CF93DF93CDB7DEB761970F
:10A78000CDBFDEBF6115710509F470C0009709F4F3
:10A790006FC04115510509F46DC03FEF320F3830DD
:10A7A00008F06AC0322E7A018C01FB01138A41E065
:10A7B0000F941C38811162C0F8014285538564856D
:10A7C0007585483EF3E05F076105710508F458C0E0
:10A7D000413B84E058076105710508F053C0C32C64
:10A7E000D12C5601E6E0AE0EB11C25010B2C000C5D
:10A7F000660877084419550966097709C8010F9456
:10A80000BA3C811141C0A50160E070E0CE01039621
:10A810000F949E469E012F5F3F4FA501BE016D5FC5
:10A820007F4FC8010F946E39C8010F94AF3CFE01F1
:10A83000EC0DFD1D12868E010D5F1F4F812C912C9A
:10A840005401A601B801C7010F948846892BF1F085
:10A85000FFEF8F1A9F0AAF0ABF0A0F5F1F4F4814FE
:10A8600059046A047B0468F780E011C080E00FC0DF
:10A8700080E00DC080E00BC080E009C080E007C030
:10A8800081E005C080E003C080E001C081E0619606
:10A89000CDBFDEBFDF91CF911F910F91FF90EF9061
:10A8A000DF90CF90BF90AF909F908F907F906F90F0
:10A8B0005F904F903F9008954F925F926F927F927A
:10A8C000AF92BF92CF92DF92EF92FF920F931F93BE
:10A8D000CF93DF93CDB7DEB76897CDBFDEBF6801FA
:10A8E00014E1E5EFF3E2DE01159601900D921A9561
:10A8F000E1F7009709F491C0C114D10409F48FC0A5
:10A90000EFEFEE0DE83008F08CC0860129013A0126
:10A910005B016C01283E83E03807410551050CF4CA
:10A9200082C01F921F921F9281E08F9383EE90E26C
:10A930009F938F93CE0101969F938F930F94C3465D
:10A940008981898B8A818A8B8B818B8B80E38D8334
:10A950008AE38E83CDBFDEBFA114B10459F0D501C7
:10A96000FE0138969E01245F3F4F8D918193E2173F
:10A97000F307D9F70F2EF0E3FF2EF02D46E0BE01CE
:10A980006B5F7F4F86E59EE30F941C3899EF980F1D
:10A99000923090F52E2DA801BE016B5F7F4F86E5AA
:10A9A0009EE3DADE882379F060E0C6012BDE88239F
:10A9B00051F04AE0BE016B5F7F4F86E59EE30F9446
:10A9C0001C388823F9F09B89993399F48A89893353
:10A9D00061F48989893321F41092883180E042C082
:10A9E0008F5F898BFA8AFB8AC9CFFB8A8F5F8A8B3C
:10A9F000C5CF9F5F9B8BC2CF882321F010928831F7
:10AA000080E030C081E080938831BE01695F7F4F74
:10AA1000C6010F94A54681E025C080E023C080E0F8
:10AA200021C080E01FC07F926F925F922F9383EED0
:10AA300090E29F938F93CE0101969F938F930F94F3
:10AA4000C3468981898B8A818A8B8B818B8B80E33A
:10AA50008D838AE38E83CDBFDEBFA114B10409F0DC
:10AA60007ECF88CF6896CDBFDEBFDF91CF911F919B
:10AA70000F91FF90EF90DF90CF90BF90AF907F90BD
:10AA80006F905F904F900895DF92EF92FF920F9337
:10AA90001F93CF93DF93CDB7DEB76497CDBFDEBFF3
:10AAA0008C0184E1E1E5F4E2DE01119601900D9262
:10AAB0008A95E1F70115110509F449C06115710581
:10AAC00009F447C080E389838AE38A8341155105ED
:10AAD00059F0DA01FE0134969E01285F3F4F9D91A7
:10AAE0009193E217F307D9F77B010F2EF0E3DF2EE6
:10AAF000F02D46E0BE016F5F7F4FC8010F941C38F8
:10AB000099EF980F9230A8F49F85993379F48E8548
:10AB1000893341F48D858933F1F08F5F8D87DE862F
:10AB2000DF86E7CFDF868F5F8E87E3CF9F5F9F87CC
:10AB3000E0CF811112C081E1FE013396D70101906F
:10AB40000D928A95E1F7F701118A81E007C080E054
:10AB500005C080E003C080E001C080E06496CDBF06
:10AB6000DEBFDF91CF911F910F91FF90EF90DF90AB
:10AB700008958091B83308950895089581E08093F1
:10AB8000B83308951092B8330895CF92DF92EF92C0
:10AB9000FF920F931F936623B9F081111DC0C12C42
:10ABA000D12C760100E010E62AEE30E040E06CE1C6
:10ABB00070E280EB98E00F9496246CE170E280EBF9
:10ABC00098E00F94E02408C0811106C06CE170E2A7
:10ABD00080EB98E00F94F6241F910F91FF90EF9077
:10ABE000DF90CF900895CF93DF931F921F92CDB740
:10ABF000DEB78091B9339091BA33A091BB33B09155
:10AC0000BC33072E75E1B695A795979587957A95EC
:10AC1000D1F7702D61E0B9DF87ED8A8341E050E024
:10AC2000BE016E5F7F4F80EB98E00F94B12441E04E
:10AC300050E0BE016F5F7F4F80EB98E00F94C82417
:10AC400089818823A4F78091B9339091BA33A09178
:10AC5000BB33B091BC33072E75E1B695A795979598
:10AC600087957A95D1F7702D60E08FDF0F900F9068
:10AC7000DF91CF91089580EB98E00F945F241092BC
:10AC8000BD3381E008951F93CF93DF93CDB7DEB737
:10AC90002C97CDBFDEBF6115710520E282079105BB
:10ACA00008F0A1C0DC01CB018093B9339093BA3393
:10ACB000A093BB33B093BC338091BD33811193DF3C
:10ACC0001092BD338091B9339091BA33A091BB33C8
:10ACD000B091BC33072E75E1B695A79597958795EA
:10ACE0007A95D1F7702D61E050DF82ED8C8741E0DD
:10ACF00050E0BE01645F7F4F80EB98E00F94B12479
:10AD00008091B9339091BA33A091BB33B091BC33E9
:10AD1000AC01BD01032E39E07695679557954795AF
:10AD20003A95D1F7302D032E3AE0440F551F661F98
:10AD3000771F3A95D1F7302D9170AA27BB27842B26
:10AD4000952BA62BB72B89839A83AB83BC838B81EE
:10AD50008D8341E050E0BE016B5F7F4F80EB98E058
:10AD60000F94B1248A818E8341E050E0BE016A5F76
:10AD70007F4F80EB98E00F94B12489818F8341E06D
:10AD800050E0BE01695F7F4F80EB98E00F94B124E3
:10AD900015E5188741E050E0BE01685F7F4F80EB0A
:10ADA00098E00F94B124198741E050E0BE01675F3D
:10ADB0007F4F80EB98E00F94B1241A8741E050E078
:10ADC000BE01665F7F4F80EB98E00F94B1241B8734
:10ADD00041E050E0BE01655F7F4F80EB98E00F944B
:10ADE000B12481E001C080E02C96CDBFDEBFDF91B1
:10ADF000CF911F910895052E59E0660F771F881F88
:10AE0000991F5A95D1F7502D6115710520E28207DF
:10AE1000910510F438CF089580E008958091B933FA
:10AE20009091BA33A091BB33B091BC330097A10588
:10AE3000B10569F00197A109B109072E75E1B69531
:10AE4000A795979587957A95D1F7702D01C080E0E9
:10AE500060E09BDE1092BD330895CF93DF93CDB7B2
:10AE6000DEB72897CDBFDEBF6115710520E28207EE
:10AE7000910508F078C0DC01CB018093B933909341
:10AE8000BA33A093BB33B093BC338091BD338111EF
:10AE9000AADE1092BD338091B9339091BA33A0915C
:10AEA000BB33B091BC33072E75E1B695A795979546
:10AEB00087957A95D1F7702D61E067DE82E8888703
:10AEC00041E050E0BE01685F7F4F80EB98E00F9457
:10AED000B1248091B9339091BA33A091BB33B09132
:10AEE000BC33AC01BD01032E39E0769567955795CB
:10AEF00047953A95D1F7302D032E3AE0440F551F70
:10AF0000661F771F3A95D1F7302D9170AA27BB277E
:10AF1000842B952BA62BB72B89839A83AB83BC8379
:10AF20008B818D8341E050E0BE016B5F7F4F80EBF2
:10AF300098E00F94B1248A818E8341E050E0BE01F5
:10AF40006A5F7F4F80EB98E00F94B12489818F83F3
:10AF500041E050E0BE01695F7F4F80EB98E00F94C5
:10AF6000B12481E001C080E02896CDBFDEBFDF9133
:10AF7000CF910895CF93DF931F92CDB7DEB7809125
:10AF8000B9339091BA33A091BB33B091BC33AC01CB
:10AF9000BD01517066277727452B462B472B31F192
:10AFA000198241E050E0BE016F5F7F4F80EB98E077
:10AFB0000F94B1248091B9339091BA33A091BB33EF
:10AFC000B091BC330196A11DB11D8093B93390930C
:10AFD000BA33A093BB33B093BC33AC01BD01517005
:10AFE00066277727452B462B472BD1F60097A105DF
:10AFF000B10569F00197A109B109072E75E1B69570
:10B00000A795979587957A95D1F7702D01C080E027
:10B0100060E0BBDD81E08093BD330F90DF91CF9185
:10B0200008950F931F93CF93DF931F92CDB7DEB791
:10B030008091BD338823B1F01092BD338091B93334
:10B040009091BA33A091BB33B091BC33BC01CD0118
:10B05000052E59E096958795779567955A95D1F77E
:10B06000502DC9DE41E050E0BE016F5F7F4F80EBA5
:10B0700098E00F94C8248091B9339091BA33A0918D
:10B08000BB33B091BC33AC01BD014F5F5F4F6F4F1D
:10B090007F4F4093B9335093BA336093BB3370936F
:10B0A000BC338A019B01117022273327012B022B0D
:10B0B000032BA1F4452B462B472B51F0072E75E1AE
:10B0C000B695A795979587957A95D1F7702D01C07C
:10B0D00080E060E05ADD81E08093BD3389810F908C
:10B0E000DF91CF911F910F9108950F931F93CF93ED
:10B0F000DF931F92CDB7DEB7182F8091BD33882321
:10B1000049F06091B9337091BA338091BB3390911B
:10B11000BC33A3DE198341E050E0BE016F5F7F4F77
:10B1200080EB98E00F94B1248091B9339091BA33B9
:10B13000A091BB33B091BC33AC01BD014F5F5F4FF9
:10B140006F4F7F4F4093B9335093BA336093BB3303
:10B150007093BC338A019B01117022273327012B86
:10B16000022B032BA1F4452B462B472B51F0072E26
:10B1700075E1B695A795979587957A95D1F7702D36
:10B1800001C080E060E001DD81E08093BD3381E0BB
:10B190000F90DF91CF911F910F910895CF93DF937F
:10B1A0001F921F92CDB7DEB78091BD33882309F47B
:10B1B00040C08091B9339091BA33A091BB33B09124
:10B1C000BC33072E75E1B695A795979587957A9527
:10B1D000D1F7702D61E0D9DC87ED8A8341E050E042
:10B1E000BE016E5F7F4F80EB98E00F94B12441E089
:10B1F00050E0BE016F5F7F4F80EB98E00F94C82452
:10B200008091B9339091BA33A091BB33B091BC33E4
:10B21000072E75E1B695A795979587957A95D1F7FD
:10B22000702D60E0B2DC89818095881F8827881F97
:10B2300001C080E00F900F90DF91CF910895CF93E0
:10B24000DF93EC01803C28E0920729F468E083E07A
:10B250000F94E02310C0803C29E0920729F468E0B5
:10B2600084E00F94E02307C0803C9A4021F468E01A
:10B2700085E00F94E023888180618883DF91CF91FE
:10B280000895EF92FF920F931F93CF937C01C42FE9
:10B29000B901A80100E010E62AEE30E00E944B63FD
:10B2A000882344F0F7018081CC0FCC0FCC70837FD2
:10B2B000C82BC083CF911F910F91FF90EF900895FD
:10B2C00080E0089591E0811101C090E09093763E76
:10B2D00081E08093442008950F931F9300E41BE5C1
:10B2E0002FE130E040E054E361E082E00E94CE7361
:10B2F000811105C06CE679E582E00E941E751F9100
:10B300000F910895CF93DF931092E3331092E433BB
:10B310000F940C25811104C01092FC33D0E012C0B0
:10B3200081508093FC332ADCD82F882359F0C0E069
:10B3300060E08C2F0F942225CF5F8091FC338C1717
:10B34000B8F7CADF8D2FDF91CF910895C5CF08954B
:10B350000F931F9306EA19E52DE030E048E450E230
:10B3600060E081E80E94CE73811105C068EA79E54A
:10B3700081E80E941E751F910F9108958091E4331A
:10B38000882341F082E00E94F7746EEB79E582E059
:10B390000C941E7508958091E433882341F081E870
:10B3A0000E94F7746BEC79E581E80C941E750895A2
:10B3B0008091502090915120A0915220B091532023
:10B3C000892B8A2B8B2B59F080910C34882324F401
:10B3D00081E80E94F77403C082E00E94F7748091B4
:10B3E000043490910534A0910634B09107348093D1
:10B3F0004C2090934D20A0934E20B0934F20A8CF87
:10B400000895E8EEF3E382E1DF011D928A95E9F702
:10B4100080EF80838AE087830895DF92EF92FF9226
:10B420000F931F93CF93DF93D82EC62FD72F122FB2
:10B43000032FF42EE52EE5DF81E080935420E8EE23
:10B44000F3E3D282E382F48205831683D487C5872F
:10B45000DF91CF911F910F91FF90EF90DF900895B2
:10B4600020E030E0A90160E074E285E0D6CF0895E5
:10B470000F931F9320910C3442276CF000915020C1
:10B480001091512020915220309153200617170718
:10B490002807390720F4E4DF8BDF80E001C081E07A
:10B4A0001F910F91089520E030E0A90160E070E065
:10B4B00084E0B3CF08950F931F93262F30E001E867
:10B4C0001AE5AC0161E081E80E94CE73811102C0EF
:10B4D000EADF6EDF1F910F91089520E030E0A901AF
:10B4E00060E078E286E099CF089520E030E0A9019D
:10B4F00060E07AE382E091CF089583DF10925420D8
:10B500000895CF93DF93811111C0EB01F6DFE8E4DA
:10B51000F0E280859185A285B3858C1B9D0BA109E6
:10B52000B10980879187A287B38742DFDF91CF91EE
:10B5300008951F93CF93DF93D82F84E1E8ECF3E3D2
:10B54000DF011D928A95E9F7DD2331F090911734E0
:10B55000E0EDF3E318E005C090911334ECECF3E375
:10B5600014E0809111348F738C3111F08F3339F4E2
:10B570008CE180838AE0818385E08383145FC12F1F
:10B58000911708F4C92F8C2F90E0A0E0B0E040E8BC
:10B59000BC01CD016DDF882309F180910D340F943A
:10B5A0002925811102C020E001C020E8DD2361F0DF
:10B5B000E8ECF3E3812F90E00297982789279827FA
:10B5C00080839183238306C0E8ECF3E38FEF810F40
:10B5D000808322836C2F88EC93E36DDFDF91CF9122
:10B5E0001F910895CF93C82F81110FC080910D3402
:10B5F0000F942925882349F020E030E0A90160E07C
:10B6000077E287E00ADFD4DE39C0AEEDB3E3E0E0F5
:10B61000F4E3818913968C931397828912968C9305
:10B620001297838911968C93119784898C93ACED32
:10B63000B3E3868911968C93119787898C936091D7
:10B64000DC337091DD33CB01A0E0B0E0BC01CD0173
:10B65000052E59E0660F771F881F991F5A95D1F75D
:10B66000502DC11102C040E001C040E801DF882335
:10B6700029F0C093E23381E08093E333CF910895C2
:10B680000F931F93CF93DF93811132C16F317105F7
:10B6900069F48091003490910134A0910234B0910A
:10B6A000033485359345A244B34431F081E080935F
:10B6B000E43364DE70DE1CC1E0E0F4E395859F7046
:10B6C00095878091FC33891718F4CADE71DE10C1AA
:10B6D000E0E0F4E340855185628573854093502016
:10B6E000509351206093522070935320478550E02F
:10B6F0004B35510508F0EEC0FA018827E85BFE4F94
:10B700008F4F0D949644C0911334C33108F0C2E1B9
:10B710008C2F90E0A0E0B0E040E8BC01CD01A8DEB5
:10B72000882309F4E5C06C2F88EE93E3C4DEE0C003
:10B73000C0911334C53208F0C4E28C2F90E0A0E031
:10B74000B0E040E8BC01CD0193DE882309F4D0C00D
:10B7500080911034837021F4D0911134DD2319F0DD
:10B760007FDE26DEC5C080910D340F943025811117
:10B77000D0E800E210E2F801D18380910D340F94FB
:10B78000372520E1FC013196A0E3B0E201900D9253
:10B790002A95E1F7F8018089882309F4A4C0823250
:10B7A00009F4A3C0E1E3F0E281E09191992309F467
:10B7B0009DC0923209F49AC08F5F8031B1F708C002
:10B7C000E82FF0E0E05EFF4D908B8F5F8031C1F796
:10B7D0006C2F80E290E26FDE8BC080E0AADE88C032
:10B7E00081E0A7DE85C0892F0F940E25823039F0C5
:10B7F000833019F0811105C006C06FDE05C075DE0B
:10B8000003C051DE01C079DED3DD72C040E868E0DC
:10B8100070E080E090E02CDE882309F469C060ECE1
:10B8200073E380910D340F941525823041F08330FD
:10B8300019F0811107C009C050DEBADD59C055DECC
:10B84000B7DD56C030DEB4DD53C0E0ECF3E380E09A
:10B8500090E0A2E0B0E084839583A683B7838081E3
:10B860009181A281B3815A2F4B2F60E070E098271D
:10B8700089279827A0E0B0E0DC0199278827842B4E
:10B88000952BA62BB72B80839183A283B38368E08B
:10B89000CF0111DE2DC08091133481FF06C0809549
:10B8A000682F6170892F0F94222527DE81DD20C04B
:10B8B00080911334811102C020DE01C0D1DD78DD1A
:10B8C00017C01BDE75DD14C081E08CDE11C080E086
:10B8D00089DE0EC020E030E0A90160E070E285E082
:10B8E0009CDD66DD05C080E001C080E090E268CFAD
:10B8F000DF91CF911F910F9108951092E33342C9C8
:10B90000089580917F3E8823F4F480768032D9F5C3
:10B910008091803E8E3FC9F58091853E9091863E14
:10B920000197A9F58091813E9091823E892B89F5FE
:10B93000EFE7FEE38CEF93E38087918781E090E06F
:10B940008287938708958076803229F58091803EA2
:10B950008F3F19F58091853E9091863E892BF9F4B1
:10B960008091813E9091823E892BD9F41092E433EC
:10B970001092E33382E00E948C7481E80E948C7400
:10B98000ABDC81E0089580E0089580E0089580E0D8
:10B99000089580E0089580E0089580E0089580E0B3
:10B9A000089580E00895CF93C091E333CC23A9F1AB
:10B9B0001092E3338091E233882389F02091DC33C5
:10B9C0003091DD334091DE335091DF336091E033CD
:10B9D0007091E13380910D340F943F2510C0209178
:10B9E000DC333091DD334091DE335091DF336091B1
:10B9F000E0337091E13380910D340F9463258230F0
:10BA000041F0833021F0811106C077DD05C065DD8E
:10BA100003C06BDD01C047DDCBDC8C2FCF910895D7
:10BA2000EF92FF920F931F93CF93DF93982F809104
:10BA30004420882309F448C0109244202115310580
:10BA400011F0890102C002E619E5911102C082E0FD
:10BA500001C081E8E9017A01AB01970160E00E9431
:10BA6000CE73811104C091E0909344202DC0CD2B62
:10BA7000D9F4809144208823E1F38091763E8111AE
:10BA800022C0E8E4F0E280859185A285B3858E1915
:10BA90009F09A109B10980879187A287B3879091F7
:10BAA000763E81E0892710C0E8E4F0E240855185C8
:10BAB000628573854E195F09610971094087518755
:10BAC0006287738701C080E0DF91CF911F910F9152
:10BAD000FF90EF900895E0912534F0912634019085
:10BAE000F081E02D228133812E0F3F1FFC01408128
:10BAF000E40FF11DE217F307A0F481818430A1F077
:10BB0000861306C014C081818430A1F08617A9F085
:10BB10008081E80FF11DE217F307A8F380E090E0C1
:10BB2000089580E090E0089580E090E008958E2FE1
:10BB30009F2F089580E090E008958E2F9F2F089505
:10BB40008091813E8F770C94E9720895909127340B
:10BB5000992381F1E0912534F09126340190F08110
:10BB6000E02D9481891740F5E0932334F093243439
:10BB7000228133812E0F3F1FE217F307F8F49181E2
:10BB8000943061F49281891309C09381961306C0A1
:10BB9000E0932334F093243481E008959081E90FF9
:10BBA000F11DE217F30758F3E0932334F0932434A4
:10BBB00080E0089580E0089580E0089580E0089591
:10BBC000EF92FF921F93CF93DF93C82F60E0BEDF09
:10BBD000182F882381F1A0912534B0912634EC2FC1
:10BBE000F0E0EE0FFF1F12968D919C911397E80FD6
:10BBF000F91FE080F180D7011696ED91FC9117971F
:10BC00001995682F8C2FA2DF182F8823A1F0C091DF
:10BC10002334D091243465E0CE015DDFEC01892B23
:10BC200021F08A810E94DB74F6CFD7011296ED9144
:10BC3000FC9113971995812FDF91CF911F91FF9060
:10BC4000EF9008951F93CF93DF93182F7FDF882302
:10BC500041F1C0912334D091243465E0CE013BDF23
:10BC6000EC01892B49F04C815D816B818A810E94B6
:10BC7000F6728111F2CF15C0A0912534B09126340F
:10BC8000E12FF0E0EE0FFF1F12968D919C9113971C
:10BC9000E80FF91F0190F081E02D0190F081E02D77
:10BCA0001995DF91CF911F9108950C948172089599
:10BCB000CF93809127348823C1F0E0912534F0910F
:10BCC00026340190F081E02D8481882371F0C0E05A
:10BCD0008C2F76DFCF5FE0912534F09126340190F0
:10BCE000F081E02D8481C81798F31092273481E009
:10BCF00090E08093283490932934CF9108950E9446
:10BD00004D72D6CF0895CF9380912734882349F17F
:10BD1000A0912534B0912634ED91FC911197848146
:10BD20008823F9F0C0E0EC2FF0E0EE0FFF1F129631
:10BD30008D919C911397E80FF91F0190F081E02DF0
:10BD40000084F185E02D309709F01995CF5FA0911F
:10BD50002534B0912634ED91FC9111978481C81758
:10BD600010F3CF9108950F931F93CF93DF93EFE7D5
:10BD7000FEE3128613861486158616861786808142
:10BD800088230CF060C22091853E3091863E2115BB
:10BD9000310509F05DC24FC28F7109F097C09091D3
:10BDA000803E963081F0983009F485C091118EC0A4
:10BDB0002230310509F0FBC162E070E088E294E3D3
:10BDC0000E94EF724EC28091813E9091823E292F57
:10BDD00033272230310589F02330310579F12130C4
:10BDE000310509F0A6C18091622090916320DC01A9
:10BDF0006C9170E00E94EF724FC0E0916220F09170
:10BE000063202189821708F0D2C19927880F991FD2
:10BE1000880F991FE0916420F0916520E80FF91FC9
:10BE200080819181FC01628173810E94EF72E091B7
:10BE3000873EF091883E82E081832EC09927813031
:10BE4000910599F058F08230910509F406C20397E4
:10BE500009F078C13CE0E5E6F4E20AC064E070E095
:10BE600088EC90E20E94EF7217C0EEEBF0E239E04E
:10BE7000A2EAB0E220E0819190E08D939D932F5F44
:10BE80002317C8F3632F660F6E5F6093A02070E0E6
:10BE900080EA90E20E94EF72EFE7FEE386819781ED
:10BEA000228533858217930708F0DBC18093893E92
:10BEB00090938A3ED6C12130310509F078C161E006
:10BEC00070E087E294E30E94EF72CBC18130E9F524
:10BED0009091803E9A30C9F52130310509F037C183
:10BEE00080912734882309F432C1C091833ED091D8
:10BEF000843E0091253410912634D801ED91FC91B7
:10BF00008481C81708F023C160E08C2F1FDE8823CE
:10BF100009F418C1CE019927880F991FD8011296EC
:10BF2000ED91FC911397E80FF91F0190F081E02D3E
:10BF300086819781FC0119958093223461E070E03D
:10BF400082E294E30E94EF728CC1823009F0FAC061
:10BF50008091803E8111EFC02230310509F027C168
:10BF60008091833E0E947E7390E080932034909372
:10BF7000213462E070E080E294E30E94EF7271C1CC
:10BF80008F7109F084C09091803E933009F4D5C040
:10BF900018F49130A1F07BC0953019F0993039F147
:10BFA00076C08091853E9091863E892B09F0FFC036
:10BFB00080EA9DE580938B3E90938C3E52C18091A8
:10BFC000853E9091863E892B09F0F1C08091813E9B
:10BFD0009091823E019709F0EAC0809128349091B7
:10BFE00029348D7F80932834909329343AC18091ED
:10BFF000853E9091863E892B09F0D9C00E94EC7253
:10C00000882309F49FC02091813E3091823E3327DE
:10C01000E0916220F0916320818990E0821793077C
:10C0200008F490C045DE8091813E9091823E8093DD
:10C030002734882309F415C199278150904C880F23
:10C04000991F880F991FE0916420F0916520E80FF7
:10C05000F91FE0932534F09326340190F081E02D10
:10C060008481882309F4FDC0C0E060E08C2FEADD04
:10C07000882309F467C0CF5FE0912534F09126341E
:10C080000190F081E02D8481C81778F3EAC08130F7
:10C09000E9F49091803E9B30C9F48091853E909167
:10C0A000863E892B09F053C080912734882309F4F8
:10C0B0004EC0EFE7FEE3C481D2818C2F81DD88235F
:10C0C00009F440C06D2F8C2FBDDD3AC08230D1F510
:10C0D0008091803E813019F08330A1F030C0809192
:10C0E000853E9091863E892B09F061C08091813E0A
:10C0F0009091823E892B09F05AC08091833E0E9424
:10C1000099731EC08091853E9091863E892B09F0DF
:10C110004EC08091813E9091823E892B09F047C0AC
:10C12000CFE7DEE38C810E948C748C810E94F774CF
:10C1300007C080E005C080E003C080E001C080E06F
:10C14000811190C080917F3E8F71813081F5809107
:10C150002734882309F471C00091833E1091843EF6
:10C16000C0912534D0912634E881F9818481081763
:10C1700008F065C060E0802FE9DC8823C1F0F80199
:10C18000FF27CF01880F991FEA81FB81E80FF91F74
:10C19000C081D181EE81FF811995682F802FD6DC77
:10C1A000882329F0EC81FD81199581115BC0809174
:10C1B0007F3E8F71823009F044C0809127348823FC
:10C1C000B1F1A0912534B0912634ED91FC911197F5
:10C1D0008481882371F1C0E0EC2FF0E0EE0FFF1FA7
:10C1E00012968D919C911397E80FF91F0081118190
:10C1F000D8011696ED91FC9117971995682F8C2F01
:10C20000A5DC882379F1D8011496ED91FC9115975E
:10C210001995811127C0CF5FA0912534B0912634A4
:10C22000ED91FC9111979481C917B0F21BC080E089
:10C2300019C080E017C080E015C080E013C080E026
:10C2400011C080E00FC0982F907609F07BCF98CE78
:10C25000982F907609F076CF9FCD33E0EAEBF0E2AD
:10C2600007CE81E0DF91CF911F910F910895803823
:10C27000910558F1672B21F4873C910571F41CC09E
:10C280008F3F910509F0F8F49C01220F331FF9014B
:10C29000EE5CF84D808191810895E4E3F8E221E0BD
:10C2A00030E0419151918417950741F02F5F3F4F46
:10C2B00020383105B1F702C020E030E020583F4F70
:10C2C000C9019927089580E090E00895813691058D
:10C2D00089F0E4E5F6E240E050E04F5F5F4F2191E6
:10C2E00031912115310591F028173907B1F7892BC4
:10C2F00019F40AC040E050E0440F551FFA01EE580F
:10C30000FB4D80819181089580E090E0089543E0A5
:10C3100050E060E880E096E00F94382443E050E07D
:10C3200064E080E296E00F94382443E050E062E05D
:10C3300080E296E00F94382440E058E160E280EA21
:10C3400096E00F94382441E050E062E080EA96E005
:10C350000F94382443E050E060E180E896E00F94C9
:10C36000382443E050E060E180E496E00F94382404
:10C3700041E050E061E080E496E00F94382441E031
:10C3800050E062E080E496E00F94382441E050E011
:10C3900060E280E696E00F94382441E050E062E0ED
:10C3A00080E096E00F94382441E050E062E080E8BD
:10C3B00096E00F94382443E050E062E080E696E097
:10C3C0000F94382440E050E061E080EA96E00F945A
:10C3D000382440E050E061E080E096E00F9438249B
:10C3E00040E050E068E080E096E00F94382441E0BF
:10C3F00050E060E480E096E00F94382440E058E19B
:10C4000061E080E896E00F94382440E050E061E07D
:10C4100080E096E00F94382440E050E060E280E055
:10C4200096E00F94382440E050E064E080E096E02D
:10C430000F94382440E050E061E080EA96E00F94E9
:10C44000382443E050E060E880E496E00F9438241C
:10C4500043E050E060E280E496E00F94382440E04E
:10C4600050E060E480E496E00F94382441E050E02E
:10C4700060E880E896E00F94382441E050E060E204
:10C4800080E896E00F94382440E050E060E480E8D3
:10C4900096E00F94382443E050E068E080E496E0B2
:10C4A0000F94382440E050E064E080E496E00F947C
:10C4B000382443E050E068E080E696E00F943824AA
:10C4C00040E050E064E080E696E00F94382443E0DA
:10C4D00050E068E080E896E00F94382440E050E0B7
:10C4E00064E080E896E00F94382443E050E068E090
:10C4F00080EA96E00F94382440E050E064E080EA5F
:10C5000096E00F94382440E058E160E480EA96E039
:10C510000F94382440E058E160E180E696E00F9403
:10C52000382440E058E161E080E296E00F9438243E
:10C5300043E050E060E880E496E00F94382443E064
:10C5400050E060E280E496E00F94382440E050E050
:10C5500060E480E496E00F94382443E050E060E823
:10C5600080EA96E00D94382408951F920F920FB63A
:10C570000F9211240BB60F928F939F93EF93FF931B
:10C58000E7E7FEE380819181019680839183FF91AB
:10C59000EF919F918F910F900BBE0F900FBE0F9058
:10C5A0001F9018951F920F920FB60F9211240BB681
:10C5B0000F92CF92DF92EF92FF920F931F932F93E0
:10C5C0003F934F935F936F937F938F939F93AF931B
:10C5D000BF93EF93FF93E7E7FEE380819181228190
:10C5E000338182179307F0F121E020930204E09158
:10C5F0007D3EF0917E3E3097A9F1609108047091E4
:10C600000904A0E0B0E0DC0199278827AB0160E0D5
:10C6100070E08C019D01042B152B262B372BC901B3
:10C62000B801A7E7BEE312960D911C91139720E085
:10C6300030E09801112700271496CD90DC901597D3
:10C64000E12CF12C0C291D292E293F29061717074B
:10C650002807390730F0C901B8016F5F7F4F8F4F4E
:10C660009F4F1995FF91EF91BF91AF919F918F913E
:10C670007F916F915F914F913F912F911F910F91FA
:10C68000FF90EF90DF90CF900F900BBE0F900FBEFA
:10C690000F901F901895CF92DF92EF92FF920F9319
:10C6A0001F93CF93DF93EC016A017B01DB01CA0189
:10C6B0000197A109B109BC01CD01600F711F821F53
:10C6C000931FA70196010F94584421383105410565
:10C6D0005105F8F4213460F4213260F4213160F422
:10C6E000293060F4253060F4233060F490E80BC00A
:10C6F00093E009C092E007C092E805C091E003C052
:10C7000091E801C090E088818C77892B888381E053
:10C7100001C08FEFDF91CF911F910F91FF90EF90AC
:10C72000DF90CF9008951F920F920FB60F921124B1
:10C730000BB60F922F933F934F935F936F937F931B
:10C740008F939F93AF93BF93EF93FF93E0917034D8
:10C75000F0917134309709F01995FF91EF91BF91E5
:10C76000AF919F918F917F916F915F914F913F9189
:10C770002F910F900BBE0F900FBE0F901F9018952A
:10C780001F920F920FB60F9211240BB60F922F9398
:10C790003F934F935F936F937F938F939F93AF9349
:10C7A000BF93EF93FF93E0916E34F0916F34309725
:10C7B00009F01995FF91EF91BF91AF919F918F91E2
:10C7C0007F916F915F914F913F912F910F900BBE91
:10C7D0000F900FBE0F901F9018951F920F920FB6DB
:10C7E0000F9211240BB60F922F933F934F935F93A9
:10C7F0006F937F938F939F93AF93BF93EF93FF9329
:10C80000E0916C34F0916D34309709F01995FF91F7
:10C81000EF91BF91AF919F918F917F916F915F91B8
:10C820004F913F912F910F900BBE0F900FBE0F9025
:10C830001F9018951F920F920FB60F9211240BB6EE
:10C840000F922F933F934F935F936F937F938F93A9
:10C850009F93AF93BF93EF93FF93E0916A34F0916E
:10C860006B34309709F01995FF91EF91BF91AF911B
:10C870009F918F917F916F915F914F913F912F91F8
:10C880000F900BBE0F900FBE0F901F9018951F9228
:10C890000F920FB60F9211240BB60F922F933F9366
:10C8A0004F935F936F937F938F939F93AF93BF93B8
:10C8B000EF93FF93E0916834F0916934309709F079
:10C8C0001995FF91EF91BF91AF919F918F917F91BA
:10C8D0006F915F914F913F912F910F900BBE0F90F1
:10C8E0000FBE0F901F9018951F920F920FB60F92C8
:10C8F00011240BB60F922F933F934F935F936F9337
:10C900007F938F939F93AF93BF93EF93FF93E091A8
:10C910006634F0916734309709F01995FF91EF91E3
:10C92000BF91AF919F918F917F916F915F914F9147
:10C930003F912F910F900BBE0F900FBE0F901F9045
:10C9400018951F920F920FB60F9211240BB60F92EB
:10C950002F933F934F935F936F937F938F939F9307
:10C96000AF93BF93EF93FF93E0916434F0916534FC
:10C97000309709F01995FF91EF91BF91AF919F9179
:10C980008F917F916F915F914F913F912F910F9078
:10C990000BBE0F900FBE0F901F9018951F920F9215
:10C9A0000FB60F9211240BB60F922F933F934F9314
:10C9B0005F936F937F938F939F93AF93BF93EF9307
:10C9C000FF93E0916234F0916334309709F0199548
:10C9D000FF91EF91BF91AF919F918F917F916F9157
:10C9E0005F914F913F912F910F900BBE0F900FBE13
:10C9F0000F901F9018951F920F920FB60F9211244F
:10CA00000BB60F922F933F934F935F936F937F9348
:10CA10008F939F93AF93BF93EF93FF93E091603415
:10CA2000F0916134309709F01995FF91EF91BF9122
:10CA3000AF919F918F917F916F915F914F913F91B6
:10CA40002F910F900BBE0F900FBE0F901F90189557
:10CA50001F920F920FB60F9211240BB60F922F93C5
:10CA60003F934F935F936F937F938F939F93AF9376
:10CA7000BF93EF93FF93E0915E34F0915F34309772
:10CA800009F01995FF91EF91BF91AF919F918F910F
:10CA90007F916F915F914F913F912F910F900BBEBE
:10CAA0000F900FBE0F901F9018951F920F920FB608
:10CAB0000F9211240BB60F922F933F934F935F93D6
:10CAC0006F937F938F939F93AF93BF93EF93FF9356
:10CAD000E0915C34F0915D34309709F01995FF9145
:10CAE000EF91BF91AF919F918F917F916F915F91E6
:10CAF0004F913F912F910F900BBE0F900FBE0F9053
:10CB00001F9018951F920F920FB60F9211240BB61B
:10CB10000F922F933F934F935F936F937F938F93D6
:10CB20009F93AF93BF93EF93FF93E0915A34F091AB
:10CB30005B34309709F01995FF91EF91BF91AF9158
:10CB40009F918F917F916F915F914F913F912F9125
:10CB50000F900BBE0F900FBE0F901F9018951F9255
:10CB60000F920FB60F9211240BB60F922F933F9393
:10CB70004F935F936F937F938F939F93AF93BF93E5
:10CB8000EF93FF93E0915834F0915934309709F0C6
:10CB90001995FF91EF91BF91AF919F918F917F91E7
:10CBA0006F915F914F913F912F910F900BBE0F901E
:10CBB0000FBE0F901F9018951F920F920FB60F92F5
:10CBC00011240BB60F922F933F934F935F936F9364
:10CBD0007F938F939F93AF93BF93EF93FF93E091D6
:10CBE0005634F0915734309709F01995FF91EF9131
:10CBF000BF91AF919F918F917F916F915F914F9175
:10CC00003F912F910F900BBE0F900FBE0F901F9072
:10CC100018951F920F920FB60F9211240BB60F9218
:10CC20002F933F934F935F936F937F938F939F9334
:10CC3000AF93BF93EF93FF93E0915434F091553449
:10CC4000309709F01995FF91EF91BF91AF919F91A6
:10CC50008F917F916F915F914F913F912F910F90A5
:10CC60000BBE0F900FBE0F901F9018951F920F9242
:10CC70000FB60F9211240BB60F922F933F934F9341
:10CC80005F936F937F938F939F93AF93BF93EF9334
:10CC9000FF93E0915234F0915334309709F0199595
:10CCA000FF91EF91BF91AF919F918F917F916F9184
:10CCB0005F914F913F912F910F900BBE0F900FBE40
:10CCC0000F901F9018951F920F920FB60F9211247C
:10CCD0000BB60F922F933F934F935F936F937F9376
:10CCE0008F939F93AF93BF93EF93FF93E091503453
:10CCF000F0915134309709F01995FF91EF91BF9160
:10CD0000AF919F918F917F916F915F914F913F91E3
:10CD10002F910F900BBE0F900FBE0F901F90189584
:10CD20001F920F920FB60F9211240BB60F922F93F2
:10CD30003F934F935F936F937F938F939F93AF93A3
:10CD4000BF93EF93FF93E0914E34F0914F343097BF
:10CD500009F01995FF91EF91BF91AF919F918F913C
:10CD60007F916F915F914F913F912F910F900BBEEB
:10CD70000F900FBE0F901F9018951F920F920FB635
:10CD80000F9211240BB60F922F933F934F935F9303
:10CD90006F937F938F939F93AF93BF93EF93FF9383
:10CDA000E0914C34F0914D34309709F01995FF9192
:10CDB000EF91BF91AF919F918F917F916F915F9113
:10CDC0004F913F912F910F900BBE0F900FBE0F9080
:10CDD0001F9018951F920F920FB60F9211240BB649
:10CDE0000F922F933F934F935F936F937F938F9304
:10CDF0009F93AF93BF93EF93FF93E0914A34F091E9
:10CE00004B34309709F01995FF91EF91BF91AF9195
:10CE10009F918F917F916F915F914F913F912F9152
:10CE20000F900BBE0F900FBE0F901F9018951F9282
:10CE30000F920FB60F9211240BB60F922F933F93C0
:10CE40004F935F936F937F938F939F93AF93BF9312
:10CE5000EF93FF93E0914834F0914934309709F013
:10CE60001995FF91EF91BF91AF919F918F917F9114
:10CE70006F915F914F913F912F910F900BBE0F904B
:10CE80000FBE0F901F9018951F920F920FB60F9222
:10CE900011240BB60F922F933F934F935F936F9391
:10CEA0007F938F939F93AF93BF93EF93FF93E09103
:10CEB0004634F0914734309709F01995FF91EF917E
:10CEC000BF91AF919F918F917F916F915F914F91A2
:10CED0003F912F910F900BBE0F900FBE0F901F90A0
:10CEE00018951F920F920FB60F9211240BB60F9246
:10CEF0002F933F934F935F936F937F938F939F9362
:10CF0000AF93BF93EF93FF93E0914434F091453496
:10CF1000309709F01995FF91EF91BF91AF919F91D3
:10CF20008F917F916F915F914F913F912F910F90D2
:10CF30000BBE0F900FBE0F901F9018951F920F926F
:10CF40000FB60F9211240BB60F922F933F934F936E
:10CF50005F936F937F938F939F93AF93BF93EF9361
:10CF6000FF93E0914234F0914334309709F01995E2
:10CF7000FF91EF91BF91AF919F918F917F916F91B1
:10CF80005F914F913F912F910F900BBE0F900FBE6D
:10CF90000F901F9018951F920F920FB60F921124A9
:10CFA0000BB60F922F933F934F935F936F937F93A3
:10CFB0008F939F93AF93BF93EF93FF93E091403490
:10CFC000F0914134309709F01995FF91EF91BF919D
:10CFD000AF919F918F917F916F915F914F913F9111
:10CFE0002F910F900BBE0F900FBE0F901F901895B2
:10CFF0001F920F920FB60F9211240BB60F922F9320
:10D000003F934F935F936F937F938F939F93AF93D0
:10D01000BF93EF93FF93E0913E34F0913F3430970C
:10D0200009F01995FF91EF91BF91AF919F918F9169
:10D030007F916F915F914F913F912F910F900BBE18
:10D040000F900FBE0F901F9018951F920F920FB662
:10D050000F9211240BB60F922F933F934F935F9330
:10D060006F937F938F939F93AF93BF93EF93FF93B0
:10D07000E0913C34F0913D34309709F01995FF91DF
:10D08000EF91BF91AF919F918F917F916F915F9140
:10D090004F913F912F910F900BBE0F900FBE0F90AD
:10D0A0001F9018951F920F920FB60F9211240BB676
:10D0B0000F922F933F934F935F936F937F938F9331
:10D0C0009F93AF93BF93EF93FF93E0913A34F09126
:10D0D0003B34309709F01995FF91EF91BF91AF91D3
:10D0E0009F918F917F916F915F914F913F912F9180
:10D0F0000F900BBE0F900FBE0F901F9018951F92B0
:10D100000F920FB60F9211240BB60F922F933F93ED
:10D110004F935F936F937F938F939F93AF93BF933F
:10D12000EF93FF93E0913834F0913934309709F060
:10D130001995FF91EF91BF91AF919F918F917F9141
:10D140006F915F914F913F912F910F900BBE0F9078
:10D150000FBE0F901F9018951F920F920FB60F924F
:10D1600011240BB60F922F933F934F935F936F93BE
:10D170007F938F939F93AF93BF93EF93FF93E09130
:10D180003634F0913734309709F01995FF91EF91CB
:10D19000BF91AF919F918F917F916F915F914F91CF
:10D1A0003F912F910F900BBE0F900FBE0F901F90CD
:10D1B00018951F920F920FB60F9211240BB60F9273
:10D1C0002F933F934F935F936F937F938F939F938F
:10D1D000AF93BF93EF93FF93E0913434F0913534E4
:10D1E000309709F01995FF91EF91BF91AF919F9101
:10D1F0008F917F916F915F914F913F912F910F9000
:10D200000BBE0F900FBE0F901F9018951F920F929C
:10D210000FB60F9211240BB60F922F933F934F939B
:10D220005F936F937F938F939F93AF93BF93EF938E
:10D23000FF93E0913234F0913334309709F019952F
:10D24000FF91EF91BF91AF919F918F917F916F91DE
:10D250005F914F913F912F910F900BBE0F900FBE9A
:10D260000F901F9018951F920F920FB60F921124D6
:10D270000BB60F922F933F934F935F936F937F93D0
:10D280008F939F93AF93BF93EF93FF93E0913034CD
:10D29000F0913134309709F01995FF91EF91BF91DA
:10D2A000AF919F918F917F916F915F914F913F913E
:10D2B0002F910F900BBE0F900FBE0F901F901895DF
:10D2C0001F920F920FB60F9211240BB60F922F934D
:10D2D0003F934F935F936F937F938F939F93AF93FE
:10D2E000BF93EF93FF93E0912E34F0912F3430975A
:10D2F00009F01995FF91EF91BF91AF919F918F9197
:10D300007F916F915F914F913F912F910F900BBE45
:10D310000F900FBE0F901F9018951F920F920FB68F
:10D320000F9211240BB60F922F933F934F935F935D
:10D330006F937F938F939F93AF93BF93EF93FF93DD
:10D34000E0912C34F0912D34309709F01995FF912C
:10D35000EF91BF91AF919F918F917F916F915F916D
:10D360004F913F912F910F900BBE0F900FBE0F90DA
:10D370001F9018951F920F920FB60F9211240BB6A3
:10D380000F922F933F934F935F936F937F938F935E
:10D390009F93AF93BF93EF93FF93E0912A34F09163
:10D3A0002B34309709F01995FF91EF91BF91AF9110
:10D3B0009F918F917F916F915F914F913F912F91AD
:10D3C0000F900BBE0F900FBE0F901F901895CF932C
:10D3D000CFB7F894282F392F211588E0380749F462
:10D3E00061E083E00F94E02364E083E00F94E023A6
:10D3F0004FC0203488E0380749F462E083E00F949E
:10D40000E02364E083E00F94E02342C0211589E02B
:10D41000380749F461E084E00F94E02364E084E09D
:10D420000F94E02335C0203489E0380749F462E0E6
:10D4300084E00F94E02364E084E00F94E02328C0AC
:10D4400021158AE0380749F461E085E00F94E02374
:10D4500064E085E00F94E0231BC020348AE03807A5
:10D4600049F462E085E00F94E02364E085E00F94E6
:10D47000E0230EC021153B4049F461E086E00F94A3
:10D48000E02364E086E00F94E02302C0CFBF01C038
:10D49000CFBFCF910895CF93CFB7F894282F392FCE
:10D4A000211588E0380749F461E083E00F94EC230C
:10D4B00064E083E00F94EC234FC0203488E0380709
:10D4C00049F462E083E00F94EC2364E083E00F947E
:10D4D000EC2342C0211589E0380749F461E084E07B
:10D4E0000F94EC2364E084E00F94EC2335C02034E7
:10D4F00089E0380749F462E084E00F94EC2364E0AB
:10D5000084E00F94EC2328C021158AE0380749F401
:10D5100061E085E00F94EC2364E085E00F94EC2358
:10D520001BC020348AE0380749F462E085E00F949C
:10D53000EC2364E085E00F94EC230EC021153B4002
:10D5400049F461E086E00F94EC2364E086E00F94F8
:10D55000EC2302C0CFBF01C0CFBFCF91089581158A
:10D5600028E0920729F46093703470937134089521
:10D57000803428E0920729F4609364347093653412
:10D580000895811529E0920729F460935C34709323
:10D590005D340895803429E0920729F46093503473
:10D5A00070935134089581152AE0920729F460930D
:10D5B000483470934934089580342AE0920729F45E
:10D5C00060933C3470933D34089581159B4021F461
:10D5D00060933434709335340895FC01918195FF44
:10D5E000FDCF608380E090E008954F925F926F924C
:10D5F0007F928F929F92AF92BF92EF92FF920F9382
:10D600001F93CF937C014A015B0128013901FC0182
:10D61000848182FF16C0D901C801689412F8B695BA
:10D62000A795979587951694D1F7B901A801032E70
:10D6300036E176956795579547953A95D1F7302D10
:10D6400015C0D901C801689413F8B695A7959795A8
:10D6500087951694D1F7B901A801032E37E1769585
:10D660006795579547953A95D1F7302D88159905C7
:10D67000AA05BB0508F4A6C084169506A606B7063B
:10D6800008F4A2C0F701848182FD04C0880C991CB3
:10D69000AA1CBB1CC301B201A50194010F945844FC
:10D6A0002F3F31054105510508F490C08FEF90E000
:10D6B000A0E0B0E0C9EF05C0281739074A075B07AB
:10D6C00058F0880F991FAA1FBB1FCD3F0CF4816033
:10D6D000CF5FC73089F74FC0CC230CF04CC0D501C9
:10D6E000C401880F991FAA1FBB1F880F991FAA1F6B
:10D6F000BB1F880F991FAA1FBB1F481A590A6A0A25
:10D700007B0ACE3FF4F48DEF9FEF8C1B9109C7FD90
:10D71000939504C0440C551C661C771C8A95D2F75F
:10D72000D501C401B695A79597958795BC01CD0104
:10D73000640D751D861D971DA50194010F94584415
:10D7400037C083E08C0FA501940104C0220F331F62
:10D75000441F551F8A95D2F7DA01C901B695A795DE
:10D7600097958795BC01CD01640D751D861D971D8C
:10D770000F9458441DC083E08C0FA501940104C090
:10D78000220F331F441F551F8A95D2F7DA01C901B2
:10D79000B695A79597958795BC01CD01640D751D2C
:10D7A000861D971D0F945844215031094109510994
:10D7B000832F8F70C295C07FC82BF701C783268344
:10D7C00081E018C080E016C080E014C0D501C4011B
:10D7D000880F991FAA1FBB1F880F991FAA1FBB1F65
:10D7E000880F991FAA1FBB1F481A590A6A0A7B0A89
:10D7F000C9EF89CFCF911F910F91FF90EF90BF900C
:10D80000AF909F908F907F906F905F904F90089512
:10D810000F931F93CF93DF93EC018B01009709F4D3
:10D820001EC1803C910529F460E180E00F94E02363
:10D8300016C1C11584E0D80729F464E080E00F9494
:10D84000E0230DC1C038E1E0DE0729F462E080E0AA
:10D850000F94E02304C1C115F1E0DF0729F461E072
:10D8600080E00F94E023FBC0C03883E0D80729F4A0
:10D8700061E081E00F94E023F2C0C039E3E0DE070D
:10D8800029F461E082E00F94E023E9C0C115F2E0E1
:10D89000DF0729F462E081E00F94E023E0C0C034A8
:10D8A00082E0D80729F462E082E00F94E023D7C039
:10D8B000C032E3E0DE0729F464E082E00F94E02365
:10D8C000CEC0C115F8E0DF0729F461E083E00F94D2
:10D8D000E023C5C0C11589E0D80729F461E084E0E0
:10D8E0000F94E023BCC0C115EAE0DE0729F461E033
:10D8F00085E00F94E023B3C0C115FBE0DF0729F4F6
:10D9000061E086E00F94E023AAC0C03488E0D80725
:10D9100029F462E083E00F94E023A1C0C034E9E081
:10D92000DE0729F462E084E00F94E02398C0C0345D
:10D93000FAE0DF0729F462E085E00F94E0238FC06E
:10D94000C03988E0D80729F464E083E00F94E0232D
:10D9500086C0C039E9E0DE0729F464E084E00F9472
:10D96000E0237DC0C039FAE0DF0729F464E085E0F8
:10D970000F94E02374C0C0398BE0D80729F464E029
:10D9800086E00F94E0236BC0C03CE8E0DE0729F49A
:10D9900068E083E00F94E02362C0C03CF9E0DF0759
:10D9A00029F468E084E00F94E02359C0C03C8AE089
:10D9B000D80729F468E085E00F94E02350C0C03A0E
:10D9C000E8E0DE0729F460E183E00F94E02347C03C
:10D9D000C03AF9E0DF0729F460E184E00F94E02326
:10D9E0003EC0C03A8AE0D80729F460E185E00F9490
:10D9F000E02335C0C03AEBE0DE0729F460E186E0C1
:10DA00000F94E0232CC0C03BF8E0DF0729F460E26C
:10DA100083E00F94E02323C0C03B89E0D80729F4BA
:10DA200060E284E00F94E0231AC0C03BEAE0DE0726
:10DA300029F460E285E00F94E02311C0C038F4E0DF
:10DA4000DF0729F460E483E00F94E02308C0C03AC4
:10DA500084E0D80721F460E485E00F94E0238D8111
:10DA60008F738D83F80195818481892B9681911123
:10DA700098E0892B8D83F801408151816281738107
:10DA800000E010E62AEE30E0CE01AFDD9C81986028
:10DA90009C839C8190619C83DF91CF911F910F911A
:10DAA0000895CF92DF92EF92FF920F931F93CF933F
:10DAB000DF93EC01D901C801B695A7959795879595
:10DAC000481759076A077B0778F46A017B01CC0C79
:10DAD000DD1CEE1CFF1CC901B801A70196010F94C3
:10DAE00058442150310902C020E030E0832F8F706C
:10DAF0008F832E83DF91CF911F910F91FF90EF9035
:10DB0000DF90CF900895EF92FF920F931F93CF93E2
:10DB1000DF93EC017B01009709F4B9C1803C9105CA
:10DB200029F460E180E00F94E023B1C181159440B5
:10DB300029F464E080E00F94E023A9C1C03881E0BB
:10DB4000D80729F462E080E00F94E023A0C1C1155A
:10DB5000E1E0DE0729F461E080E00F94E02397C163
:10DB6000C038F3E0DF0729F461E081E00F94E0239F
:10DB70008EC1C03933E0D30729F461E082E00F940D
:10DB8000E02385C1C11582E0D80729F462E081E075
:10DB90000F94E0237CC1C034E2E0DE0729F462E0A8
:10DBA00082E00F94E02373C1C032F3E0DF0729F471
:10DBB00064E082E00F94E0236AC1C11538E0D30726
:10DBC00029F461E083E00F94E02361C1C11589E08D
:10DBD000D80729F461E084E00F94E02358C1C1150F
:10DBE000EAE0DE0729F461E085E00F94E0234FC10D
:10DBF000C115FBE0DF0729F461E086E00F94E02324
:10DC000046C1C03438E0D30729F462E083E00F94C2
:10DC1000E0233DC1C03489E0D80729F462E084E004
:10DC20000F94E02334C1C034EAE0DE0729F462E057
:10DC300085E00F94E0232BC1C039F8E0DF0729F419
:10DC400064E083E00F94E02322C1C03939E0D307B8
:10DC500029F464E084E00F94E02319C1C0398AE01C
:10DC6000D80729F464E085E00F94E02310C1C0399F
:10DC7000EBE0DE0729F464E086E00F94E02307C1BF
:10DC8000C03CF8E0DF0729F468E083E00F94E0236C
:10DC9000FEC0C03C39E0D30729F468E084E00F946B
:10DCA000E023F5C0C03C8AE0D80729F468E085E0AD
:10DCB0000F94E023ECC0C03AE8E0DE0769F460E1CD
:10DCC00083E00F94E023E0EAF8E084818F7E848390
:10DCD000F7012481225053C0C03AF9E0DF0729F44C
:10DCE00060E184E00F94E023D2C0C03A3AE0D30769
:10DCF00029F460E185E00F94E023C9C0C03A8BE0CD
:10DD0000D80729F460E186E00F94E023C0C0C03B4F
:10DD1000E8E0DE0729F460E283E00F94E023B7C077
:10DD2000C03BF9E0DF0729F460E284E00F94E023D0
:10DD3000AEC0C03B3AE0D30729F460E285E00F941F
:10DD4000E023A5C0C03884E0D80729F460E483E06C
:10DD50000F94E0239CC0C03AE4E0DE0729F460E4BD
:10DD600085E00F94E02393C08C818F7E8C83FB0130
:10DD700024812250CE01C03AF8E0DF0731F48091CF
:10DD80004E0684FD8CC011E18BC0803B38E09307C8
:10DD900079F0803AE9E09E0731F430916E0634FD67
:10DDA00082C019E110C0803BF9E09F0789F001C0F3
:10DDB00015E1803A3AE0930731F480918E0684FDB4
:10DDC00074C011E212C0803BEAE09E0759F001C026
:10DDD0001DE1803A9B4049F48091AE0684FD04C069
:10DDE00019E203C015E201C01DE2E12FE695E695B8
:10DDF000E69530E2E39FF0011124FA5F177081E0AD
:10DE000090E0012E02C0880F991F0A94E2F78183E7
:10DE1000223010F040E001C040E4DF015096A10F35
:10DE2000B11D3FB7F8942C9127702C939C91942BA3
:10DE30009C933FBF85838D81806C8D83F7018481A6
:10DE40008D7F813021F48D8182608D8303C08D812F
:10DE50008D7F8D83F7018581882321F08D818460FA
:10DE60008D8303C08D818B7F8D83F701408151812C
:10DE70006281738100E010E62AEE30E0CE0111DE0F
:10DE80008C8188608C838C8180618C8310C08C81B4
:10DE90008F7E8C83F70124812250CE0176CF15E14D
:10DEA00080EA98E080CF1DE18ECF15E29ECFDF9112
:10DEB000CF911F910F91FF90EF9008950F93E8EC91
:10DEC000F4E080818F7D808380818F7D8083E0E797
:10DED000F5E302E00593109272351092733500E27B
:10DEE000069300E40693E8E6F5E300E2069300E417
:10DEF0000693EFE7FEE314861586168617861286CC
:10DF0000138610925B350F9108950F9385E08093EF
:10DF10005B35E1E7F5E304E00593E9E6F5E304E0CA
:10DF200005930F9108950F9383E080935B351092D2
:10DF3000723510927335E0E7F5E302E006930F9136
:10DF40000895E0918B3EF0918C3E309709F0199541
:10DF500008950F93CF93DF9380915B35833019F44D
:10DF6000F0DFACDF5EC08091573590915835C0919D
:10DF7000893ED0918A3EC81BD90B71F52091593545
:10DF800030915A35820F931F8093593590935A35AB
:10DF90002091853E3091863E8217930721F0809133
:10DFA0007234882341F084E080935B35E8E6F5E342
:10DFB00002E0069336C0E0918D3EF0918E3E3097A0
:10DFC00099F01995882381F01092573510925835A1
:10DFD000C091893ED0918A3EC034D10528F010927C
:10DFE0007234C0E4D0E003C081E080937234ECE589
:10DFF000F5E3C68BD78B809157359091583520919A
:10E00000873E3091883E280F391F208F318FC80FEF
:10E01000D91FC0935735D0935835E0E7F5E302E0B8
:10E020000693DF91CF910F910895FC018181E82F34
:10E03000E7708E2F90E0FC013197E730F105D8F4BE
:10E040008827ED55FE4F8F4F0D94964480E190E068
:10E05000089580E290E0089580E490E0089580E8DB
:10E0600090E0089580E091E0089580E092E00895C6
:10E070008FEF93E0089588E090E00895282F2F70A7
:10E0800030E0220F331F082E000C990B8827990FC0
:10E09000881F9927820F931F02979C01220F331F1D
:10E0A000220F331F220F331F820F931F8D509B4C63
:10E0B00008950F93CF938091CC0480FF63C081E0DB
:10E0C0008093CC04E8E6F5E300E80693E0E7F5E3A7
:10E0D00000E806938093CA04E8E6F5E300E10693BE
:10E0E00080915B35882329F08350823008F429DF42
:10E0F000E5DE80916A3590916B35089709F044C050
:10E1000088E0E7E1F5E3AFE7BEE301900D928A9581
:10E11000E1F7E8ECF4E080818062808380818062B6
:10E1200080830E94B35EC82F811103C0EEDEC1E080
:10E130002CC080917F3E88236CF410925935109248
:10E140005A35109257351092583582E080935B35DE
:10E1500000DF1BC08091853E9091863E892B11F493
:10E16000E2DE13C01092593510925A35109257358D
:10E170001092583581E080935B35E8E6F5E302E0E4
:10E18000069303C0C0E001C0C1E08C2FCF910F9176
:10E1900008958F929F92AF92BF92DF92EF92FF927B
:10E1A0000F931F93CF93DF93D82E68DF8C01CD2D73
:10E1B000CF70D0E0CE01880F991FCD2D0D2C000C13
:10E1C000DD0BCC27DD0FCC1FDD27C80FD91FCE01FB
:10E1D000880F991F880F991F880F991F9C01285934
:10E1E0003A4C7901C90121DF4C01DD200CF07BC0E4
:10E1F000FE01EE0FFF1FEE0FFF1FEE0FFF1FE45A91
:10E20000FA4C22893389D80115968D919C911697E5
:10E21000820F931F15968D939C93169713962D91AD
:10E220003C9114978217930709F447C0281B390BB8
:10E230002115B4E03B0740F02FEF33E0C901B401F2
:10E240000F943144281B390BF801808181FF0AC0EB
:10E25000C901B4010F94314441E0892B09F040E039
:10E26000842F01C080E0D8019C9180FB91F99C93A0
:10E27000FE01EE0FFF1FEE0FFF1FEE0FFF1FE45A10
:10E28000FA4C128A138A2687378711962D913C9172
:10E29000129715968D919C911697820F931FCC0F14
:10E2A000DD1FCC0FDD1FCC0FDD1FC459DA4C888376
:10E2B0009983F70102E00693E4C0D8018C9181FFB5
:10E2C000CDC08D7F8C93CC0FDD1FCC0FDD1FCC0F0D
:10E2D000DD1FC45ADA4C1A8A1B8A1E861F86F70174
:10E2E00002E00693CEC0FE01EE0FFF1FEE0FFF1FF0
:10E2F000EE0FFF1FE45AFA4CA684B784D8018C9124
:10E3000082FF1BC01196ED91FC91129715962D91ED
:10E310003C91169713968D919C911497B4010F948C
:10E320003144B0E4DB9EB00111246D5C7B4CAC0148
:10E33000CF01820F931F0F949546F80125813681F6
:10E340002A0D3B1D25833683838194818217930791
:10E3500068F485839683CC0FDD1FCC0FDD1FCC0FB7
:10E36000DD1FC45ADA4C8A899B8978C0FE01EE0F02
:10E37000FF1FEE0FFF1FEE0FFF1FE45AFA4C4289FA
:10E380005389A416B50609F069C02817390709F49E
:10E3900065C0AC01421B530B9A01211554E03507AF
:10E3A00048F02FEF33E0C901B4010F943144281B2A
:10E3B000390B06C0C901B4010F943144281B390B35
:10E3C000FE01EE0FFF1FEE0FFF1FEE0FFF1FE45ABF
:10E3D000FA4C168617862815390500F5D8018C9158
:10E3E00084608C93B0E4DB9EC00111248D5C9B4C57
:10E3F000FE01EE0FFF1FEE0FFF1FEE0FFF1FE45990
:10E40000FA4C80839183CC0FDD1FCC0FDD1FCC0F26
:10E41000DD1FC45ADA4C8A8A9B8A1CC0F8014181EC
:10E42000528185819681840F951FFE01EE0FFF1F9B
:10E43000EE0FFF1FEE0FFF1FE459FA4C808391830C
:10E44000CC0FDD1FCC0FDD1FCC0FDD1FC45ADA4C03
:10E450002A8B3B8BF70102E0069313C0D8018C9105
:10E4600080FF0FC08E7F8C931796ED91FC911897CB
:10E47000309739F015966D917C9116974D2D80E06F
:10E480001995DF91CF911F910F91FF90EF90DF9041
:10E49000BF90AF909F908F900895CF93CFB7F8948F
:10E4A000E1ECF4E080818E7F80831092C0041082C2
:10E4B0000F942F2410929C35CFBFCF9108959FB712
:10E4C000F89481E080939C35EAECF4E080E480836A
:10E4D00080E28083E1ECF4E0808181608083A9ECBC
:10E4E000B4E08C9182608C93E8ECF4E080818064ED
:10E4F00080838C9181608C938081806880839FBFB2
:10E500000895CF93DF93C0E6D0E0188280E30F94A4
:10E51000F723E0ECF4E080818064808381E08883ED
:10E52000CFB7F894ECE5F5E31586158A158E15A29C
:10E5300015A615AAE3EFF4E380818E7F8083ECEFCC
:10E54000F4E380818E7F8083E5E0F5E380818E7F38
:10E550008083EEE0F5E380818E7F80836AE170E066
:10E5600082E00F94F1418F3F19F08093FA0403C0C9
:10E570008FE18093FA046BE170E082E00F94F14147
:10E580008F3F19F08093FB0403C08FE18093FB045D
:10E59000E0ECF4E080818260808380818068808309
:10E5A00080818061808388E695E38683978380817C
:10E5B000806280838FEF8093C504E8ECF4E0808173
:10E5C0008160808310929C357ADFCFBFDF91CF913D
:10E5D00008958093C30408958091C3040895EFE7DC
:10E5E000FEE380879187628773870895282F2F70B5
:10E5F00030E0220F331F082E000C990B8827990F4B
:10E60000881F9927820F931FFC01EE0FFF1FEE0F4B
:10E61000FF1FEE0FFF1FE45AFA4C2585207C09F0FE
:10E6200069C06370613011F018F404C060EC03C07D
:10E6300060E801C060E440385105E9F050F4403230
:10E640005105A9F040345105A1F040315105D9F4EC
:10E650000CC0411522E0520791F04F3F23E05207D2
:10E6600081F04115514079F408C021E00DC022E04D
:10E670000BC023E009C024E007C025E005C026E068
:10E6800003C027E001C020E0FC01EE0FFF1FEE0FEA
:10E69000FF1FEE0FFF1FE45AFA4C158636E0348751
:10E6A000262B2587FC01EE0FFF1FEE0FFF1FEE0F3D
:10E6B000FF1FE45AFA4C2585207C203C69F4FC01BC
:10E6C000EE0FFF1FEE0FFF1FEE0FFF1FE45AFA4C75
:10E6D00025852770273081F0880F991F880F991F93
:10E6E000880F991FFC01E45AFA4C85858062858762
:10E6F00081E0089580E0089581E00895E82FEF70AB
:10E70000F0E0EE0FFF1F082E000C990B8827990FE1
:10E71000881F9927E80FF91FEE0FFF1FEE0FFF1F4D
:10E72000EE0FFF1FE45AFA4C858582FB882780F99B
:10E730000895282F2F7030E0A901440F551F282F6E
:10E74000082E000C330B2227330F221F3327240FF0
:10E75000351FF901EE0FFF1FEE0FFF1FEE0FFF1F1A
:10E76000E45AFA4C958592FF17C0220F331F220FEF
:10E77000331F220F331FF901E45AFA4C95859B7F12
:10E7800095877CDCFC01808180FF06C08E7F8083C2
:10E790000780F085E02D199581E008958F929F9272
:10E7A000AF92BF92CF92DF92EF92FF920F931F939F
:10E7B000CF93DF93982E862E6A0179015FDC5C018E
:10E7C000292DC92DCF70D0E0CE01880F991FC92DFA
:10E7D000092C000CDD0BCC27DD0FCC1FDD27C80F6B
:10E7E000D91FFE01EE0FFF1FEE0FFF1FEE0FFF1FE1
:10E7F000E45AFA4C8585807C09F47EC0FE01EE0F58
:10E80000FF1FEE0FFF1FEE0FFF1FE45AFA4C858526
:10E81000807C803C61F0FE01EE0FFF1FEE0FFF1FBA
:10E82000EE0FFF1FE45AFA4C858582FD67C08FB753
:10E83000F894F501908190FF03C08FBF80E05FC026
:10E84000F5019081916090838FBFC182D282E38273
:10E85000F4821582168207831087811006C091E02A
:10E86000E114F10419F090E001C091E0F50180811C
:10E8700090FB81F98B7F808322235CF4CC0FDD1F1A
:10E88000CC0FDD1FCC0FDD1FC45ADA4C1A8A1B8A4D
:10E890002FC0FE01EE0FFF1FEE0FFF1FEE0FFF1F39
:10E8A000E45AFA4C8585807C803CB1F4CE01880F17
:10E8B000991F880F991F880F991F88599A4CB5DBAB
:10E8C000BC01C7010F943144892B31F0F5018081DF
:10E8D0008E7F808380E013C0CC0FDD1FCC0FDD1F47
:10E8E000CC0FDD1FC45ADA4C1E861F861A8A1B8A7B
:10E8F000892D4FDC81E003C080E001C080E0DF9122
:10E90000CF911F910F91FF90EF90DF90CF90BF902C
:10E91000AF909F908F900895FF920F931F93CF9386
:10E92000DF93182FC82FCF70D0E0CE01880F991F2A
:10E93000C12F012E000CDD0BCC27DD0FCC1FDD27F6
:10E94000C80FD91F812F9ADBDC01FE01EE0FFF1FDC
:10E95000EE0FFF1FEE0FFF1FE859FA4C02E0059380
:10E960008C9180FF22C08E7F8C931796ED91FC9145
:10E9700018973097D1F011235CF4CC0FDD1FCC0F2A
:10E98000DD1FCC0FDD1FC45ADA4C6A897B890AC0AF
:10E99000CC0FDD1FCC0FDD1FCC0FDD1FC45ADA4CAE
:10E9A0006E857F85412F81E01995DF91CF911F9171
:10E9B0000F91FF900895CF93C82FAEDFEC2FEF702B
:10E9C000F0E0EE0FFF1F8C2FCC0F990B8827990FCB
:10E9D000881F9927E80FF91FEE0FFF1FEE0FFF1F8B
:10E9E000EE0FFF1FE45AFA4C1586CF9108950F934E
:10E9F000E82FEF70F0E0EE0FFF1F282F082E000C1D
:10EA0000330B2227330F221F3327E20FF31FEE0FA2
:10EA1000FF1FEE0FFF1FEE0FFF1FDF01A45ABA4CBE
:10EA20001D969C911D9794601D969C93E859FA4CF5
:10EA300001E0069371DF81E00F9108950F931F931A
:10EA4000CF93DF938B01C82FCF70D0E0CC0FDD1FA9
:10EA5000282F082E000C330B2227330F221F3327B9
:10EA6000C20FD31F0BDBCC0FDD1FCC0FDD1FCC0F74
:10EA7000DD1FC45ADA4C2D8522FF0AC0FC0120811B
:10EA800020FD0AC0216020830783108781E005C034
:10EA9000F801199581E001C080E0DF91CF911F91CD
:10EAA0000F9108951F920F920FB60F9211240BB67B
:10EAB0000F920F932F933F934F935F936F937F9397
:10EAC0008F939F93AF93BF93EF93FF938091CB046A
:10EAD000882344F480E88093CA040E94835E0E94E5
:10EAE000B95587C08091CB0482FF20C084E0809319
:10EAF000CA048091703586FF7CC08091CC0481FD72
:10EB000078C0D7DA811175C080915B35813011F4FE
:10EB10000ADA6FC0843009F06CC0E1E7F5E304E085
:10EB20000593E9E6F5E304E0059363C08091CB0427
:10EB300081FF5AC082E08093CA048091683586FFC5
:10EB400058C08091CC0481FD54C0B3DA811151C00A
:10EB500080915B35823041F484E080935B35E8E658
:10EB6000F5E302E0069345C0833009F042C0E1E7D7
:10EB7000F5E304E00593E9E6F5E304E0059339C025
:10EB800080E18093CA0481E0C7DE81E8C5DE0E948F
:10EB9000585E1092C304ECE5F5E3158696E0948781
:10EBA00083E48587158A948B858B87E195E3808B39
:10EBB000918B84D91EC08091CB0486FF08C080E46D
:10EBC0008093CA0410929C350E94BC5512C080915B
:10EBD000CB0485FF0EC080E28093CA0481E080935D
:10EBE0009C350E94BD5505C08091CB0484FFE3CFC6
:10EBF000C7CFFF91EF91BF91AF919F918F917F917F
:10EC00006F915F914F913F912F910F910F900BBE9C
:10EC10000F900FBE0F901F9018951F920F920FB676
:10EC20000F9211240BB60F920F931F932F933F93C4
:10EC30004F935F936F937F938F939F93AF93BF9304
:10EC4000CF93DF93EF93FF938091CC0481FD03C0BA
:10EC500030DA8111C2C082E08093CC048091C50477
:10EC60008195880FE8E6F5E3E81BF1092081318101
:10EC70002856354336952795369527953695279509
:10EC8000822F869520FD02C090E001C090E8890F98
:10EC9000E82FEF70F0E0EE0FFF1F282F082E000C7A
:10ECA000330B2227330F221F3327E20FF31FDF011D
:10ECB000AA0FBB1FAA0FBB1FAA0FBB1FA45ABA4C97
:10ECC0001C969C9195FF89C0EE0FFF1FEE0FFF1F52
:10ECD000EE0FFF1FE859FA4C00E20693811178C04D
:10ECE00080915B35843019F42CD9E8D876C0009136
:10ECF0006A3510916B358091893E90918A3EC09122
:10ED00005735D091583598012C0F3D1F8217930726
:10ED100018F48C010C1B1D0B8091873E9091883E4E
:10ED2000A80167E175E38C0F9D1F0F949546C00FF6
:10ED3000D11FC0935735D09358350034110569F46D
:10ED40008091593590915A358C0F9D1F2091853EA9
:10ED50003091863E8217930780F0EFE7FEE3C2878B
:10ED6000D3870684F785E02D309729F01995811116
:10ED700002C0CBD832C0D7D830C08091893E9091A4
:10ED80008A3EC817D907F9F4E0918D3EF0918E3E86
:10ED9000309711F4BAD821C01995811102C0B5D8A5
:10EDA0001CC02091593530915A358091573590913A
:10EDB0005835820F931F8093593590935A3510928E
:10EDC000573510925835E8E6F5E302E0069305C0A2
:10EDD000803811F4BED801C0DCD9FF91EF91DF91EA
:10EDE000CF91BF91AF919F918F917F916F915F91E3
:10EDF0004F913F912F911F910F910F900BBE0F904C
:10EE00000FBE0F901F9018959091800024E0829F74
:10EE1000B00111246C7392709160692B80E890E0CE
:10EE20000F949241E0E8F0E0828180FDFDCF0895EB
:10EE3000609180006C73636080E890E00F94924171
:10EE4000E0E8F0E0828180FDFDCF0895CF92DF926F
:10EE5000EF92FF92CF93DF93EC016B01E12CF12C49
:10EE600060E070E68AEE90E0A70196010F945844A6
:10EE7000CA01B9012FEF3FEF40E050E00F94584432
:10EE80002115310529F481E08C8321E030E02DC08B
:10EE90002230310528F482E08C8322E030E025C066
:10EEA0002430310528F483E08C8324E030E01DC059
:10EEB0002830310528F484E08C8328E030E015C048
:10EEC0002034310528F485E08C8320E430E00DC047
:10EED0002F3F310509F028F486E08C8320E031E0F3
:10EEE00004C087E08C8320E034E040E050E060E044
:10EEF00070E68AEE90E00F945844CA01B901A70168
:10EF000096010F9458442D833E832436310518F41E
:10EF10001C821D821E82DF91CF91FF90EF90DF90C7
:10EF2000CF9008950F931F93CF93DF93EC01890146
:10EF3000862F90E08730910508F08BC0FC01882770
:10EF4000E655FE4F8F4F0D94964480E098E08883FD
:10EF50009983E0E4F6E0308181E090E02FEF240F28
:10EF600002C0880F991F2A95E2F7832B808371C016
:10EF700080E498E088839983E0E4F6E0308181E0E2
:10EF800090E023E0240F02C0880F991F2A95E2F732
:10EF9000832B80835EC080E099E088839983E0E6DC
:10EFA000F6E0308181E090E02FEF240F02C0880F5F
:10EFB000991F2A95E2F7832B80834BC080E499E068
:10EFC00088839983E0E6F6E0308181E090E023E0F9
:10EFD000240F02C0880F991F2A95E2F7832B8083A4
:10EFE00038C080E09AE088839983E0E8F6E03081D9
:10EFF00081E090E02FEF240F02C0880F991F2A951F
:10F00000E2F7832B808325C080E49AE0888399838C
:10F01000E0E8F6E0308181E090E023E0240F02C0D8
:10F02000880F991F2A95E2F7832B808312C080E016
:10F030009BE088839983E0EAF6E0308181E090E00C
:10F040002FEF240F02C0880F991F2A95E2F7832B18
:10F0500080834A83423061F018F4413031F010C0AF
:10F06000433049F0443051F00BC080E18B8308C03D
:10F0700080E28B8305C080E48B8302C080E88B83B1
:10F08000888199810E94E769E881F9818181887F7F
:10F09000836081831D821E821C82E881F9818081C8
:10F0A000807F8083B801CE01D1DEDF91CF911F91A7
:10F0B0000F910895CF93DF93EC012D813E81A62F10
:10F0C000B0E00F949E4424E630E040E050E00F941E
:10F0D00058448A81E881F981E6FD17C0823061F0E9
:10F0E00018F4813031F01BC0833049F0843051F086
:10F0F00016C020AF31AF13C022AF33AF10C024AF62
:10F1000035AF0DC026AF37AF0AC0813019F082305D
:10F1100021F005C020AF31AF02C022AF33AF8D81E7
:10F120009E81E881F98186A397A38B81E881F9818B
:10F13000E6FD04C09181892B818304C09181807395
:10F14000892B8183E881F9818081807F9C81892B53
:10F150008083DF91CF910895CF93DF93EC01411528
:10F16000510509F443C0ACEEB0E420E030E0922F4A
:10F17000F901E25CFC4EE491ED932F5F3F4F2730A5
:10F180003105A9F7FA01DE01CCEED0E480818B8352
:10F1900081818C83F901E451FF4B8CE28083E2E0B2
:10F1A000E90FF0E0E451FF4B6083C4E0C90F9D5FBD
:10F1B000E92FF0E0E451FF4B8DE78083D0E0FE01C2
:10F1C000E451FF4B108221E0AE016CEE70E4CD0102
:10F1D0000F94D9110E947829811108C021E0AE0155
:10F1E0006CEE70E487E697E30F94D911DF91CF912D
:10F1F00008954F925F926F927F928F929F92AF92FB
:10F20000BF92DF92EF92FF920F931F93CF93DF9302
:10F210001F92CDB7DEB77C014115510509F466C1D7
:10F2200088E08983ACEEB0E420E030E0922FF90171
:10F23000E25CFC4EE491ED932F5F3F4F27303105A8
:10F24000A9F7FA01162FACEEB0E4808113968C93E7
:10F250001397818114968C9302E0090FF901E45110
:10F26000FF4B8CE28083623088F5862F0E9483F901
:10F270008823B1F0812F0E9448F99F938F931F92AA
:10F280001F9382E399E29F938F93E02FF0E0E45184
:10F29000FF4BFF93EF930F94C346CDBFDEBF08C172
:10F2A000812F0E94DBB89F938F931F921F9382E35D
:10F2B00099E29F938F93E02FF0E0E451FF4BFF938F
:10F2C000EF930F94C346CDBFDEBFF2C0663109F0A5
:10F2D00078C086E10E948CF82B013C010E94D5F198
:10F2E0004B015C01672B682B692BF1F4C301B20160
:10F2F00020E13EE040E050E00F947A445F934F936A
:10F300003F932F931F9286E18F9389E399E29F9316
:10F310008F93E02FF0E0E451FF4BFF93EF930F94B6
:10F32000C346CDBFDEBFC4C0802F0E9476B89923EC
:10F3300034F5C301B20120E13EE040E050E00F941B
:10F340007A44CA01B9010F94F216BF92AF929F920C
:10F350008F929F938F937F936F931F9286E18F93EA
:10F3600081E499E29F938F93E02FF0E0E451FF4B0B
:10F37000FF93EF930F94C346CDBFDEBF99C0BF92FA
:10F38000AF929F928F92C301B20120E13EE040E034
:10F3900050E00F947A445F934F933F932F931F92C3
:10F3A00086E18F938EE499E29F938F93E02FF0E0B4
:10F3B000E451FF4BFF93EF930F94C346CDBFDEBFE5
:10F3C00077C0663071F5E02FF0E0E451FF4B86E343
:10F3D00080836894DD24D2F8D90E9D5FE92FF0E098
:10F3E000E451FF4B8CE2808386E00E948CF88B0115
:10F3F0009C018D2D90E04BE0BE016F5F7F4F8451EB
:10F400009F4B0F944B17E981ED0DAE2FB0E0A45147
:10F41000BF4B8DE78C93EF5FF0E0E451FF4B108220
:10F4200047C0653071F5E02FF0E0E451FF4B85E314
:10F4300080836894DD24D2F8D90E9D5FE92FF0E037
:10F44000E451FF4B8CE2808385E00E948CF88B01B5
:10F450009C018D2D90E04BE0BE016F5F7F4F84518A
:10F460009F4B0F949718E981ED0DAE2FB0E0A4519A
:10F47000BF4B8DE78C93EF5FF0E0E451FF4B1082C0
:10F4800017C0862F0E948CF89F938F937F936F9362
:10F490001F921F9389E399E29F938F93802F90E0AF
:10F4A00084519F4B9F938F930F94C346CDBFDEBF74
:10F4B000ECEEF0E401900020E9F73197EC5EF044C7
:10F4C000E983AF01552721E06CEE70E4C7010F948A
:10F4D000D9110E947829811109C0498150E021E0A9
:10F4E0006CEE70E487E697E30F94D9110F90DF91EB
:10F4F000CF911F910F91FF90EF90DF90BF90AF9051
:10F500009F908F907F906F905F904F900895AC0187
:10F510006115710571F1E7E4F3E1ACEEB0E424EFBD
:10F5200030E494919D933196A217B307D1F7FB0174
:10F53000CA01ACEEB0E4208113962C93139721817D
:10F5400014962C93149718961C92189721E048E073
:10F5500050E0BD010F94D9110E947829811109C092
:10F5600021E048E050E06CEE70E487E697E30D940C
:10F57000D9110895EF92FF920F931F93CF93DF93CA
:10F580008C016115710509F47FC04115510509F41D
:10F590007BC0E5E3F3E1ACEEB0E4C4EFD0E49491DA
:10F5A0009D933196AC17BD07D1F7FA017B01CCEEE4
:10F5B000D0E480818B8381818C831F922F938AE595
:10F5C00099E29F938F9384EF90E49F938F930F948E
:10F5D000C34609900020E9F72197CC5ED044F7019B
:10F5E00081810F900F900F900F900F900F908111CD
:10F5F00015C080811F928F9385E791E29F938F932F
:10F60000DD27C451DF4BDF93CF930F94C3460F9098
:10F610000F900F900F900F900F9016C01F928F9326
:10F62000F70180811F928F9382E791E29F938F93DE
:10F63000DD27C451DF4BDF93CF930F94C346EDB763
:10F64000FEB73896EDBFFEBFECEEF0E4019000206F
:10F65000E9F73197EC5EF044EF01DD2721E0AE01E0
:10F660006CEE70E4C8010F94D9110E9478298111C1
:10F670000BC00756174341F021E0AE016CEE70E479
:10F6800087E697E30F94D911DF91CF911F910F91E6
:10F69000FF90EF900895CF93DF93EC014115510552
:10F6A00009F43FC0662361F0E7E4F3E1ACEEB0E4B7
:10F6B00090E024912D939F5F31969730D1F70BC046
:10F6C000EEE3F3E1ACEEB0E490E024912D939F5F84
:10F6D00031969730D1F7DA01CE01ECEEF0E42C91BF
:10F6E000238311962C9124832CE227833CE43087DA
:10F6F000218720E322872DE72387148621E04CE031
:10F7000050E0BF010F94D9110E947829811109C0DE
:10F7100021E04CE050E06CEE70E487E697E30F9454
:10F72000D911DF91CF910895EF92FF920F931F931C
:10F73000CF93DF9300D01F92CDB7DEB70097C9F10A
:10F7400066307105C0F1FC0120812035B1F52181C1
:10F750002C32A9F524812C32A1F57A018C010B5FA2
:10F760001F4FAB01455051099E012F5F3F4FB8011C
:10F770008CE20F942217882349F149815A814B5F0B
:10F780005F4F49835A8346305105E8F045509E014A
:10F790002D5F3F4F60E0C8010F94AA158823B1F098
:10F7A0008B819C818C31910580F4F701808381E00D
:10F7B0000DC080E00BC080E009C080E007C080E0A1
:10F7C00005C080E003C080E001C080E02496CDBF8A
:10F7D000DEBFDF91CF911F910F91FF90EF900895C1
:10F7E000CF92DF92EF92FF920F931F93CF93DF930D
:10F7F000CDB7DEB72C97CDBFDEBF009709F423C18C
:10F800006630710508F421C1FC012081203509F022
:10F810001EC121812C3209F01CC124812C3209F037
:10F820001AC17B018C016C01F5E0CF0ED11CAB013C
:10F83000455051099E012F5F3F4FB6018CE20F9456
:10F840002217982F882309F415C149815A814B5FEB
:10F850005F4F49835A834630510508F4FEC0455036
:10F860009E012D5F3F4F60E0C6010F94AA15982FAF
:10F87000882309F4FFC02B813C812C31310508F02D
:10F88000EEC049815A81DA011196AE15BF0508F024
:10F89000E8C02C31310508F0E6C0F9018827EF54A3
:10F8A000FE4F8F4F0D949644C8018A0F9B1FFC0199
:10F8B00060816D3241F4FA013296EE15FF0508F0D1
:10F8C000D4C040E002C0FD0141E02631310559F4C9
:10F8D0006E2D6E1B9E01275F3F4FC8018E0F9F1F2D
:10F8E0000E94E5E812C02630310541F46E2D6A1BF6
:10F8F000AE01475F5F4F0E94B2EB07C06E2D6A1BDF
:10F90000AE01475F5F4F0E94CEEC882309F4AFC081
:10F9100049855A856B857C858B810E94CEB9982F4D
:10F92000882309F4A7C049855A856B857C858B811E
:10F930000E949FF891E09EC04E2D4A1B9E012B5FB6
:10F940003F4F60E0C8018A0F9B1F0F943516982F18
:10F95000882309F48FC04D815E816F817885498746
:10F960005A876B877C878B810E94CEB9982F88231A
:10F9700009F480C089859A85AB85BC850B97A10564
:10F98000B10541F484EB9AE30E94F32D982F88236C
:10F9900009F470C049855A856B857C858B810E94EE
:10F9A0009FF891E067C04E2D4A1B9E012B5F3F4F91
:10F9B00060E0C8018A0F9B1F0F943516982F88238B
:10F9C00009F458C04D815E816F81788549875A87D7
:10F9D0006B877C878B810E94CEB9982F882349F052
:10F9E00049855A856B857C858B810E949FF891E0C3
:10F9F00041C02B813C81A9014C5051094630510531
:10FA0000C8F549855A856B857C85452B462B472B48
:10FA100089F540E050E0BA01822F0E949FF891E002
:10FA200029C0C7018A1B9B0B899718F56E2D6A1B8D
:10FA3000422FC8018A0F9B1F0E940AF991E0811191
:10FA400019C090E017C090E015C090E013C090E09E
:10FA500011C090E00FC090E00DC090E00BC090E0AE
:10FA600009C090E007C090E005C090E003C090E0BE
:10FA700001C090E0892F2C96CDBFDEBFDF91CF91E2
:10FA80001F910F91FF90EF90DF90CF9008950F930B
:10FA90001F93CF93DF931F921F92CDB7DEB70097CE
:10FAA00041F16630710538F1FC012081203529F5DE
:10FAB00021812C3221F524812C3219F58C01AB01E6
:10FAC00045505109BC016B5F7F4F9E012F5F3F4F37
:10FAD0008CE20F9422178823B9F089819A810596C8
:10FAE000069788F081E0F8019581963469F080E00E
:10FAF0000BC080E009C080E007C080E005C080E066
:10FB000003C080E001C080E00F900F90DF91CF91A3
:10FB10001F910F910895EF92FF920F931F93CF9330
:10FB2000DF9300D000D0CDB7DEB7009709F453C003
:10FB30006630710508F451C0FC012081203509F0C0
:10FB40004EC021812C3209F04CC024812C3209F0A6
:10FB50004AC07B018C01AB0145505109BC016B5F70
:10FB60007F4F9E012F5F3F4F8CE20F942217882317
:10FB700009F442C089819A819C012B5F3F4F298300
:10FB80003A832630310588F1F8012581263479F54C
:10FB900006968E159F0568F54E2D481B9E012D5F1C
:10FBA0003F4F60E0800F911F0F943516882321F19D
:10FBB0006B817C818D819E818B019C01015011099B
:10FBC00021093109073E134021053105A0F40E94A7
:10FBD0005FB981E011C080E00FC080E00DC080E01F
:10FBE0000BC080E009C080E007C080E005C080E075
:10FBF00003C080E001C080E02696CDBFDEBFDF916C
:10FC0000CF911F910F91FF90EF9008950F931F9345
:10FC1000CF93DF93EC016115710509F444C0ACEE9C
:10FC2000B0E420E030E0922FF901E25CFC4EE49178
:10FC3000ED932F5F3F4F27303105A9F7FB01ACEE65
:10FC4000B0E4808113968C931397818114968C93E2
:10FC50001497F901E451FF4B8CE280839E5FE92FFA
:10FC6000F0E0E451FF4B86E49DE7808391831282AC
:10FC7000FD0101900020E9F73197EC5EF0448F011F
:10FC8000112721E0A801BD01CE010F94D9110E94D6
:10FC90007829811108C021E0A8016CEE70E487E6A4
:10FCA00097E30F94D911DF91CF911F910F91089590
:10FCB000FC01892B61F06530710558F08081803539
:10FCC00051F481E091819C3239F080E0089580E028
:10FCD000089580E0089580E00895009799F06330DA
:10FCE000710590F0FC012081203581F421812C32B6
:10FCF00079F424812C3271F485818354823060F050
:10FD000080E0089580E0089580E0089580E00895FF
:10FD100080E0089580E0089581E00895009791F0D3
:10FD20006330710588F0FC012081203579F4218150
:10FD30002C3271F424812C3269F485818F3461F086
:10FD400080E0089580E0089580E0089580E00895BF
:10FD500080E0089580E0089581E00895009791F093
:10FD60006330710588F0FC012081203579F4218110
:10FD70002C3271F424812C3269F48581873561F04D
:10FD800080E0089580E0089580E0089580E008957F
:10FD900080E0089580E0089581E00895CF92DF9299
:10FDA000EF92FF920F931F93CF93DF93411551056D
:10FDB00009F4AFC0009709F4AEC06630710508F4CD
:10FDC000ACC0FC012081203509F0A9C021812C3272
:10FDD00009F0A7C024812C3209F0A5C085818735A0
:10FDE00009F0A3C0EA0184EB9AE30E9494138830DF
:10FDF00009F49DC084EB9AE30E949413863009F4C1
:10FE000098C00F94E6090E948E5061E08AEB9AE355
:10FE10000E9402530E94C7F90E94651C813079F547
:10FE200082E00E9484B86B017C01DD24EE24FF2473
:10FE3000B701A60182E00E949FF8B701A60182E007
:10FE40000E946CB80E947829811119C084E1EEE506
:10FE5000F9E2A7E4B2E401900D928A95E1F7E7E4B4
:10FE6000F2E401900020E9F73197AF014754524482
:10FE700020E067E472E487E697E30F94D911CE019E
:10FE80000E94B41B80E00E9452B89B01AC016894B0
:10FE9000EE24E2F806EB12E2BE01685E7F4FCE016F
:10FEA00006960E945C548D8340E050E0BA01CE017A
:10FEB0000E94A32D8D81882351F182E00E9476B8A3
:10FEC000062F8BE00E9476B821E0611120E046E524
:10FED0005EE3BE016D5C7F4FCE01C5960E94604D12
:10FEE000CE010E948A1B9E01275A3D4FAE01485AFF
:10FEF0005D4FBE016D5A7D4FCE018E5A9D4F0E94BF
:10FF00002A2C0E949A3268E0CE010E9481138D81D2
:10FF100011C080E00FC080E00DC080E00BC080E029
:10FF200009C080E007C080E005C080E003C080E039
:10FF300001C080E0DF91CF911F910F91FF90EF9072
:10FF4000DF90CF900895CF92DF92EF92FF920F93C0
:10FF5000CF93DF934115510509F4B0C0009709F420
:10FF6000AFC06630710508F4ADC0FC0120812035BA
:10FF700009F0AAC021812C3209F0A8C024812C32BA
:10FF800009F0A6C0EA018581833409F493C0843462
:10FF900009F0A0C00E9414B90E9465F984EB9AE3AD
:10FFA0000E949413883009F497C084EB9AE30E946E
:10FFB0009413863009F492C00F94E6090E948E5083
:10FFC00061E08AEB9AE30E9402530E94C7F90E9403
:10FFD000651C813079F582E00E9484B86B017C0158
:10FFE000DD24EE24FF24B701A60182E00E949FF8E1
:10FFF000B701A60182E00E946CB80E9478298111A5
:020000021000EC
:1000000019C084E1EEE5F9E2A7E4B2E401900D92B3
:100010008A95E1F7E7E4F2E401900020E9F73197EF
:10002000AF014754524420E067E472E487E697E367
:100030000F94D91180E00E9452B89B01AC01BE011F
:10004000685E7F4FCE0106960E9496508D8340E0F9
:1000500050E0BA01CE010E94A32D8D81882341F189
:1000600082E00E9476B8062F8BE00E9476B821E0ED
:10007000611120E046E55EE3BE016D5C7F4FCE017D
:10008000C5960E94604DCE010E948A1B9E01275A90
:100090003D4FAE01485A5D4FBE016D5A7D4FCE01B6
:1000A0008E5A9D4F0E942A2C68E0CE010E94811337
:1000B0008D8115C00E9465F981E011C080E00FC0FC
:1000C00080E00DC080E00BC080E009C080E007C088
:1000D00080E005C080E003C080E001C080E0DF91E7
:1000E000CF910F91FF90EF90DF90CF900895BF9246
:1000F000CF92DF92EF92FF920F931F93CF93DF93F4
:100100001F92CDB7DEB76115710509F464C0DB013C
:100110007C01ECEEF0E48BE7808380E781838CE266
:1001200082839C91938311969C91948385839FE411
:100130009683878380E00E9498BF8B019C0148E0F2
:10014000BE016F5F7F4F84EF90E40F94F918E9814F
:10015000E85FD12C0F2EFCE2BF2EF02DCC24C394EF
:10016000CE0EF0E0E451FF4BB082D3948D2D0E946F
:1001700098BF8B019C018C2D90E048E0BE016F5F21
:100180007F4F84519F4B0F94F918E981EC0D83E068
:10019000D812E4CF81E08E0FF0E0E451FF4B9DE7F1
:1001A0009083482F50E0FA01E451FF4B108289837D
:1001B00021E06CEE70E4C7010F94D9110E947829F8
:1001C000811109C0498150E021E06CEE70E487E6BE
:1001D00097E30F94D9110F90DF91CF911F910F9159
:1001E000FF90EF90DF90CF90BF900895CF93DF9373
:1001F00041155105A9F10097A9F165307105A0F1EC
:10020000FC012081203591F521812C3289F5228154
:10021000263481F5EA0184818235E9F0833531F0B5
:10022000843451F50E943EB981E027C00F94E6095D
:10023000BE016D5C7F4FCE01C5960E94654B84EB7D
:100240009AE30E941D2281110F94080ACE010E9498
:1002500012298D8112C0CA01C5960E942FF10DC0CE
:1002600080E00BC080E009C080E007C080E005C0EE
:1002700080E003C080E001C080E0DF91CF9108956D
:10028000FC01892B79F06630710570F0808183352F
:1002900069F481818C3261F481E094819C3249F06F
:1002A00080E0089580E0089580E0089580E008955A
:1002B00080E008950F93CF93DF93009709F476C001
:1002C0006630710508F474C0FC016081633509F083
:1002D00071C061816C3209F06FC064816C3209F0C9
:1002E0006DC04115510509F46BC02115310509F4A4
:1002F00069C08581813309F067C0B901EA01F9015C
:100300001082CA010E940420882309F45FC0CE0134
:100310000E94E51F81112BC0CE010E94122961E0CD
:10032000CE010E94412664E0CE010E94811361E06B
:10033000CE010E94D61F19820E94DF9CE8E2F1E400
:10034000808190E0DC01A85DBE4B25853685880F55
:10035000991FFC01E85DFE4B418152811F960C9173
:1003600061E084EB9AE30E94702481E032C00E9435
:10037000782981112DC083E1E2E7F9E2ACEEB0E427
:1003800001900D928A95E1F7ECEEF0E401900020E7
:10039000E9F73197AF014C5E504421E06CEE70E418
:1003A00087E697E30F94D91181E013C080E011C074
:1003B00080E00FC080E00DC080E00BC080E009C08D
:1003C00080E007C080E005C080E003C081E001C09C
:1003D00081E0DF91CF910F9108950F93CF93DF9339
:1003E000009709F45EC16630710508F45CC1DC0158
:1003F0002C91233509F059C111962C9111972C326B
:1004000009F055C114962C9114972C3209F051C162
:100410004115510509F44FC11596EC918E2F90E0CE
:10042000FC01F097E534F10508F047C1EA0188279F
:10043000E353FE4F8F4F0D949644CA010E949413CC
:10044000843031F0CE010E949413893009F037C115
:10045000CE010E94621FCE010E945EFCCE010E946E
:1004600012290F94E60960E084EB9AE30E9441268A
:1004700063E0CE010E94811319820E94CC9CE8E2C5
:10048000F1E4808190E0DC01A85DBE4B25853685D6
:10049000880F991FFC01E85DFE4B418152811F9638
:1004A0000C9161E084EB9AE30E94702491E016C104
:1004B000CA010E94E51F882309F403C181E08983F2
:1004C00060E0CE010E94781460E0CE010E946614C4
:1004D0000E9478298111F7C080E1E5E8F9E2ACEEED
:1004E000B0E401900D928A95E1F7ECEEF0E4019012
:1004F0000020E9F73197AF014C5E504421E06CEEEB
:1005000070E487E697E30F94D91191E0E7C0CA0140
:100510000E94E51F882309F4D8C060E0CE010E9444
:10052000781460E0CE010E946614FE01EE5AFD4F81
:10053000DE01A85ABD4F8C918083319611968C9123
:10054000808319820E9478298111C1C080E1E5E988
:10055000F9E2ACEEB0E401900D928A95E1F7ECEE91
:10056000F0E401900020E9F73197AF014C5E504470
:1005700021E06CEE70E487E697E30F94D91191E0E7
:10058000ADC0CA010E94E51F982F882309F4A6C0B8
:10059000CE010E94DE2691E08111A0C090E09EC0B5
:1005A000CA010E94E51F882329F0CE010E94682617
:1005B000982F94C00E94EABF91E090C0CA010E94A7
:1005C000E51F982F882309F489C00F94E60960E09D
:1005D00084EB9AE30E94412669E0CE010E948113D8
:1005E0001982CE010E946EFCCE010E941E1CCE011B
:1005F0000F9408010F94EA0C61E0CE010E94D61F0F
:1006000091E06CC0CA010E949413893009F061C066
:1006100066E57EE3CE010F94A500CE010E9465FC45
:100620008D3009F058C0CE010E946EFCCE010F94AF
:1006300008010F94EA0C91E051C0CA010E94941382
:10064000893009F04AC0CE010E945EFCCE010E94B2
:10065000122961E0CE010E94412664E0CE010E9491
:10066000811361E0CE010E94D61F19820E94DF9C97
:10067000E8E2F1E4808190E0DC01A85DBE4B2585D5
:100680003685880F991FFC01E85DFE4B4181528140
:100690001F960C9161E084EB9AE30E94702491E034
:1006A0001DC090E01BC090E019C090E017C090E022
:1006B00015C090E013C090E011C090E00FC091E031
:1006C0000DC091E00BC091E009C091E007C091E03E
:1006D00005C090E003C091E001C090E0892FDF9158
:1006E000CF910F910895FC01892B61F0663071055F
:1006F00058F080818D3451F481E091819C3239F041
:1007000080E0089580E0089580E0089580E00895F5
:10071000FC01892B61F06630710558F080818235CB
:1007200051F481E091819C3239F080E0089580E0BD
:10073000089580E0089580E00895FC01892B61F020
:100740006530710558F080818A3551F481E09181DE
:100750009C3239F080E0089580E0089580E00895AB
:1007600080E00895CF92DF92EF92FF920F931F9354
:10077000CF93DF93CDB7DEB72897CDBFDEBF00970D
:1007800009F457C06530710508F455C0FC0120819B
:100790002A3509F052C021812C3209F050C07B016A
:1007A0008C016C01F2E0CF0ED11CAB01425051091B
:1007B0009E012F5F3F4FB6018CE20F9422178823D2
:1007C00009F446C049815A814E5F5F4F49835A837D
:1007D00043305105B0F142509E012D5F3F4F60E024
:1007E000C6010F94AA15882399F18B819C810397E8
:1007F00050F589819A8101968E159F0530F54E2D11
:10080000481B9E012B5F3F4F60E0800F911F0F94AC
:1008100035168823E9F06D817E818F81988562305D
:1008200071058105910598F48B810E9422D481E0A5
:100830000FC080E00DC080E00BC080E009C080E008
:1008400007C080E005C080E003C080E001C080E018
:100850002896CDBFDEBFDF91CF911F910F91FF9002
:10086000EF90DF90CF9008952F923F924F925F923A
:100870006F927F928F929F92AF92BF92CF92DF92B0
:10088000EF92FF920F931F93CF93DF93CDB7DEB715
:100890006397CDBFDEBF8C01F62E81E08D830115FD
:1008A000110509F423C38093CE2089E10E9476B814
:1008B000672B682B692B09F025C30E9464F4B82EBE
:1008C000811103C0F11020C385C384EB9AE30E9419
:1008D0005720B82E882309F47DC384EB9AE30E9445
:1008E00094138F87F11004C08150823008F400C344
:1008F0002F85243031F484EB9AE30E94562933E0AB
:100900003F870E9468FA0E9451FA84EB9AE30E94A2
:100910001D2281110F94080A84EB9AE30E94122988
:1009200082E00E9476B8E62E8FEF8E0D8A3008F0B6
:10093000E1C2AE014A5F5F4FBE016B5F7F4F8E2DFC
:100940000E9492218E810E948DD38E8184700E949C
:1009500001D48D810E9482F60F2EFCEECF2EF0E4A2
:10096000DF2EF02D8BE7D6018C938DE611968C93BC
:1009700011978CE212968C93129787E713968C93BB
:1009800020E044E050E0B601C8010F94D9111F9255
:10099000EF9285EA99E29F938F93DF92CF920F9423
:1009A000C346F60101900020E9F73197AF014C5E94
:1009B000504420E0B601C8010F94D911EAE9F1E5ED
:1009C00087858F9386858F9385858F9384858F9375
:1009D0000F2EF9EAAF2EF9E2BF2EF02DBF92AF92A3
:1009E000DF92CF920F94C346F60101900020E9F701
:1009F0003197AF014C5E504420E0B601C8010F941E
:100A0000D9118AE00E9476B89F938F937F936F935A
:100A1000BF92AF92DF92CF920F94C346F60101903E
:100A20000020E9F73197AF014C5E504420E0B60159
:100A3000C8010F94D9118BE00E9476B89F938F93D1
:100A40007F936F93BF92AF92DF92CF920F94C34682
:100A5000F60101900020E9F73197AF014C5E504458
:100A600020E0B601C8010F94D9110F2EF4EBCF2E60
:100A7000F1E5DF2EF02DCDBFDEBF412C512C320130
:100A800045010F2EFCEEAF2EF0E4BF2EF02D2BC053
:100A9000D6018C9111969C91119712962C911297D8
:100AA00013963C91B4E0CB0ED11C3F932F939F93B0
:100AB0008F939F928F92BF92AF920F94C346F5018E
:100AC00001900020E9F73197AF014C5E504420E0DF
:100AD000B501C8010F94D911EFEF4E1A5E0A6E0AE4
:100AE0007E0ACDBFDEBF0F94E70C90E0A0E0B0E03F
:100AF000481659066A067B0658F28DE78093EC404B
:100B000021E041E050E06CEE70E4C8010F94D9118F
:100B100065E084EB9AE30E9481130F94E60984EB6D
:100B20009AE30E945B240E943B5660E072E080E002
:100B300090E00E942D5710928F3E1092903E8DE3D0
:100B400091E40E9449A20E94CE588111FCCFB82E98
:100B5000F11004C00E944A1F8823E1F389E00E943B
:100B600076B86F3171058105910508F59B01AC01DF
:100B7000012E1CE0220F331F441F551F1A95D1F779
:100B8000102D2B873C874D875E87CA01B9010E94D3
:100B90000AFA0F94B00A81E00F94000D80E090E112
:100BA000A0E0B0E08F839887A987BA873FC09B01F8
:100BB000AC01012E19E0220F331F441F551F1A9557
:100BC000D1F7102D2B873C874D875E87CA01B9016D
:100BD0000E940AFA0F94B00A0F94300D80E092E060
:100BE000A0E0B0E08F839887A987BA871FC0412C07
:100BF000512C32019F2CCB84DC84ED84FE840F9435
:100C00006D0D8823E1F08D810F94DA086DE371E4B6
:100C10000E94ACA2A82E0F945C0D9FEF491A590AAE
:100C2000690A790AA1100BC0F92C0FC02B853C85ED
:100C30004D855E85232B242B252BC9F606C04C142D
:100C40005D046E047F04D8F2F92C0F94570D8DE3E8
:100C500091E40E9410A3E82E0E94BA570F94130744
:100C6000EE2031F06F8584EB9AE30E948113B2C1CC
:100C700086E693E40E9419C5882351F0F11008C05C
:100C80006091654470E086E693E40E9470A309C019
:100C9000ECEEF0E41082118262E070E0CF010E947D
:100CA00070A360E072E080E090E00E9443560E94F2
:100CB000CE588111FCCF8B859C85AD85BE85892B57
:100CC0008A2B8B2B09F4F3C0C12CD12C76010F2E6B
:100CD000FCEE2F2EF0E43F2EF02D4F8058846984D7
:100CE0007A8491E0491A5108610871080E945FA353
:100CF00080938F3E9093903EAE014F5F5F4FBC015B
:100D00008D810E948A14882309F463C1C701B6014A
:100D10002F81388549855A850F9458444B015C01D1
:100D2000672B682B692BA1F5C701B6012F81388588
:100D300049855A850F945844288B398B4A8B5B8B95
:100D400089E00E9476B8AB89AF93BA89BF93E989ED
:100D5000EF93F889FF939F938F937F936F932EEA7E
:100D600039E23F932F933F922F920F94C346F101A4
:100D700001900020E9F73197AF014C5E504420E02C
:100D8000B101C8010F94D9111092CE20CDBFDEBFA2
:100D90002F81388549855A85211582E0380741051C
:100DA000510509F4BAC0211530414105510509F436
:100DB000DDC0D701C60187709927AA27BB27892BD9
:100DC0008A2B8B2B09F043C08C818F938B818F935F
:100DD0008A818F9389818F93A6EFB9E2BF93AF93F6
:100DE0003F922F920F94C346F10101900020E9F742
:100DF0003197AF014C5E504420E0B101C8010F941F
:100E0000D911C701B6012F81388549855A850F94BC
:100E100058442F5F3F4F4F4F5F4F6F8178858985D3
:100E20009A850F941644CDBFDEBFA7019601285FB7
:100E30003F4F4F4F5F4F621773078407950719F4B1
:100E40001092CE20C0C031E03093CE20BCC01092B2
:100E5000CE2084149504A604B70479F4EDE7D101FB
:100E6000EC9321E041E050E0B101C8010F94D911A9
:100E70000FC0ECE2D101EC9304C08091CE20882316
:100E800039F020E041E050E0B101C8010F94D911E0
:100E9000FFEFCF1ADF0AEF0AFF0A2B853C854D854D
:100EA0005E85C216D306E406F50609F01FCF0E9440
:100EB0000E570F9413070F94A21A86E59EE30F9422
:100EC000683C6F8584EB9AE30E9481130E94DFFAED
:100ED00084EB9AE30E941D2281110F94080A84EB8F
:100EE0009AE30E941229BB24B39474C0B12C72C03F
:100EF000B12C70C0B12C6EC084EB9AE30E949413A5
:100F00008F87F6CCFF24F39484EB9AE30E9457205A
:100F1000B82E882309F45EC0EFCF8C818F938B812C
:100F20008F938A818F9389818F9346EF59E25F93E4
:100F30004F933F922F920F94C346F10101900020EE
:100F4000E9F73197AF014C5E504420E0B101C80190
:100F50000F94D91191E09093CE20CDBFDEBF4814FD
:100F600059046A047B0409F084CF78CF8C818F9375
:100F70008B818F938A818F9389818F93E6EFF9E23A
:100F8000FF93EF933F922F920F94C346F10101908C
:100F90000020E9F73197AF014C5E504420E0B101E9
:100FA000C8010F94D91131E03093CE20CDBFDEBF00
:100FB000481459046A047B0409F05BCF4FCFECE27C
:100FC000D101EC935ACF84149504A604B704B9F761
:100FD00045CFB82E8B2D6396CDBFDEBFDF91CF916D
:100FE0001F910F91FF90EF90DF90CF90BF90AF9047
:100FF0009F908F907F906F905F904F903F902F9039
:101000000895CF92DF92EF92FF921F93CF93DF93D9
:101010006115710509F474C04630510508F472C0B9
:10102000DB01EC91ED3409F06FC01196EC91EC32DC
:1010300009F06CC02115310509F46AC0009709F464
:1010400069C069017A01EB012D81203341F440E050
:1010500060E00ADC11E0811160C010E05EC0233561
:1010600041F5C6010E946420182F882309F455C059
:10107000C7010697029718F40E9431A40CC08E8114
:101080008C3219F00E9431A406C069EF6E0DCE01BA
:1010900007960E94FCA3A601485E5F4FB6016B5CF9
:1010A0007F4F80E00E94F84611E0811136C010E0C9
:1010B00034C00E947829182F81112EC08D811F9273
:1010C0008F938AEB99E29F938F93CCEED0E4DF93DA
:1010D000CF930F94C34609900020E9F72197AE0102
:1010E0004C5E504421E06CEE70E487E697E30F9489
:1010F000D9110F900F900F900F900F900F900DC07F
:1011000010E00BC010E009C010E007C010E005C0FF
:1011100010E003C010E001C010E0812FDF91CF91FB
:101120001F91FF90EF90DF90CF900895FC01892BE5
:10113000A9F068307105A0F08081813599F4818132
:101140008C3291F484818C3289F486818C3281F4E2
:1011500081E09581903369F080E0089580E0089502
:1011600080E0089580E0089580E0089580E008958B
:1011700080E00895EF92FF920F931F93CF93DF9338
:1011800000D0CDB7DEB79CE29B8321153105A9F1D4
:1011900061157105A1F1FA013197F39790F582334A
:1011A00090F5803391F5C9017A018B010E94941367
:1011B000843069F59E012F5F3F4F41E050E0BE0152
:1011C0006D5F7F4F86E59EE30F94BA3A9E012F5FD5
:1011D0003F4FA701B80186E59EE30F94BA3A86E532
:1011E0009EE30F94683C0F949F0C81E99EE30E945C
:1011F000F99B0F94750B81E00BC080E009C080E083
:1012000007C080E005C080E003C081E001C080E04D
:101210002396CDBFDEBFDF91CF911F910F91FF903D
:10122000EF900895FC01892B61F06330710558F04F
:1012300080818C3451F481E091819C3239F080E0DE
:10124000089580E0089580E0089580E00895452B9A
:10125000B1F00097B1F0672BB1F0FC0185818136C8
:10126000A1F486ED9FE30E942C9C811110C060E0E8
:1012700070E086ED9FE30E94379C81E0089580E056
:10128000089580E0089580E0089580E0089580E06A
:101290000895CF93DF93452B41F1009741F16531DC
:1012A000710538F1FC012581203729F5278120338C
:1012B00019F41092E43F09C0213321F421E0209376
:1012C000E43F03C022E02093E43FEC0186ED9FE37E
:1012D0000E942C9C811111C0BE01675F7F4F86ED7B
:1012E0009FE30E94379C81E009C080E007C080E056
:1012F00005C080E003C080E001C080E0DF91CF91B5
:101300000895CF93DF93452B61F1009761F165312B
:10131000710558F1FC0125812E3649F527812033CE
:1013200019F41092E43F09C0213321F421E0209305
:10133000E43F03C022E02093E43FEC0186ED9FE30D
:101340000E942C9C811115C08091E43F882399F064
:10135000BE01675F7F4F86ED9FE30E94589C81E04E
:101360000BC080E009C080E007C080E005C080E0DD
:1013700003C080E001C081E0DF91CF910895009724
:1013800099F06630710590F0FC018581833681F417
:1013900086ED9FE30E942C9C882361F00E94CE9AE8
:1013A0001092D63F81E0089580E0089580E008958E
:1013B00080E0089581E00895FC01892B49F06630B2
:1013C000710540F081E09581933729F080E0089520
:1013D00080E0089580E00895FC01892B49F0663093
:1013E000710540F081E09581953629F080E00895FF
:1013F00080E0089580E00895BF92CF92DF92EF924F
:10140000FF920F931F93CF93DF9300D0CDB7DEB73A
:101410009CE29B83882359F00091C43F002311F084
:1014200010E009C00091913E1091923E04C00091DD
:10143000C53F1091C63F0D3291E0190710F00CE244
:1014400011E00115110509F44CC0B82E9E012F5F63
:101450003F4F41E050E0BE016D5F7F4F86E59EE368
:101460000F94BA3A1092933E1092943E20E030E0EE
:10147000C12CD12C0F2EF1E9EF2EFEE3FF2EF02D23
:10148000F901EF56F14C95819B839E012F5F3F4FF1
:1014900041E050E0BE016D5F7F4F86E59EE30F9413
:1014A000BA3A29813A81232B19F4EFEFCE1ADE0ADA
:1014B000F701228133812F5F3F4F2283338320172F
:1014C0003107F0F286E59EE30F94683CB11004C04A
:1014D0001092C53F1092C63F81E0CD2819F080E000
:1014E00001C080E02396CDBFDEBFDF91CF911F9179
:1014F0000F91FF90EF90DF90CF90BF900895FC0187
:10150000892B49F06630710540F081E09581943671
:1015100029F080E0089580E0089580E00895ECEEE1
:10152000F0E42BE720832CE621832CE22283662340
:1015300021F02FE62093EF4003C025E62093EF40F3
:10154000ECEEF0E42DE72483158221E045E050E045
:10155000BF010F94D9110E947829811109C021E09F
:1015600045E050E06CEE70E487E697E30D94D91106
:101570000895EF92FF920F931F93CF93DF9361151E
:10158000710509F410C2009709F40DC2FB01208116
:10159000222309F408C2EB018C010E9478298111F1
:1015A00025C088811F928F938FEB99E29F938F9331
:1015B0000F2EF7E4EF2EF2E4FF2EF02DFF92EF92C4
:1015C0000F94C346F70101900020E9F73197AF016E
:1015D0004754524421E0B70187E697E30F94D911AD
:1015E0000F900F900F900F900F900F90888190E0C8
:1015F0008A30910508F0D1C1FC018827EE5EFD4FCD
:101600008F4F0D9496448FE09DE30E948A9A0F9429
:10161000B00A0AEE10E41EC068E670E48FE09DE3B5
:101620000F948511F80180818130A1F40E947829FE
:1016300081110BC0409168405091694021E06AE6F9
:1016400070E487E697E30F94D91188E690E40F944D
:10165000761107C00F94C70A683873418105910558
:10166000D8F289819FEF980F983020F088818F5FA2
:10167000888399C1888397C1ECEEF0E483E5808389
:101680008DE481838CE282838E85823021F481E334
:101690008093EF4003C080E38093EF401092F040CE
:1016A00021E044E050E06CEE70E48FE09DE30F94A5
:1016B000D91188818F5F88830F94B00ACAEED0E475
:1016C0001DC068E670E48FE09DE30F94851188816A
:1016D0008130A1F40E94782981110BC040916840AB
:1016E0005091694021E06AE670E487E697E30F9441
:1016F000D91188E690E40F94761155C10F94C70A6A
:101700006233710581059105E0F24DC1ECEEF0E424
:1017100083E5808380E581838CE282838E858111DD
:101720000CC081E3838382E3848383E3858384E342
:10173000868388818F5F88831AC0813059F4ECEEEC
:10174000F0E480E3838384838583868388818F5F4D
:1017500088830DC0ECEEF0E481E3838382E384832D
:1017600083E3858384E3868388818F5F88831092F7
:10177000F34021E047E050E06CEE70E48FE09DE341
:101780000F94D9110F94B00ACAEED0E41DC068E6D8
:1017900070E48FE09DE30F94851188818130A1F47E
:1017A0000E94782981110BC0409168405091694096
:1017B00021E06AE670E487E697E30F94D91188E6A2
:1017C00090E40F947611EFC00F94C70A623371054D
:1017D00081059105E0F2E7C0ECEEF0E483E580835B
:1017E00082E581838CE28283DE011296EFEEF0E4E3
:1017F0002BEF30E48D918193E217F307D9F7109224
:10180000FB4021E04FE050E06CEE70E48FE09DE3A0
:101810000F94D91188818F5F88830F94B00ACAEE24
:10182000D0E41DC068E670E48FE09DE30F9485115D
:1018300088818130A1F40E94782981110BC04091E8
:1018400068405091694021E06AE670E487E697E3DA
:101850000F94D91188E690E40F947611A4C00F94E8
:10186000C70A6233710581059105E0F29CC0ECEE78
:10187000F0E482E580838CE2818381E382831382BA
:1018800021E043E050E0BF018FE09DE30F94D911C8
:1018900088818F5F888387C08FE09DE30E948A9A4A
:1018A0000F94B00A0AEE10E41EC068E670E48FE000
:1018B0009DE30F948511F80180818130A1F40E948D
:1018C000782981110BC0409168405091694021E016
:1018D0006AE670E487E697E30F94D91188E690E40E
:1018E0000F94761107C00F94C70A62337105810502
:1018F0009105D8F288818F5F888355C0ECEEF0E4C3
:1019000083E480838CE28183DE011296EEEEF0E4C4
:101910002AEF30E48D918193E217F307D9F7109203
:10192000FA4021E04EE050E06CEE70E48FE09DE381
:101930000F94D91188818F5F88830F948D0633C0EF
:101940000E94AE9C882361F061E0C801E8DD0F943D
:101950008D068FE09DE30E94AC9A1882198223C005
:101960000F94790681319742F0F060E0C801D7DD2D
:101970000F948D068FE09DE30E94AC9A1882198225
:1019800012C00F947906883E934068F00E94DF9A57
:101990000F948D061882198206C08FE09DE30E9485
:1019A000AC9A18821982DF91CF911F910F91FF900D
:1019B000EF900895ECEEF0E42BE720832CE62183F2
:1019C0002CE22283605D63832DE72483158221E06E
:1019D00045E050E0BF010F94D9110E947829811190
:1019E00009C021E045E050E06CEE70E487E697E343
:1019F0000D94D9110895DF92EF92FF920F931F93E8
:101A0000CF93DF93009709F481C1EC01888190E0C6
:101A10008931910508F075C1FC018827E45EFD4F0E
:101A20008F4F0D9496448EE698E30E948A9A88819F
:101A30008F5F88836BC1ECEEF0E487E480838BE4F6
:101A40008183128221E042E050E0BF018EE698E3FC
:101A50000F94D91188818F5F888385EE9FE30F945F
:101A6000761122968CE0FE0111928A95E9F74EC11B
:101A70000F94B00AF12C07E610E429C065EE7FE36D
:101A80008EE698E30F948511F80180818130F9F496
:101A90008091E53F9091E63F059731F48091E73FD3
:101AA000813311F4FF24F3940E94782981110BC033
:101AB0004091E53F5091E63F21E067EE7FE387E606
:101AC00097E30F94D91185EE9FE30F9476110F944D
:101AD000C70A623371058105910580F2FF2021F06C
:101AE00088818F5F888312C188E088830FC1ECEE04
:101AF000F0E487E4808386E48183148221E042E07D
:101B000050E0BF018EE698E30F94D91188818F5F72
:101B10008883FCC00F94B00AD12C07E610E40F2E86
:101B2000F3EFEF2EFFE3FF2EF02D2EC065EE7FE3E7
:101B30008EE698E30F948511F8018081813021F5BC
:101B40008091E53F9091E63F0C9759F4E7EEFFE373
:101B5000DE01129681918D93EE15FF05D9F7DD24F4
:101B6000D3940E94782981110BC04091E53F509198
:101B7000E63F21E067EE7FE387E697E30F94D91114
:101B800085EE9FE30F9476110F94C70A62337105B7
:101B90008105910558F2DD2021F088818F5F8883CF
:101BA000B5C088E08883B2C0ECEEF0E483E58083C2
:101BB00082E581838CE28283DE011296EFEEF0E40F
:101BC0002BEF30E48D918193E217F307D9F7109250
:101BD000FB4021E04FE050E06CEE70E48EE698E3CD
:101BE0000F94D91188818F5F888390C0ECEEF0E468
:101BF00083E580838DE481838CE2828386E3838323
:101C0000148221E044E050E0BF018EE698E30F9497
